:100000000C94FF180C942A190C942A190C942A1990
:100010000C942A190C942A190C942A190C942A1954
:100020000C942A190C942A190C942A190C942A1944
:100030000C942A190C94AC190C942A190C942A19B2
:100040000C942A190C945D7F0C942A190C942A198B
:100050000C942A190C942A190C942B880C940B1AC2
:100060000C942A190C94D0540C942A190C942A1923
:100070000C942A190C942A190C942A190C942A19F4
:100080000C942A190C942A190C942A190C942A19E4
:100090000C942A190C942A190C942A190C948D9AF0
:1000A0000C942A190C942A190C942A190C942A19C4
:1000B0000C942A190C942A190C942A190C942A19B4
:1000C0000C942A190C942A190C942A190C942A19A4
:1000D0000C942A190C942A190C942A190C942A1994
:1000E0000C942A19084AD73B3BCE016E84BCBFFD55
:1000F000C12F3D6C74319ABD56833DDA3D00C77FF8
:1001000011BED9E4BB4C3E916BAAAABE0000008090
:100110003F05A84CCDB2D44EB93836A9020C50B91F
:10012000918688083CA6AAAA2ABE000000803F0249
:1001300000002100240027002A002D003000330099
:1001400001010000040107010A010000220025004E
:1001500028002B002E0031003400020100000501B0
:1001600008010B01000020002300260029002C00BC
:100170002F003200000100000301060109010505FE
:100180000505070508080808020202020A0A08080D
:10019000040404040101010101010101030303033B
:1001A00003030303040707070C0C0C0C0C0C0C0CCA
:1001B0000202020206060606060606060B0B0B0BDB
:1001C0000B0B0B0B01021020200808102040102000
:1001D000408002010201080402010102040810200B
:1001E0004080804020100804020180040201804009
:1001F0002010080402010804020101020408102072
:10020000408001020408102040800000090A020812
:100210000B0C0D07060304010000000000000000A5
:1002200000000000000000000000000000000000CE
:1002300000000000000011100F000000000000008E
:1002400000000000000000000000000000000000AE
:100250004D383420582059205A2045006563686F76
:100260003A0043616E6E6F7420656E746572207320
:1002700075626469723A20004D3234004D32332089
:100280002573006175746F25692E67004572726F62
:10029000723A006572726F722077726974696E6764
:1002A00020746F2066696C6500436172642065721A
:1002B000726F723A004E6F74205344207072696EF0
:1002C00074696E67002F005344207072696E746900
:1002D0006E67206279746520002E0044656C657439
:1002E000696F6E206661696C65642C2046696C6577
:1002F0003A200046696C652064656C657465643AF3
:10030000002E006F70656E206661696C65642C203C
:1003100046696C653A200057726974696E6720748B
:100320006F2066696C653A20002E006F70656E2044
:100330006661696C65642C2046696C653A20002E04
:10034000006F70656E206661696C65642C2046697B
:100350006C653A200046696C652073656C65637452
:100360006564002053697A653A200046696C65200F
:100370006F70656E65643A20002E006F70656E20A8
:100380006661696C65642C2046696C653A2000538F
:10039000442063617264206F6B006F70656E526FF2
:1003A0006F74206661696C656400766F6C756D654D
:1003B0002E696E6974206661696C6564005344201F
:1003C000696E6974206661696C006563686F3A00E4
:1003D00048617264636F6465642044656661756C2E
:1003E000742053657474696E6773204C6F61646523
:1003F000640053746F7265642073657474696E670A
:10040000732072657472696576656400204400200B
:1004100049002020204D33303120500050494420E5
:1004200073657474696E67733A00205A002059002E
:1004300020204D323036205800486F6D65206F66A1
:100440006673657420286D6D293A00204500205A96
:100450000020580020420020540020204D3230352A
:10046000205300416476616E636564207661726931
:1004700061626C65733A20533D4D696E2066656517
:10048000647261746520286D6D2F73292C20543D92
:100490004D696E2074726176656C20666565647264
:1004A00061746520286D6D2F73292C20423D6D6984
:1004B0006E696D756D207365676D656E7420746906
:1004C0006D6520286D73292C20583D6D6178696D0C
:1004D000756D205859206A65726B20286D6D2F73D9
:1004E000292C20205A3D6D6178696D756D205A2048
:1004F0006A65726B20286D6D2F73292C2020453D75
:100500006D6178696D756D2045206A65726B202874
:100510006D6D2F73290020540020204D323034207F
:100520005300416363656C65726174696F6E3A2054
:10053000533D616363656C65726174696F6E2C20F5
:10054000543D7265747261637420616363656C65A8
:10055000726174696F6E00204500205A00205900B6
:1005600020204D3230312058004D6178696D756D15
:1005700020416363656C65726174696F6E20286DDC
:100580006D2F7332293A00204500205A002059006F
:1005900020204D3230332058004D6178696D756DE3
:1005A0002066656564726174657320286D6D2F73B4
:1005B000293A00204500205A0020590020204D39BA
:1005C0003220580053746570732070657220756E08
:1005D00069743A0053657474696E67732053746F5D
:1005E000726564006563686F3A004572726F723AB3
:1005F000005072696E7465722073746F70706564F8
:100600002064756520746F206572726F72732E207E
:1006100046697820746865206572726F7220616E19
:100620006420757365204D39393920746F207265E7
:1006300073746172742E202854656D7065726174D4
:100640007572652069732072657365742E20536519
:1006500074206974206166746572207265737461B8
:100660007274696E6729005072696E7465722068D1
:10067000616C7465642E206B696C6C282920636141
:100680006C6C656421006F6B00526573656E643A33
:1006900020002200556E6B6E6F776E20636F6D6D5C
:1006A000616E643A20220020423A300020423A3102
:1006B000006F6B20523A002200556E6B6E6F776EA2
:1006C00020636F6D6D616E643A2022007A5F6D6108
:1006D000783A2000795F6D61783A2000785F6D6923
:1006E0006E3A20005A3A00593A0020436F756E74F2
:1006F00020583A2000453A005A3A00593A00583AF0
:10070000004649524D574152455F4E414D453A4D85
:1007100061726C696E2056313B20537072696E7441
:1007200065722F6772626C206D61736875702066E8
:100730006F722067656E36204649524D57415245CB
:100740005F55524C3A687474703A2F2F6669726D17
:10075000776172652E756C74696D616B65722E635D
:100760006F6D2050524F544F434F4C5F564552537C
:10077000494F4E3A312E30204D414348494E455F56
:10078000545950453A556C74696D616B65722045DA
:10079000585452554445525F434F554E543A310ACE
:1007A0000020423A0020453A00543A0020573A00CF
:1007B00020453A00543A002042403A0020403A0096
:1007C000202F0020423A00202F006F6B20543A0067
:1007D0002569206D696E2C202569207365630045AD
:1007E0006E642066696C65206C697374004265678D
:1007F000696E2066696C65206C6973740000000086
:100800000000006643000066430000000000000096
:100810000000000000000066430000664300006620
:10082000430000664300006643000066430000A0EA
:10083000400000A04000004040FF01012569206801
:100840006F757273202569206D696E75746573000C
:10085000446F6E65207072696E74696E6720666998
:100860006C65005072696E7465722073746F70707D
:1008700065642064756520746F206572726F727391
:100880002E2046697820746865206572726F722028
:10089000616E6420757365204D39393920746F207D
:1008A000726573746172742E202854656D70657260
:1008B00061747572652069732072657365742E208A
:1008C0005365742069742061667465722072657363
:1008D00074617274696E6729006F6B004E6F204CF3
:1008E000696E65204E756D62657220776974682047
:1008F000636865636B73756D2C204C617374204C59
:10090000696E653A20004E6F20436865636B7375AE
:100910006D2077697468206C696E65206E756D62F4
:1009200065722C204C617374204C696E653A20000E
:10093000636865636B73756D206D69736D61746356
:10094000682C204C617374204C696E653A20004C11
:10095000696E65204E756D626572206973206E6FD9
:1009600074204C617374204C696E65204E756D6205
:1009700065722B312C204C617374204C696E653A82
:1009800020004D31313000446F6E6520736176690F
:100990006E672066696C652E006F6B004D32390002
:1009A0002020506C616E6E6572427566666572429B
:1009B000797465733A20002046726565204D656D37
:1009C0006F72793A20004A616E202039203230312E
:1009D0003400436F6D70696C65643A20005665722F
:1009E00073696F6E2031342E30312E3100207C201F
:1009F000417574686F723A20004A616E2020392078
:100A0000323031342031323A34313A333600204CEE
:100A100061737420557064617465643A2000312EEE
:100A2000302E30004D61726C696E200020536F666D
:100A30007477617265205265736574002057617424
:100A40006368646F67205265736574002042726F3B
:100A5000776E206F75742052657365740020457839
:100A60007465726E616C20526573657400506F77A7
:100A700065725570007374617274002200656E7146
:100A80007565696E672022002200656E7175656963
:100A90006E672022006563686F3A0020746F6F20D4
:100AA0006C6F6E6720657874727573696F6E2070F5
:100AB000726576656E7465640020636F6C64206592
:100AC0007874727573696F6E2070726576656E7476
:100AD00065640000002110422063308440A550C6A8
:100AE00060E770088129914AA16BB18CC1ADD1CE6C
:100AF000E1EFF13112100273325222B5529442F7F3
:100B000072D662399318837BB35AA3BDD39CC3FFBB
:100B1000F3DEE36224433420040114E664C774A4C2
:100B20004485546AA54BB528850995EEE5CFF5AC0B
:100B3000C58DD55336722611163006D776F66695D2
:100B400056B4465BB77AA719973887DFF7FEE79D5B
:100B5000D7BCC7C448E5588668A778400861180222
:100B6000282338CCC9EDD98EE9AFF9488969990AAB
:100B7000A92BB9F55AD44AB77A966A711A500A3332
:100B80003A122AFDDBDCCBBFFB9EEB799B588B3BFB
:100B9000BB1AABA66C877CE44CC55C222C033C6082
:100BA0000C411CAEED8FFDECCDCDDD2AAD0BBD684B
:100BB0008D499D977EB66ED55EF44E133E322E5112
:100BC0001E700E9FFFBEEFDDDFFCCF1BBF3AAF599B
:100BD0009F788F8891A981CAB1EBA10CD12DC14E0C
:100BE000F16FE18010A100C230E32004502540469F
:100BF000706760B9839893FBA3DAB33DC31CD37FBE
:100C0000E35EF3B1029012F322D2323542145277EE
:100C1000625672EAB5CBA5A89589856EF54FE52C8D
:100C2000D50DC5E234C324A014810466744764243E
:100C3000540544DBA7FAB79987B8975FE77EF71D9D
:100C4000C73CD7D326F2369106B01657667676158E
:100C50004634564CD96DC90EF92FE9C899E9898AED
:100C6000B9ABA94458654806782768C018E10882DE
:100C700038A3287DCB5CDB3FEB1EFBF98BD89BBBFD
:100C8000AB9ABB754A545A376A167AF10AD01AB32E
:100C90002A923A2EFD0FED6CDD4DCDAABD8BADE84D
:100CA0009DC98D267C076C645C454CA23C832CE07E
:100CB0001CC10C1FEF3EFF5DCF7CDF9BAFBABFD9DD
:100CC0008FF89F176E367E554E745E932EB23ED1CE
:100CD0000EF01E7C3C3E5E2B3D3F2F5B5D3B2C2A85
:100CE000225C0045313A200045303A20005A3A2033
:100CF00000593A2000583A20004D53312C4D5332C0
:100D00002050696E730A0024F404D9201BC40C5CC3
:100D10000E9804C4095F0265077101F405F900FB30
:100D200004B30048048700C1036900580355000359
:100D3000034500BE023A008402310053022A002912
:100D400002250004022000E4011C00C8011900AFC4
:100D50000117009801140084011300710110006153
:100D600001100051010E0043010D0036010B002B54
:100D7000010B0020010B00150109000C0109000303
:100D8000010800FB000800F3000800EB000700E486
:100D9000000600DE000600D8000600D2000600CCE7
:100DA000000500C7000500C2000500BD000400B931
:100DB000000400B5000400B1000400AD000400A967
:100DC000000400A5000300A20003009F0004009B94
:100DD00000030098000300950002009300030090B8
:100DE0000003008D0002008B0003008800020086D3
:100DF00000020084000300810002007F0002007DE9
:100E00000002007B000200790002007700010076FA
:100E10000002007400020072000100710002006F05
:100E20000002006D0001006C0002006A0001006910
:100E30000002006700010066000100650001006417
:100E40000002006200010061000100600001005F1B
:100E50000002005D0001005C0001005B0001005A1F
:100E60000001005900010058000100570001005620
:100E70000001005500010054000100530000005320
:100E80000001005200010051000100500001004F1C
:100E90000001004E0000004E0001004D0001004C1A
:100EA0000001004B0000004B0001004A0001004916
:100EB0000001004800000048000100470001004612
:100EC000000000460001004500000045000100440C
:100ED0000001004300000043000100420000004206
:100EE0000001004100000041000100400001003FFE
:100EF0000000003F0001003E0000003E0001003DF8
:100F00000000003D0001003C0000003C0000003CEF
:100F10000001003B0000003B0001003A0000003AE5
:100F200000010039000000390001003800000038DD
:100F300000000038000100370000003700010036D3
:100F400000000036000000360001003500000035CA
:100F500000000035000100340000003400000034BF
:100F600000010033000000330000003300010032B4
:100F700000000032000000320001003100000031AA
:100F8000000000310001003000000030000000309F
:100F90000001002F0000002F0000002F0000002F94
:100FA0000001002E0000002E0000002E0001002D88
:100FB0000000002D0000002D0000002D0001002C7D
:100FC0000000002C0000002C0000002C0001002B71
:100FD0000000002B0000002B0000002B0001002A65
:100FE0000000002A0000002A0000002A0001002959
:100FF000000000290000002900000029000000294D
:10100000000100280000002800000028000000283F
:101010000000002800010027000000270000002732
:101020000000002700000027000100260000002625
:101030000000002600000026000000260001002518
:10104000000000250000002500000025000000250C
:1010500000000025000100240000002400000024FE
:1010600000000024000000240001002300000023F1
:1010700000000023000000230000002300000023E4
:1010800000000023000100220000002200000022D6
:1010900000000022000000220000002200010021C8
:1010A00000000021000000210000002100000021BC
:1010B00000000021000000210001002000000020AD
:1010C00000000020000000200000002000000020A0
:1010D00000000020000000200001001F0000001F91
:1010E0000000001F0000001F0000001F0000001F84
:1010F0000000001F0001001E0000001E0000001E76
:101100000000001E00000024F4D43050C38E20C222
:10111000A24017828B7011127A910D816CD90AA8A6
:1011200061E108C7586607615143061E4B5D05C162
:1011300045A7041A411104093D9803713931034050
:1011400036DB0265339102D4305402802E1D0263D7
:101150002CEE01752AC501B028A001102781018F4E
:101160002564012B244B01E0223401AC211F018DA9
:10117000200D01801FFC00841EED00971DDF00B8CC
:101180001CD200E61BC600201BBC00641AB200B2D1
:1011900019A8000A19A0006A189900D117910040F7
:1011A000178B00B516840031167E00B31579003A0E
:1011B000157300C7146F0058146A00EE1366008898
:1011C00013630025135E00C7125B006C12570015F5
:1011D000125400C111510070114F0021114B00D663
:1011E0001049008D1047004610440002104200C014
:1011F0000F4000800F3E00420F3C00060F3B00CB2B
:101200000E3800930E37005C0E3500270E3400F3C5
:101210000D3200C10D3100900D3000600D2E0032F6
:101220000D2D00050D2C00D90C2B00AE0C290085CE
:101230000C29005C0C2700350C27000E0C2600E85A
:101240000B2400C40B2400A00B23007D0B23005AA9
:101250000B2100390B2100180B2000F80A1F00D9C0
:101260000A1E00BB0A1E009D0A1D00800A1D0063A5
:101270000A1C00470A1B002C0A1B00110A1A00F75F
:10128000091A00DD091900C4091900AB09190092F7
:101290000917007B091800630917004C091600366E
:1012A000091600200916000A091500F5081500E0C6
:1012B000081400CC081400B8081400A40814009006
:1012C0000813007D0812006B08130058081200462E
:1012D000081200340811002308110012081100013F
:1012E000081100F0071000E0071000D0071000C040
:1012F000071000B0070F00A107100091070E008330
:10130000070F0074070F0065070E0057070E00490E
:10131000070E003B070D002E070E0020070D0013DF
:10132000070D0006070D00F9060C00ED060D00E0A4
:10133000060C00D4060C00C8060C00BC060C00B05D
:10134000060C00A4060B0099060C008D060B00820B
:10135000060B0077060B006C060B0061060A0057AF
:10136000060B004C060A0042060A0038060A002E48
:10137000060A0024060A001A060A001006090007D9
:10138000060A00FD050900F4050900EB050900E265
:10139000050900D9050900D0050900C7050900BEE7
:1013A000050900B5050800AD050800A50509009C64
:1013B000050800940508008C050800840508007CD9
:1013C000050800740508006C050700650508005D48
:1013D000050700560508004E0507004705070040B1
:1013E00005080038050700310507002A0507002316
:1013F0000507001C050600160507000F0507000875
:1014000005060002050700FB040600F5040700EED0
:10141000040600E8040600E2040700DB040600D529
:10142000040600CF040600C9040600C3040600BD7C
:10143000040600B7040600B1040500AC040600A6CB
:10144000040600A00405009B040600950405009016
:101450000406008A04050085040500800406007A5D
:1014600004050075040500700405006B04050066A2
:10147000040500610405005C0405005704050052E2
:101480000405004D04050048040500430405003E22
:101490000404003A04050035040500300404002C5F
:1014A00004050027040400230405001E0404001A98
:1014B00004040016040500110404000D04040009CE
:1014C0000405000404040000040400FC030400F804
:1014D000030400F4030400F0030400EC030400E838
:1014E000030400E4030400E0030400DC030400D868
:1014F000030400D4030400D0030400CC030400C898
:10150000030300C50303006563686F3A00205A3A7D
:101510000020593A0020583A00656E6473746F7069
:1015200073206869743A20004572726F723A0054F1
:10153000656D70657261747572652068656174654A
:101540006420626564207377697463686564206FE2
:1015500066662E204D415854454D5020747269677F
:101560006765726564202121003A204578747275A0
:10157000646572207377697463686564206F66665A
:101580002E204D494E54454D502074726967676551
:101590007265642021003A20457874727564657222
:1015A000207377697463686564206F66662E204DCA
:1015B000415854454D50207472696767657265647F
:1015C000202100202D20496E76616C6964206578A9
:1015D000747275646572206E756D6265722021008B
:1015E00000000000300E0100C00E0A00500F140071
:1015F000D00F1E0060102800E010320070113C0077
:10160000F01146007012500000135A00801364005D
:1016100000146E00901478001015820090158C0054
:10162000101696009016A0001017AA009017B4008C
:101630001018BE009018C8001019D2009019DC00D4
:10164000101AE600801AF000001BFA00801B04014B
:10165000F01B0E01701C1801F01C2201601D2C01F2
:10166000E01D3601501E4001D01E4A01401F5401AA
:10167000B01F5E0130206801A020720110217C01A2
:1016800090218601002290016026F401902A5802E0
:10169000802EBC0250322003E03584035039E80329
:1016A000803C4C04504944204175746F74756E65DC
:1016B0002066696E697368656421205075742074B2
:1016C0006865204B702C204B6920616E64204B6450
:1016D00020636F6E7374616E747320696E746F2013
:1016E000436F6E66696775726174696F6E2E68000C
:1016F000504944204175746F74756E652066616948
:101700006C6564212074696D656F75740020403AC2
:10171000006F6B20543A006F6B20423A00504944EE
:10172000204175746F74756E65206661696C6564BF
:10173000212054656D706572617475726520746FD7
:101740006F206869676800204B643A2000204B696D
:101750003A2000204B703A200020436C617369638B
:101760002050494420002054753A2000204B753AFF
:101770002000206D61783A2000206D696E3A2000CB
:1017800020643A200020626961733A20004D41498B
:101790004E54454E414E4345004D415445524941FA
:1017A0004C005052494E54005072696E74696E6715
:1017B0002077697468205553422E2E2E0073757061
:1017C000706F727440756C74696D616B65722E63B5
:1017D0006F6D00436F6E746163743A0053616665A8
:1017E000747920636972637569740054656D702043
:1017F00073656E736F72204245440054656D7020AE
:1018000073656E736F72004552524F52202D2053F4
:10181000544F5050454400801506060606FEFEFE55
:10182000FEFC00000000000000FCFEFEFEFC0000CC
:10183000000EFEFEFEFE0000E0FCFEFEFCE0E0000E
:101840000000CECECE000000C0C0C0C0C0C080002E
:10185000000000000080C0C0800000000000008088
:1018600080C0C0C0C0C0C0C080800000000006FEB4
:10187000FEFEFE0000000080C0C0C00000000000AE
:10188000008080C0C0C080808000000000C0C0C058
:10189000C00080C0C0C0C08000000000007FFFFF0B
:1018A000FFFF80000000000080FFFFFFFFFF00003F
:1018B0000000FFFFFFFF000000FFFFFFFF00000030
:1018C0000000FFFFFF00000081F1FFFF3F0F3FFF1F
:1018D000FCF0F0FCFF3F0F3FFFFEF880000000C16E
:1018E000E1F1F17131010183FFFFFFFC000000FF16
:1018F000FFFFFF000C3EFFFFF7C301000000FCFEEE
:10190000FF8703113131333F3F3F1E000001FFFFCE
:10191000FFFF0703010101010000000000000103B7
:1019200007070F0F0F0F0F0F0F0707070F0F060007
:101930000000070F0F07000000070F0F070000004F
:1019400000000F0F0F0000060F0F0701000000013D
:10195000070F0F070100000001070F0F060000032B
:10196000070F0F0E0E060703070F0F0700000007F3
:101970000F0F0700000000030F0F0F060000000309
:1019800007070F0E0E0E0E0E0E06000000000F0FC2
:101990000F0F000000000000008015090909F9017F
:1019A00001010103FE0000000000FE03010101032C
:1019B000FE001FF101010101FFF01E030101031EE2
:1019C00010F000FF313131FF00E0202020202020E6
:1019D00060C080000080C060202060C00000000067
:1019E000C04060202020202020206040C080000FC8
:1019F000F901010101FF0080C060202020E000000B
:101A00000080C04060202020604040C08000E02076
:101A1000202020E0602020202060C0000000FF8007
:101A2000000000007FC0808080C07F0000000000B8
:101A3000FF0000FF00000000FF01FF00000000FFAA
:101A4000010100FF000000FF00C37A0E0000C0701B
:101A5000C000030E0E0300C070C00001077CC00070
:101A6000E3321A0A0A8ACAFAC67C00000003FE00A2
:101A7000FF00000000FF73C10000083CE68300FE89
:101A800003010078FCEE4A4E4C404040613F03FEAB
:101A900000000000F80C0602020203000000000330
:101AA000060C08181010101010101018081810103C
:101AB000190F000F181010180F000F181010180F22
:101AC0000000001F1010101F0F191010180E030037
:101AD000030E181010180E0300030E181010190F23
:101AE000070C181010111119080C181010180F00FD
:101AF0000F181010180F0001071C101010190F01FB
:101B0000070C081810111111111111190F00001FE5
:101B1000101010101F0000000000002F40000000F7
:101B2000000000000000000000808080C0E0FEFF98
:101B3000191E9898981818181818189E9F991E38EA
:101B4000F0E00000000000000000000000000000C5
:101B500000000000003CFEFFFF99F1E1C3FFFF0021
:101B6000006363636060606060606363630000FFE4
:101B7000FF7C38000000000000000000000080C072
:101B800060B0D8D81CFCFF3F0F8FCFC7C7C7C6C6F1
:101B9000C6C6C6C6C6C6C6C6C6C6C6C6C6C6C7C7E3
:101BA000C4CC0C1CF8F870C00000000EFFF92A2B02
:101BB0002B2828FCFFFF0000FFFFFFFFFFFFFFBFF8
:101BC000B717B5BDB500B5B5F717FFBFBFFFFFFF2E
:101BD000FF0000FFFFFCFF0700C0F0FFFFFDDD1D61
:101BE00019193FFFFF0000FFFFFFFFFFFFFFFBF1A1
:101BF000FBFBEAEEC0EEEAFAF0FAFAFFFFFFFFFFA6
:101C00000000FFFF0F1FF8E00003070F0F1B18195C
:101C1000FBFEFFFFF0E0C0C1E1F1F1F1F1F1F1F104
:101C2000F1F1F1F1F9F9F9F9F9F9797979F1F010BE
:101C3000181F070603030000000000000000F8FF63
:101C4000EFDFBF7FFFFFFF404143437F2120202183
:101C50007FFFFFFF3FB091D1DFD050581F1FF0F042
:101C600000000000000000000000000003070F1E3D
:101C70003D7B77EED1DEDECF4B4B696968686860EB
:101C80003F3F373737353430101018181A1B0F06FE
:101C90000000000000100FFC0E0FCFCFCFCECCCC39
:101CA000CCCCCCCCDCC0C007707E7F7F7F7F7F7FB9
:101CB0007F7F7F7F7F0F017120FFFFFFFFFFFFFF0F
:101CC000FFFFFFFCE000000000000000000000E05B
:101CD000FCFFFFFFFFFFFFFFFFFFFF000000000012
:101CE00000000000000000000000000000000000F4
:101CF0000000000000FFFFFFFFFFFFFF00000000EB
:101D000000000000000000000000000000000000D3
:101D100000000000000000000000000000000000C3
:101D200000000000000000000000FFFFFFFFFFFFB9
:101D3000FF7FFFFFFFFFFFF8800000000080F0FF43
:101D4000FFFFFFFF3FFFFFFFFFFFFFFF000000302F
:101D5000F8F8FCFC7E7E7E3E3E3E3E7E7EFEFEFC35
:101D6000FCF8E0800000FFFFFFFFFFFFFF000080A6
:101D7000C0E0F0F8FCFEFE7E3E1E0E06C0E0F0F86D
:101D8000FCFCFE7E3E3E3E3E3E7EFEFCFCF8F0C08D
:101D9000800000FEFEFEFEFEFEFEFEFFFFFFFFFFD8
:101DA000FFFF00031FFFFFFFFFFFFCE0E0FCFFFF62
:101DB000FFFFFF1F0100FFFFFFFFFFFFFF0000C04D
:101DC000E0F0F0F8F8FC7C7C3C3C3E1E1E1EFFFF61
:101DD000FFFFFFFFFF0000FFFFFFFFFFFFFFFEFF12
:101DE000FFFFFFFFFFFFF1C080000000FFFFFFFFCC
:101DF000FFFFFF3C3C3C3C3C3C3C3C3C3F3F3F3FCE
:101E00003F3F00000000000000000000FFFFFFFF58
:101E1000FFFFFF00000000073FFFFFFFFFFFFFFF86
:101E2000FF3F0700000000FFFFFFFFFFFFFF000074
:101E30003F7FFFFFFFFFFCFCF8F8F87C7C3C3EFF97
:101E4000FFFFFFFFFFFF0000FFFFFFFFFFFFFF039C
:101E500001000003071F7FFFFFFFFEFCF0E38F1F61
:101E60003F3F7F7FFEFCF8F8F0F0F0F8F8FCFC7ED6
:101E70007E3C300000FEFEFEFEFEFEFEFE43414EB6
:101E800043454C002073656300206D696E00206837
:101E90006F75720020686F7572730000000000009B
:101EA00000005F00000007000700147F147F142467
:101EB0002A7F2A12231308646236495522500005EE
:101EC000030000001C2241000041221C00082A1CC3
:101ED0002A0808083E0808005030000008080808D2
:101EE00008006060000020100804023E5149453E91
:101EF00000427F400042615149462141454B311823
:101F000014127F1027454545393C4A494930017133
:101F10000905033649494936064949291E0036361E
:101F20000000005636000000081422411414141456
:101F30001441221408000201510906324979413E38
:101F40007E1111117E7F494949363E414141227F30
:101F50004141221C7F494949417F090901013E4114
:101F60004151327F0808087F00417F4100204041F5
:101F70003F017F081422417F404040407F0204021D
:101F80007F7F0408107F3E4141413E7F09090906D9
:101F90003E4151215E7F091929464649494931018F
:101FA000017F01013F4040403F1F2040201F7F2014
:101FB00018207F63140814630304780403615149F3
:101FC000454300007F4141020408102041417F0049
:101FD00000040201020440404040400001020400AD
:101FE00020545454787F484444383844444420387A
:101FF0004444487F3854545418087E090102081498
:1020000054543C7F0804047800447D400020404440
:102010003D00007F10284400417F40007C041804EC
:10202000787C0804047838444444387C1414140838
:10203000081414187C7C08040408485454542004E0
:102040003F4440203C4040207C1C2040201C3C4021
:1020500030403C44281028440C5050503C446454B8
:102060004C44000836410000007F00000041360863
:102070000008082A1C08081C2A08086275696C6494
:10208000706C6174652E006F662061646A7573748C
:10209000696E6720796F75720074726F7567687406
:1020A000207468652070726F6365737300492077D0
:1020B000696C6C20677569646520796F75004341B0
:1020C0004E43454C00434F4E54494E554500473111
:1020D00020462569205A25692058256920592569F7
:1020E00000473238205A302058302059300066726C
:1020F0006F6D20746865206275696C64706C6174C2
:10210000652E0061206D696C6C696D657465722067
:102110006177617900756E74696C20746865206EF2
:102120006F7A7A6C6520697300526F7461746520F0
:1021300074686520627574746F6E00342F323100DC
:10214000434F4E54494E554500434F4E54494E550A
:102150004500473120462569205A30004731204646
:1021600025692058256920592569004731204625D1
:1021700069205A350066726F6D207468652062753B
:10218000696C64706C6174652E0069732061206DE8
:10219000696C6C696D657465722061776179007333
:1021A000637265772074696C6C20746865206E6F4B
:1021B0007A7A6C65005475726E206C656674206264
:1021C00075696C64706C61746500352F3231004341
:1021D0004F4E54494E554500473120462569205AF7
:1021E0003000473120462569205825692059256946
:1021F00000473120462569205A350066726F6D20F0
:10220000746865206275696C64706C6174652E0019
:1022100069732061206D696C6C696D6574657220ED
:10222000617761790073637265772074696C6C20E3
:10223000746865206E6F7A7A6C65005475726E20D2
:102240007269676874206275696C64706C6174652A
:1022500000362F323100434F4E54494E55450074DD
:102260006865206275696C64706C617465206C656A
:1022700076656C2E00706170657220746F206669DF
:102280006E652D74756E65006E6F772075736520B1
:1022900061207368656574206F66005265706561C2
:1022A00074207468697320737465702C206275746F
:1022B00000372F323100434F4E54494E55450047A9
:1022C0003120462569205A300047312046256920B3
:1022D0005825692059256900473120462569205A2B
:1022E000350062697420726573697374616E636529
:1022F0002E00756E74696C20796F75206665656C4B
:102300002061006275696C64706C61746520616E37
:1023100064206E6F7A7A6C6500536C696465206125
:10232000207061706572206265747765656E003833
:102330002F323100434F4E54494E554500434F4EC6
:1023400054494E554500746865206C656674206379
:102350006F726E65722E2E2E00526570656174204C
:102360007468697320666F7200392F323100434FF1
:102370004E54494E5545007468652072696768740B
:1023800020636F726E65722E2E2E0052657065612D
:1023900074207468697320666F720031302F323197
:1023A00000434F4E54494E554500444F4E4500742E
:1023B0006F20696E73657274206D617465726961F6
:1023C0006C2E00746865206E657874207374657077
:1023D00020697300746865206275696C64706C6153
:1023E0007465004E6F772074686174207765206C87
:1023F0006576656C65640031312F323100434F4E94
:1024000054494E5545004731204631323030302056
:1024100058313130205930006D6174657269616CDA
:10242000206C6F6164696E67007072696E746865B4
:1024300061642068656174696E6720666F72005020
:102440006C6561736520776169742C0031322F32BD
:10245000310061626F766520746865206172726F09
:10246000772E00796F757220556C74696D616B659C
:1024700072322C0066726F6D20746865207265611F
:1024800072206F6600496E73657274206E657720E6
:102490006D6174657269616C0031332F32310043B4
:1024A0004F4E54494E5545004C6F6164696E67202C
:1024B0006D6174657269616C2E2E2E0031342F327D
:1024C000310066726F6D206E6F7A7A6C652E2E2EDB
:1024D000006D6174657269616C2065786974730060
:1024E0005075736820627574746F6E207768656EBE
:1024F0000031352F323100434F4E54494E5545007F
:10250000556C74696D616B6572322E00696E73650E
:102510007274656420696E2074686520006D617452
:10252000657269616C20796F752068617665004E0F
:102530006578742C2073656C65637420746865001D
:1025400031362F32310052454144590031372F3254
:10255000310041425300504C410069732074686956
:10256000732072696768743F004142532061732091
:102570006D6174657269616C2C00596F75206861BA
:1025800076652063686F73656E0031382F323100D5
:102590004E4F005945530069742069732075736963
:1025A0006E672E006F66206D6174657269616C00E4
:1025B0006B6E6F77732077686174206B696E64004F
:1025C0004E6F7720796F757220556C74696D616BF1
:1025D0006572320031392F323100434F4E54494E2B
:1025E0005545006D616B6520612033442050726950
:1025F0006E74210049276D207265616479206C65D5
:102600007427730032302F32310041524520594F28
:10261000552052454144593F00746F207072696ED5
:10262000742069742100616E642070726573732078
:1026300074686520627574746F6E006F6E207468C4
:10264000652053442D636172640053656C65637447
:102650002061207072696E742066696C6500323189
:102660002F3231004C45542753205052494E5400CC
:1026700052656164696E6720636172642E2E2E005C
:1026800032312F323100796F757220556C74696D5B
:10269000616B6572322E2E2E007468617420636146
:1026A0006D65207769746800506C65617365206999
:1026B0006E736572742053442D636172640032310D
:1026C0002F323100697320746869732072696768FA
:1026D000743F00504C41206173206D6174657269D4
:1026E000616C2C00596F7520686176652063686F96
:1026F00073656E0031382F3231004E4F005945530B
:1027000000473238205A3000627574746F6E20743E
:102710006F20636F6E74696E756500556C74696DBA
:10272000616B657221205072657373207468650057
:1027300073746172747570206F6620796F757200A2
:1027400057656C636F6D6520746F207468652066D3
:102750006972737400312F323100434F4E54494E29
:10276000554500612066697273742072756E20771A
:10277000697A6172642E0077616C6B20796F7520C5
:102780007468726F75676800666972737420737419
:10279000617274757020492077696C6C00426563C2
:1027A0006175736520746869732069732074686546
:1027B00000322F323100434F4E54494E55450047A9
:1027C0003120462569205A256900473238205A3081
:1027D00000676F696E6720746F20646F2074686192
:1027E00074206E6F772E0061646A7573746D656E08
:1027F00074732C20776520617265007765206E65A3
:10280000656420746F20646F20736F6D650041668E
:10281000746572207472616E73706F727461746922
:102820006F6E00332F323100434F4E54494E5545A1
:1028300000473120462569205A25692058256920FE
:10284000592569004732382058302059300043005C
:10285000432F00436C69636B20746F20726574753D
:10286000726E004275696C64706C61746520746589
:102870006D702E3A0052455455524E004144564117
:102880004E434544004255494C442D7C504C4154E4
:1028900045004731205A343000473238205A300042
:1028A000473238205A3000473238205830205930CB
:1028B00000414456414E43454400746F20646566B0
:1028C00061756C743F00526573657420657665723E
:1028D000797468696E67004E4F005945530056651C
:1028E0007273696F6E2031342E30312E31004A619F
:1028F0006E20203820323031342031323A34303AB0
:1029000031380052657475726E006D6D2F7365639A
:10291000004D6178207370656564205A006D6D2FDD
:10292000736563004D61782073706565642059009C
:102930006D6D2F736563004D6178207370656564FC
:102940002058006D6D2F73656300582F59204A651C
:10295000726B0030306D6D2F7365635E32004163C2
:1029600063656C65726174696F6E004D4F54494FB9
:102970004E006D6D2F736563006D6D2F7365630081
:102980006D6D2F736563006D6D2F736563006D6DE5
:102990002F7365635E32003F3F3F004D61782073C7
:1029A00070656564205A004D6178207370656564B8
:1029B0002059004D61782073706565642058005877
:1029C0002F59204A65726B00416363656C657261C3
:1029D00074696F6E003C2052455455524E006D6D27
:1029E0002F73656300526574726163742073706540
:1029F0006564006D6D0052657472616374206C656E
:102A00006E6774680052455452414354494F4E001A
:102A10006D6D2F736563006D6D003F3F3F00526524
:102A200074726163742073706565640052657472BA
:102A3000616374206C656E677468003C2052455475
:102A400055524E004300432F00436C69636B207462
:102A50006F2072657475726E00526F7461746520B8
:102A6000746F2065787472756465004E6F7A7A6C45
:102A7000652074656D70657261747572653A0043A6
:102A800000432F00436C69636B20746F2072657480
:102A900075726E004E6F7A7A6C652074656D706524
:102AA0007261747572653A002500427269676874D4
:102AB0006E657373004C45440025003F3F3F002086
:102AC000476C6F77207768656E20646F6E650020B5
:102AD0004F6E207768696C65207072696E74696EDC
:102AE000670020416C77617973204F666600204152
:102AF0006C77617973204F6E004272696768746EFB
:102B0000657373003C2052455455524E003F3F3F81
:102B100000466163746F7279207265736574005644
:102B2000657273696F6E004D6F74696F6E207365A7
:102B30007474696E67730052657472616374696F4F
:102B40006E2073657474696E6773004D6F766520CF
:102B50006D6174657269616C0052616973652062B0
:102B600075696C64706C617465004C6F7765722078
:102B70006275696C64706C61746500486F6D652086
:102B80006865616400486561747570206275696C80
:102B900064706C61746500486561747570206E6F57
:102BA0007A7A6C65004C45442073657474696E676D
:102BB00073003C2052455455524E00414253005040
:102BC0004C410052455455524E0053455454494EC1
:102BD0004753004348414E4745004D4154455249F3
:102BE000414C0053656C6563746564206D61746568
:102BF0007269616C3A004F4B0025004D617465723B
:102C000069616C20666C6F7700250046616E2073E9
:102C100070656564006D6D004D6174657269616C0D
:102C2000204469616D657465720043004275696C8A
:102C300064706C6174652054656D702E004300549F
:102C4000656D7065726174757265004D41544552D1
:102C500049414C0050524553455453004E6577202E
:102C6000707265736574003C2052455455524E0095
:102C7000250025006D6D00430043003F3F3F00539A
:102C8000746F72652061732070726573657400469D
:102C90006C6F7720250046616E004469616D657434
:102CA000657200486561746564206275696C647062
:102CB0006C6174650054656D7065726174757265E0
:102CC000003C2052455455524E004D6F6469667960
:102CD000207468652073657474696E6773002500DD
:102CE00046616E3A2000430043002500466C6F7732
:102CF0003A006D6D00437573746F6D697A65003CC1
:102D00002052455455524E00666F72206D617465B5
:102D10007269616C2072656D6F76616C00486561E7
:102D200074696E67207072696E74686561640047CB
:102D300032382058302059300052657665727369F8
:102D40006E67206D6174657269616C0052656D6FAC
:102D50007665206D6174657269616C0043414E4314
:102D6000454C0052454144590047312046256920D1
:102D70005825692059256900473238205830205994
:102D8000300061626F766520746865206172726FD1
:102D9000772E00796F7572206D616368696E652C9E
:102DA0000066726F6D20746865206261636B736981
:102DB0006465206F6600496E73657274206E657776
:102DC000206D6174657269616C0043414E43454CEE
:102DD00000524541445900466F7277617264696ED2
:102DE00067206D6174657269616C00636F6D6573F6
:102DF000206F757420746865206E6F7A7A6C650038
:102E0000576169742074696C6C206D6174657269B6
:102E1000616C0043414E43454C00524541445900CA
:102E20004300432F00436C69636B20746F2072650D
:102E30007475726E004E6F7A7A6C652074656D7071
:102E4000657261747572653A00534420434152447F
:102E5000004731204631323030302058352059314A
:102E60003000473238003B464C41564F523A556C81
:102E7000746947436F6465003B464C41564F523A74
:102E8000556C746947436F6465004E6F2066696CCA
:102E9000657320666F756E6421004F4B004F4B00C9
:102EA00052656164696E6720636172642E2E2E0024
:102EB000506C6561736520696E736572742063611F
:102EC0007264004E6F2053442D4341524421003C14
:102ED000204241434B003C2052455455524E00661F
:102EE000726F6D2074686520736C696365722E0063
:102EF00073657474696E672077697468207365748C
:102F000074696E67006F76657272696465206D61C1
:102F10006368696E6500546869732066696C652032
:102F200077696C6C0043414E43454C00434F4E540F
:102F3000494E5545004D383400473238004731205E
:102F4000463135303020453000473932204525693B
:102F500000436F64653A0053442D6361726421003D
:102F600072656164696E67004572726F722077687E
:102F7000696C650052455455524E20544F204D41C6
:102F8000494E00746865207072696E742E00596F26
:102F9000752063616E2072656D6F76650050726991
:102FA0006E742066696E697368656400430043202F
:102FB000005072696E74657220636F6F6C696E6722
:102FC00020646F776E004241434B20544F204D45A3
:102FD0004E550054696D65206C6566740054696DCA
:102FE00065206C65667420756E6B6E6F776E00433E
:102FF00000430048656174696E67206275696C649E
:10300000706C617465004300430048656174696ECB
:1030100067005072696E74696E673A0041424F52A0
:10302000540054554E450041626F727420746865B7
:10303000207072696E743F004E4F00594553002551
:10304000004272696768746E6573730025004D6194
:1030500074657269616C20666C6F7700250046614B
:103060006E2073706565640025005072696E74206F
:1030700073706565640054554E45006D6D2F736522
:1030800063005265747261637420737065656400D7
:103090006D6D0052657472616374206C656E677447
:1030A000680052455452414354494F4E006D6D2FB4
:1030B000736563006D6D003F3F3F00526574726140
:1030C0006374207370656564005265747261637423
:1030D000206C656E677468003C2052455455524E12
:1030E0000025002500250043004300430043002540
:1030F000004C4544204272696768746E65737300C2
:1031000052657472616374696F6E004D61746572AB
:1031100069616C20666C6F770046616E2073706524
:103120006564004275696C64706C617465207465D7
:103130006D702E0054656D706572617475726500F6
:103140005370656564003C2052455455524E005002
:103150007265706172696E6720746F207072696E3B
:10316000743A0048656174696E672075702E2E2E62
:103170000041424F52540054554E45004E6F206955
:103180006E666F20617661696C61626C65006D00CE
:103190006D004D6174657269616C3A200054696D0F
:1031A000653A20003B4D4154455249414C3A003B61
:1031B00054494D453A00466F6C64657200494E466D
:1031C000494E4954594E414ECDCCCC3D0AD7233CB3
:1031D00017B7D13877CC2B329595E6241FB14F0A1B
:1031E000000020410000C84200401C4620BCBE4CEC
:1031F000CA1B0E5AAEC59D74DD2F6055D82F112401
:103200001FBECFEFD1E2DEBFCDBF00E00CBF14E0A8
:10321000A0E0B2E0ECE7FAEB01E00BBF02C00790E0
:103220000D92A232B107D9F717E1A2E2B4E001C0D2
:103230001D92A935B107E1F711E3CCEFD1E304C04A
:103240002297FE010E942EDDC83FD107C9F704D0A6
:103250000C9421D40C940000CF93DF9332D10E94C0
:103260005352C0E0D0E00E94C7512097E1F30E9482
:103270000000F9CFCF92DF92EF92FF920F931F934E
:10328000CF93DF937C016B018A01C0E0D0E00FC0D7
:10329000D6016D916D01D701ED91FC910190F08106
:1032A000E02DC7011995C80FD91F01501040011515
:1032B000110571F7CE01DF91CF911F910F91FF9012
:1032C000EF90DF90CF9008958230B9F0833028F4EA
:1032D000882351F0813051F50AC0843011F18430D7
:1032E000E8F0853019F520C010926E0008958091A5
:1032F0006F008D7F80936F000895809170008D7FA7
:103300008093700081E08093B0008091B100887F4D
:1033100084608093B1001092B30008951092710000
:1033200008951092720008951092730008951F93EB
:10333000182F80913B03811711F09FEF06C0EFE239
:10334000F1E094918FEF80933B03892FBDDF812FB4
:1033500060E0AAD21F9108951F920F920FB60F92AC
:103360000BB60F9211242F933F934F935F936F935C
:103370007F938F939F93AF93BF93EF93FF9380912E
:10338000220490912304A0912404B0912504009775
:10339000A105B10551F1E0912604F0912704808147
:1033A000909128048927808380912204909123049E
:1033B000A0912404B0912504181619061A061B06BC
:1033C000BCF48091220490912304A0912404B09134
:1033D00025040197A109B109809322049093230445
:1033E000A0932404B093250403C080913B039FDF86
:1033F000FF91EF91BF91AF919F918F917F916F91CD
:103400005F914F913F912F910F900BBE0F900FBE88
:103410000F901F9018951F920F920FB60F921124C4
:103420002F933F938F939F93AF93BF9380912D04DE
:1034300090912E04A0912F04B0913004309131046A
:103440000196A11DB11D232F2D5F2D3720F02D5783
:103450000196A11DB11D2093310480932D049093FA
:103460002E04A0932F04B0933004809129049091EE
:103470002A04A0912B04B0912C040196A11DB11D2A
:103480008093290490932A04A0932B04B0932C04D6
:10349000BF91AF919F918F913F912F910F900FBE50
:1034A0000F901F9018958FB7F89420912D043091AC
:1034B0002E0440912F04509130048FBFB901CA01EE
:1034C0000895789484B5826084BD84B5816084BD9C
:1034D00085B5826085BD85B5816085BDEEE6F0E08D
:1034E000808181608083E1E8F0E0108280818260E9
:1034F0008083808181608083E0E8F0E0808181606A
:103500008083E1EBF0E0808184608083E0EBF0E099
:10351000808181608083E1E9F0E080818260808346
:10352000808181608083E0E9F0E080818160808338
:10353000E1EAF0E080818260808380818160808325
:10354000E0EAF0E0808181608083E1E2F1E0808167
:1035500082608083808181608083E0E2F1E080810D
:1035600081608083EAE7F0E08081846080838081ED
:103570008260808380818160808380818068808395
:103580001092C10008951F93CF93DF93182FEB0182
:1035900061E0D7D0209709F4CAC0CF3FD10509F424
:1035A000C9C0E12FF0E0E65FFD4F8491893009F456
:1035B00066C08A30B0F48430F1F1853040F4823056
:1035C00059F1833070F5813009F0AEC020C08730EA
:1035D00009F443C0883008F048C0863009F0A4C020
:1035E00034C08D3009F478C08E3038F48B3009F453
:1035F0005AC08C3008F066C04CC0803109F480C0DD
:10360000813109F487C08F3009F08EC06FC084B556
:10361000806884BDC7BD91C084B5806284BDC8BDCB
:103620008CC080918000806880938000D093890056
:10363000C093880082C08091800080628093800067
:10364000D0938B00C0938A0078C08091B0008068CE
:103650008093B000C093B30070C08091B0008062CE
:103660008093B000C093B40068C0809190008068DF
:1036700080939000D0939900C09398005EC0809191
:103680009000806280939000D0939B00C0939A003A
:1036900054C080919000886080939000D0939D00EA
:1036A000C0939C004AC08091A00080688093A000D5
:1036B0008091A0008F7B8093A000D093A900C0933D
:1036C000A8003BC08091A00080628093A000D093AE
:1036D000AB00C093AA0031C08091A00088608093A5
:1036E000A000D093AD00C093AC0027C08091200112
:1036F000806880932001D0932901C09328011DC0C8
:1037000080912001806280932001D0932B01C0938F
:103710002A0113C080912001886080932001D093FA
:103720002D01C0932C0109C0C038D1051CF4812F94
:1037300060E002C0812F61E0B7D0DF91CF911F918F
:103740000895CF93DF93482F50E0CA018C539E4FCA
:10375000FC01349142585E4FFA018491882369F14B
:1037600090E0880F991FFC01E05DFE4FA591B49198
:10377000FC01E65BFE4FC591D491662351F42FB74F
:10378000F8948C91932F909589238C938881892329
:103790000BC0623061F42FB7F8948C91932F909501
:1037A00089238C938881832B88832FBF06C09FB782
:1037B000F8948C91832B8C939FBFDF91CF910895C8
:1037C000893009F449C08A30A0F4843051F1853041
:1037D00040F4823079F1833000F5813009F063C024
:1037E00026C0873079F1883098F5863009F05BC0C3
:1037F00025C08D3009F442C08E3028F48B30B1F1F1
:103800008C30C0F52DC0803109F442C0813109F4FB
:1038100045C08F3009F047C037C0809180008F7756
:1038200003C0809180008F7D80938000089584B5CF
:103830008F7702C084B58F7D84BD08958091B000DC
:103840008F7703C08091B0008F7D8093B000089582
:10385000809190008F7707C0809190008F7D03C08A
:1038600080919000877F8093900008958091A000C0
:103870008F7707C08091A0008F7D03C08091A0004A
:10388000877F8093A0000895809120018F7703C0E7
:10389000809120018F7D80932001089580912001E7
:1038A000877F809320010895FF920F931F93F62E38
:1038B000482F50E0CA01865F9D4FFC012491CA0148
:1038C0008C539E4FFC01149142585E4FFA010491B3
:1038D0000023C1F0222311F0822F72DFE02FF0E0ED
:1038E000EE0FFF1FE65BFE4FA591B4919FB7F894D2
:1038F000FF2021F48C911095812302C08C91812BA3
:103900008C939FBF1F910F91FF900895AC01DB0135
:10391000FA0190E02EE28C91803229F0983009F47F
:1039200021938C9181939F5F11969B30A1F7108218
:10393000CA010895FC01128217A60895FC0187A50B
:10394000882311F081E082830895FC018281811136
:1039500012820895CF93DF93EC01FC01EA55FE4FEC
:103960008081882309F461C081508083DE01AB5AD5
:10397000BF4FFE01EC58FF4F8BE101900D9281503B
:10398000E1F7FE01ED5AFF4FCE58DF4F8881998154
:10399000C257D0409183808330E0BE016A557E4F8C
:1039A0003FC0832F90E0AC014F5F5F4FDC01E5E04B
:1039B000AA0FBB1FEA95E1F7A81BB90BAC0FBD1FFF
:1039C000FA0125E0EE0FFF1F2A95E1F7E41BF50B46
:1039D000EC0FFD1FAC58BF4FEC58FF4F2BE101908F
:1039E0000D922150E1F7FC0125E0EE0FFF1F2A9513
:1039F000E1F7E81BF90BEC0FFD1FEE58FF4FDA0162
:103A000085E0AA0FBB1F8A95E1F7A41BB50BAC0F8D
:103A1000BD1FAE58BF4F8D919C91918380833F5FB6
:103A2000FB018081381708F4BCCFDF91CF91089556
:103A3000FC018AE194E0918380838781882321F0CF
:103A4000CF0104960C94D67008950F931F938C01A8
:103A50000E94497F0E94457EC80181539E4F0E946B
:103A6000D670F801128280E592E00E94DE531F9129
:103A70000F910895CF92DF92EF92FF920F931F93D1
:103A8000DF93CF93CDB7DEB76F970FB6F894DEBF55
:103A90000FBECDBF8C016B01085A1F4FD8018C910E
:103AA00008551040882321F480E3E82EF12C03C050
:103AB000B1E5EB2EF12CE00EF11E8AE194E09A8341
:103AC00089831C821B8218861D82B7016C5F7F4F21
:103AD000CE010596A60121E00E940F78882391F57A
:103AE000ECE5F2E0949108C08091C00085FFFCCF26
:103AF0009093C600319694919923B1F7E2E6F2E0F3
:103B0000949108C08091C00085FFFCCF9093C600BF
:103B1000319694919923B1F709C08091C00085FF37
:103B2000FCCF0894C11CD11C9093C600F601908173
:103B3000992399F78091C00085FFFCCF8AE080939C
:103B4000C60056C0F801EA55FE4F80818A3008F061
:103B50003EC08F5F8083282F30E0C9010197FC01B0
:103B6000A5E0EE0FFF1FAA95E1F7E81BF90BEC5853
:103B7000FF4FE00FF11F21503040AF01415E5F4F1A
:103B8000BF018BE1DB010D90BD01DA010D92AD01AA
:103B90008150C1F7929182913296968F858F7F974F
:103BA0002115310541F7D801AC58BF4FF7013496C4
:103BB0008BE101900D928150E1F70E581F4FF701F4
:103BC00082819381D8018D939C9302571040D80134
:103BD000AB5ABF4FFE0135968BE101900D9281509B
:103BE000E1F70D5A1F4F8B819C81F80191838083EF
:103BF000CE0101961DDF6F960FB6F894DEBF0FBEA3
:103C0000CDBFCF91DF911F910F91FF90EF90DF908B
:103C1000CF900895EF92FF920F931F938C019FEC2A
:103C2000E92E91E0F92EE00EF11EC7010E94877087
:103C3000C7010E94D670F801108211821F910F9166
:103C4000FF90EF900895CF92DF92EF92FF920F9343
:103C50001F93CF93DF937C016B01DB010D9000205C
:103C6000E9F78D0101501040061B170BEFECF1E056
:103C7000EE0EFF1ED7011C92E1E3FEEFEE0EFF1EDB
:103C8000CB016EE470E00E94C8D4EC01009731F4DF
:103C9000F8013197EC0DFD1D86010EC060E270E069
:103CA0000E94C8D48C010F5F1F4FCE016AE270E002
:103CB0000E94C8D4FC0131978DE081838AE0828321
:103CC0001382C70185539E4FB8010E9409798FEC7A
:103CD00091E0E80EF91ED7018C91882319F1ECE8E8
:103CE000F2E0949108C08091C00085FFFCCF9093D2
:103CF000C600319694919923B1F7E3E9F2E09491EB
:103D000008C08091C00085FFFCCF9093C60031961B
:103D100094919923B1F78091C00085FFFCCF8AE090
:103D20008093C600DF91CF911F910F91FF90EF908C
:103D3000DF90CF900895CF93DF93EC018FA5882378
:103D400009F43DC0E7ECF2E0949108C08091C00016
:103D500085FFFCCF9093C600319694919923B1F7DB
:103D6000CE50DE4F488159816A817B81C25FD1404C
:103D700084E49AE02AE030E00E94F755E5ECF2E0B6
:103D8000949108C08091C00085FFFCCF9093C6003D
:103D9000319694919923B1F7C651DE4F48815981EC
:103DA0006A817B81CA5ED14084E49AE02AE030E0F7
:103DB0000E94F7558091C00085FFFCCF12C0E5EB53
:103DC000F2E0949108C08091C00085FFFCCF9093F1
:103DD000C600319694919923B1F78091C00085FF78
:103DE000FCCF8AE08093C600C755DE4F688166230A
:103DF000E1F0E9EAF2E0949108C08091C00085FF0B
:103E0000FCCF9093C600319694919923B1F784E446
:103E10009AE070E04AE050E00E9446568091C0006F
:103E200085FFFCCF8AE08093C600DF91CF91089593
:103E30002F923F924F925F926F927F928F929F92BA
:103E4000AF92BF92CF92DF92EF92FF920F931F93A8
:103E5000DF93CF93CDB7DEB7AD970FB6F894DEBF43
:103E60000FBECDBF5C014B014DA7FC0187A5882388
:103E700009F4E1C13FEC432E31E0532E4A0C5B1CA8
:103E8000C2010E94D670F50112821A8A1D8A198A0F
:103E9000188A8AE194E09F878E872FE4C22ED12C66
:103EA000CA0CDB1C80E390E0A80EB91EF601B182BB
:103EB000A08280ED9FEFA80EB91EF40180818F32A1
:103EC00009F08DC0C4016FE270E00E94C8D47C018B
:103ED0000894E11CF11C3E010894611C711C160140
:103EE00078C0C7016FE270E00E94C8D46C010097EF
:103EF00009F483C0E816F90608F07FC08C010E199A
:103F00001F09C301B701A8010E94E8D4060D171DBF
:103F1000F8011082F30107C08091C00085FFFCCF3B
:103F200031969093C60090819923B1F78091C0009B
:103F300085FFFCCFFAE0F093C600F101608171814A
:103F40006115710519F460E070E002C06C5F7F4F8D
:103F5000CE014296A30121E00E940F78882371F5DB
:103F6000EBE7F3E0949108C08091C00085FFFCCF9F
:103F70009093C600319694919923B1F7FE01319642
:103F800007C08091C00085FFFCCF31969093C6009A
:103F900090819923B1F7E9E7F3E0949108C080910B
:103FA000C00085FFFCCF9093C60031969491992371
:103FB000B1F78091C00085FFFCCF37C18EE090E063
:103FC0008C0F9D1FF1019183808376010894E11C81
:103FD000F11C92E0E916F10408F083CF0BC0E1E593
:103FE000F0E0AE0EBF1EF601B182A0828FEA9FEF15
:103FF000A80EB91E082DF92C01C00E2DF501E15BAC
:10400000FF4F9DA5992309F4ADC0608171816115B1
:10401000710519F460E070E002C06C5F7F4FC2016F
:10402000402F5F2D21E00E940F78882309F46AC099
:10403000E0EEF1E0AE0EBF1EF501408151816281DC
:1040400073818AE090E0A80EB91EF5014083518388
:104050006283738386E19EEFA80EB91EEBE6F3E060
:10406000949108C08091C00085FFFCCF9093C6005A
:10407000319694919923B1F7802F9F2D9C01F901DE
:1040800007C08091C00085FFFCCF31969093C60099
:1040900090819923B1F7E3E6F3E0949108C0809111
:1040A000C00085FFFCCF9093C60031969491992370
:1040B000B1F784E49AE02AE030E00E94F75580915D
:1040C000C00085FFFCCF8AE08093C600E2EFF1E0FC
:1040D000AE0EBF1EF5011082118212821382E5E539
:1040E000F3E0949108C08091C00085FFFCCF9093CD
:1040F000C600319694919923B1F78091C00085FF55
:10410000FCCF93C0E1E4F3E0949108C08091C0003B
:1041100085FFFCCF9093C600319694919923B1F717
:10412000802F9F2D9C01F90107C08091C00085FF61
:10413000FCCF31969093C60090819923B1F7EFE3BD
:10414000F3E0949108C08091C00085FFFCCF90936C
:10415000C600319694919923B1F78091C00085FFF4
:10416000FCCF63C0608171816115710519F460E055
:1041700070E002C06C5F7F4FC201402F5F2D26E5CB
:104180000E940F78882381F5EBE2F3E0949108C058
:104190008091C00085FFFCCF9093C600319694912A
:1041A0009923B1F7802F9F2D9C01F90107C08091C1
:1041B000C00085FFFCCF31969093C6009081992373
:1041C000B1F7E9E2F3E0949108C08091C00085FF67
:1041D000FCCF9093C600319694919923B1F78091CA
:1041E000C00085FFFCCF21C081E0F5018083E7E1BD
:1041F000F3E0949108C08091C00085FFFCCF9093BC
:10420000C600319694919923B1F7F40107C08091CB
:10421000C00085FFFCCF31969093C6009081992312
:10422000B1F78091C00085FFFCCF8AE08093C60083
:10423000CE010E96FDDBAD960FB6F894DEBF0FBE35
:10424000CDBFCF91DF911F910F91FF90EF90DF9045
:10425000CF90BF90AF909F908F907F906F905F9026
:104260004F903F902F900895FC0181E08183CF0112
:1042700040E0DECD2F923F924F925F926F927F92FD
:104280008F929F92AF92BF92CF92DF92EF92FF9266
:104290000F931F93DF93CF93CDB7DEB7AC970FB6D5
:1042A000F894DEBF0FBECDBF5C014B01FC0187A5BA
:1042B000882309F437C1C50181539E4F0E94D670EF
:1042C000F50112821A8A1D8A198A188A8AE194E0F5
:1042D0009F878E875FE4C52ED12CCA0CDB1C20E3A0
:1042E00030E0A20EB31EF601B182A08220ED3FEFB6
:1042F000A20EB31EF40180818F3209F090C0C40178
:104300006FE270E00E94C8D47C010894E11CF11CAB
:104310003E010894611C711C260142E1242E312CBF
:104320002C0E3D1E77C0C7016FE270E00E94C8D41A
:104330006C01009709F481C0E816F90608F07DC009
:104340008C010E191F09C301B701A8010E94E8D40E
:10435000060D171DF8011082F30107C08091C000FF
:1043600085FFFCCF31969093C60090819923B1F7D9
:104370008091C00085FFFCCFFAE0F093C600F20107
:10438000608171816115710519F460E070E002C00F
:104390006C5F7F4FC101A30121E00E940F78882349
:1043A00071F5E3E0F3E0949108C08091C00085FFCF
:1043B000FCCF9093C600319694919923B1F7FE01FA
:1043C000319607C08091C00085FFFCCF3196909355
:1043D000C60090819923B1F7E1E0F3E0949108C021
:1043E0008091C00085FFFCCF9093C60031969491D8
:1043F0009923B1F78091C00085FFFCCF8DC02EE0DE
:1044000030E02C0F3D1FF2013183208376010894A8
:10441000E11CF11CE114F10409F085CF0BC081E52A
:1044200090E0A80EB91EF601B182A0822FEA3FEFFC
:10443000A20EB31ED82C092D02C0DE2C0F2D8FE446
:1044400090E0A80EB91EF5018081918121EB3FEF2C
:10445000A20EB31E009719F480E090E001C004960C
:104460006D2D702F0E94DB78882339F1E3EFF2E0A5
:10447000949108C08091C00085FFFCCF9093C60046
:10448000319694919923B1F78D2D902F9C01F901CC
:1044900007C08091C00085FFFCCF31969093C60085
:1044A00090819923B1F782EF91E0A80EB91EF50132
:1044B000108211821282138232C0EBEDF2E09491ED
:1044C00008C08091C00085FFFCCF9093C600319654
:1044D00094919923B1F78D2D902F9C01F90107C07C
:1044E0008091C00085FFFCCF31969093C6009081EB
:1044F0009923B1F7E9EDF2E0949108C08091C000F2
:1045000085FFFCCF9093C600319694919923B1F723
:104510008091C00085FFFCCF8AE08093C600CE0169
:104520000E9686DAAC960FB6F894DEBF0FBECDBFFE
:10453000CF91DF911F910F91FF90EF90DF90CF907F
:10454000BF90AF909F908F907F906F905F904F90B3
:104550003F902F900895EF92FF920F931F93CF9368
:10456000DF938C01FC0117A687A9882321F0C801DD
:10457000C4960E94D67068EAE62E61E0F62EE00E40
:10458000F11EC70160E045E30E94AA6E882309F589
:10459000ECE5F2E0949108C08091C00085FFFCCF6B
:1045A0009093C600319694919923B1F7EDEBF3E027
:1045B000949108C08091C00085FFFCCF9093C60005
:1045C000319694919923B1F78091C00085FFFCCF7B
:1045D0007DC0E801C355DE4FCE01B70141E00E9426
:1045E000A679882341F5CE01B70140E00E94A67963
:1045F000882309F5ECE8F2E0949108C08091C000AE
:1046000085FFFCCF9093C600319694919923B1F722
:10461000EAEAF3E0949108C08091C00085FFFCCFE6
:104620009093C600319694919923B1F78091C00080
:1046300085FFFCCF4BC0C801C496BE010E94AD737C
:10464000882309F5ECE8F2E0949108C08091C0005D
:1046500085FFFCCF9093C600319694919923B1F7D2
:10466000EAE9F3E0949108C08091C00085FFFCCF97
:104670009093C600319694919923B1F78091C00030
:1046800085FFFCCF23C081E0F80187A7ECE5F2E0CD
:10469000949108C08091C00085FFFCCF9093C60024
:1046A000319694919923B1F7EFE8F3E0949108C023
:1046B0008091C00085FFFCCF9093C6003196949105
:1046C0009923B1F78091C00085FFFCCF8AE08093E9
:1046D000C600D801AB5ABF4FF801F4968BE10190A8
:1046E0000D928150E1F7F80182A993A90D5A1F4F4D
:1046F000F8019183808303551040C801C096015B87
:104700001F4FF80191838083DF91CF911F910F910B
:10471000FF90EF9008952F923F924F925F926F9289
:104720007F929F92AF92BF92CF92DF92EF92FF92D1
:104730000F931F93DF93CF93CDB7DEB7CC55D04007
:104740000FB6F894DEBF0FBECDBF6C01662311F526
:1047500026EF31E0C20ED31ED6018C91EAE0FEEFC7
:10476000CE0EDF1E882309F4E7C02EEE31E0C20E24
:10477000D31ED601ED90FD900D911C91E2E1FEEF6C
:10478000CE0EDF1E0E94531AE616F7060807190719
:1047900008F4D2C026EF31E0C20ED31ED6011C921F
:1047A000EAE0FEEFCE0EDF1ED6019F968C918823A5
:1047B00039F4C601D0DEF60187A5882309F4BCC010
:1047C00000D000D0EDB7FEB731967E010894E11C11
:1047D000F11CADB7BEB71296FC92EE92119783E82A
:1047E00092E093838283D6019D968D919C919E97B2
:1047F000958384830E9417D58701EDB7FEB736965F
:104800000FB6F894FEBF0FBEEDBF570108C0D80128
:104810008C9190E00E942CD4F80181938F01F501D6
:1048200001900020E9F73197EA19FB09802F8E19D2
:104830008E176CF3A4E3AA2EB12CAC0CBD1CC501E1
:1048400040E050E060E070E00E94BD6F9924FDE31D
:10485000EF2EF12CEC0EFD1E2E010894411C511C74
:10486000EFE16E2E712C6C0E7D1E7CE7272E72E020
:10487000372E42C0D8018C9190E00E942CD4F801D0
:1048800081938F01F70101900020E9F73197EE192C
:10489000FF09802F8E198E176CF327968FAD2797FF
:1048A0008E3751F1C701B20145E050E00E94DAD4E1
:1048B000009711F500D000D0EDB7FEB73196ADB737
:1048C000BEB712967C926E921197338222825582E5
:1048D00044820E9417D5EDB7FEB736960FB6F8940E
:1048E000FEBF0FBEEDBFC3010E94575488E792E0A0
:1048F0000E94DE5399249394C501B70140E050E033
:104900000E94CC72181614F48701BCCF992041F490
:104910008FEF9FEFD6019E969C938E939D9706C036
:10492000F60185A596A5019696A785A729EA31E007
:10493000C20ED31ED6011C92C45ADF4F0FB6F89494
:10494000DEBF0FBECDBFCF91DF911F910F91FF90C2
:10495000EF90DF90CF90BF90AF909F907F906F903F
:104960005F904F903F902F9008952F923F924F92DB
:104970005F926F927F928F929F92AF92BF92CF92EF
:10498000DF92EF92FF920F931F93DF93CF93CDB7F8
:10499000DEB7CD58D0400FB6F894DEBF0FBECDBF06
:1049A0008C013B016A0184E090E0C80ED91EF80139
:1049B0007196C757DF4FF983E883C958D040C801C3
:1049C0000496C957DF4F99838883C758D040CA5788
:1049D000DF4F1882C658D04036E6E32EF12CEC0E9D
:1049E000FD1E27EF822E21E0922E800E911E98EF61
:1049F000A92E91E0B92EA00EB11E8EE0282E312CEA
:104A00002C0E3D1EB7E44B2E512C4C0E5D1EF201B8
:104A10003496C557DF4FF983E883CB58D040ECE597
:104A2000F2E08491C357DF4F8883CD58D04021C135
:104A3000F7018385282F30E0A9014871507040317B
:104A4000510509F024C1F4019081913009F41FC18E
:104A5000923009F41CC1CE010196B7010E94861C58
:104A60001E86F3018081882329F4C10160E072E091
:104A70000E94BDD4C101B3010E94BDD4C101BE01D9
:104A80006F5F7F4F0E94BDD4C10160E072E00E9461
:104A9000BDD41CA61FA61BA61AA68AE194E099A75E
:104AA00088A7CE018C96B601AE014F5F5F4F21E023
:104AB0000E940F78882309F03EC0F401808188238A
:104AC000D1F5C357DF4F9881CD58D040ECE5F2E0E7
:104AD00008C08091C00085FFFCCF9093C60031963E
:104AE00094919923B1F7E2E0F2E007C08091C00011
:104AF00085FFFCCF31969093C60090819923B1F742
:104B00008091C00085FFFCCFFAE0F093C600FE0163
:104B1000319607C08091C00085FFFCCF31969093FD
:104B2000C60090819923B1F78091C00085FFFCCF2A
:104B30008AE08093C600C557DF4FA881B981CB5862
:104B4000D040FE01BC968BE101900D928150E1F7BF
:104B50008AA59BA5F201938382838AE194E09183E5
:104B60008083C801B101A20100DFC2010E94181DAB
:104B7000CE0188960E94181D7CC0953E09F479C02C
:104B80009E3209F476C09F3509F473C0F80191890B
:104B9000992331F09E3209F46CC09F3509F469C045
:104BA00023FD67C080E04031510509F481E0F80140
:104BB00084A7882349F4F7018085873409F059C018
:104BC00081858E3709F455C0C957DF4F8881998197
:104BD000C758D040B7010E94861CF4018081882309
:104BE00029F5F30107C08091C00085FFFCCF319605
:104BF0009093C60090819923B1F7C957DF4FE881A0
:104C0000F981C758D04007C08091C00085FFFCCF14
:104C100031969093C60090819923B1F78091C0009E
:104C200085FFFCCFFAE0F093C60023C0813039F451
:104C3000F501808191810196918380831AC0823031
:104C4000C1F4CA57DF4FF881C658D0402F2F30E04B
:104C5000F5018081918128173907F1F0CA57DF4F9C
:104C6000F881C658D040FF5FCA57DF4FF883C65857
:104C7000D040C601B701C757DF4F48815981C95895
:104C8000D0400E94CC7218160CF4D2CE05C0F701A9
:104C90009081992309F071CFC357DF4F0FB6F89475
:104CA000DEBF0FBECDBFCF91DF911F910F91FF905F
:104CB000EF90DF90CF90BF90AF909F908F907F90BC
:104CC0006F905F904F903F902F900895EF92FF92DA
:104CD0000F931F93DF93CF93CDB7DEB76F970FB6C8
:104CE000F894DEBF0FBECDBF7C018C01015B1F4F6E
:104CF0008F5A9F4FF8019183808327EF31E0E20EB6
:104D0000F31E21E0F70121937F011182108228E038
:104D10003EEFE20EF31E049640E050E060E070E0EB
:104D20000E94BD6FF80120813181DE011596F901E5
:104D300034968BE101900D928150E1F7F901828167
:104D400093819C838B838AE194E09A838983C70152
:104D500065E172E08E010F5F1F4FA80106DEC801FA
:104D60000E94181DF701E850FE4F808191816F96D7
:104D70000FB6F894DEBF0FBECDBFCF91DF911F916C
:104D80000F91FF90EF900895EF92FF920F931F9372
:104D9000DF93CF93CDB7DEB76F970FB6F894DEBF32
:104DA0000FBECDBF7C018C01015B1F4F8F5A9F4FFF
:104DB000F8019183808327EF31E0E20EF31E22E0B9
:104DC000F701208329E03EEFE20EF31EF701E850E1
:104DD000FE4F60831182049640E050E060E070E096
:104DE0000E94BD6FF80120813181DE011596F90125
:104DF00034968BE101900D928150E1F7F9018281A7
:104E000093819C838B838AE194E09A838983C70191
:104E100065E172E08E010F5F1F4FA801A6DDC8019A
:104E20000E94181D6F960FB6F894DEBF0FBECDBF5F
:104E3000CF91DF911F910F91FF90EF900895EF9226
:104E4000FF920F931F93DF93CF93CDB7DEB76F978A
:104E50000FB6F894DEBF0FBECDBF7C0187EF91E0A7
:104E6000E80EF91EF701108289E09EEFE80EF91EA8
:104E700087010C5C1F4FC80140E050E060E070E02B
:104E80000E94BD6FDE011596F8018BE101900D9235
:104E90008150E1F7F70182A993A99C838B838AE172
:104EA00094E09A838983C70165E172E08E010F5F08
:104EB0001F4FA8015ADDC8010E94181D6F960FB63A
:104EC000F894DEBF0FBECDBFCF91DF911F910F9140
:104ED000FF90EF9008950F931F93CF93DF93DC0122
:104EE000D4961C92D497D7961C92D797D3961C929F
:104EF0001E92D2978AE194E0D1969C938E93D0979C
:104F0000AB5ABF4F1C9213961C92A855B040FD019E
:104F1000EF5AFF4FAD5ABF4F11961C921E92A355E8
:104F2000B04091838083ED01C059DF4FFE0120E046
:104F300030E0482F148217821382128240839183BB
:104F4000215E3F4F7F9681E02633380799F7A755BA
:104F5000BE4F89E18C9313961C9258961C921B9617
:104F60001C9213961C92A25DB140FD01E553FE4FC9
:104F7000A353BE4F11961C921E92408391835D965F
:104F80001D921D921D921C92139718961D921D92B0
:104F90001D921C921397A25FB14012961C92129719
:104FA0009F961C929F971C9211961C9211978D01AF
:104FB00002511E4FF8011082118212821382AA55EB
:104FC000BE4F1C92FE01C90111920197E9F7A05B47
:104FD000BF4F81E08C93A65FB1409E961C921E92BB
:104FE0009D970E94531A68577C4E8F4F9F4FF80130
:104FF0006083718382839383DF91CF911F910F919F
:105000000895DF93CF93CDB7DEB7E0970FB6F8944E
:10501000DEBF0FBECDBFDE011196EAECF3E080E10A
:1050200001900D928150E1F7DE015196EAEBF3E039
:1050300080E101900D928150E1F7DE019196EAEA5C
:10504000F3E080E101900D928150E1F789819A812E
:10505000AB81BC818093590A90935A0AA0935B0A52
:10506000B0935C0A89899A89AB89BC898093490A83
:1050700090934A0AA0934B0AB0934C0A89A19AA133
:10508000ABA1BCA180936D0A90936E0AA0936F0AA6
:10509000B093700A8D819E81AF81B88580935D0A3F
:1050A00090935E0AA0935F0AB093600A8D899E89EF
:1050B000AF89B88D80934D0A90934E0AA0934F0A02
:1050C000B093500A8DA19EA1AFA1B8A58093710A9B
:1050D0009093720AA093730AB093740A89859A8593
:1050E000AB85BC858093610A9093620AA093630AA2
:1050F000B093640A898D9A8DAB8DBC8D8093510AD3
:105100009093520AA093530AB093540A89A59AA582
:10511000ABA5BCA58093750A9093760AA093770AF5
:10512000B093780A8D859E85AF85B8898093650A8E
:105130009093660AA093670AB093680A8D8D9E8D3E
:10514000AF8DB8A18093550A9093560AA093570A41
:10515000B093580A8DA59EA5AFA5B8A98093790AEA
:1051600090937A0AA0937B0AB0937C0A0E94A85A73
:1051700080E090E4ACE9B5E48093810A9093820AE0
:10518000A093830AB093840A8093850A9093860A39
:10519000A093870AB093880A20E030E040E050E016
:1051A00020937D0A30937E0A40937F0A5093800AB1
:1051B00080E29EE4A0E0B0E08093450A9093460A26
:1051C000A093470AB093480A2093950A3093960A11
:1051D0004093970A5093980A80E090E0A0EAB1E4E7
:1051E0008093890A90938A0AA0938B0AB0938C0AC1
:1051F0008DEC9CECACECBEE380938D0A90938E0A10
:10520000A0938F0AB093900A80E090E0A0EAB0E407
:105210008093910A9093920AA093930AB093940A70
:1052200020934C0630934D0640934E0650934F0604
:10523000209348063093490640934A0650934B0604
:105240002093440630934506409346065093470604
:1052500086E696E6A2E4B1E4809385039093860304
:10526000A0938703B093880360E070E080E89FE339
:105270000E946C876093890370938A0380938B03E9
:1052800090938C036BE774E184E192E40E94788749
:1052900060938D0370938E0380938F03909390039C
:1052A0000E94608680E090E0A0E8BFE380939103D5
:1052B00090939203A0939303B093940384E195E0B9
:1052C00090937B0380937A0390937D0380937C0378
:1052D00082EE94E090937F0380937E0384E6809334
:1052E000A90310926812EAECF3E0949108C080914F
:1052F000C00085FFFCCF9093C6003196949199230E
:10530000B1F7E0EDF3E0949108C08091C00085FF13
:10531000FCCF9093C600319694919923B1F7809178
:10532000C00085FFFCCF8AE08093C600E0960FB6F0
:10533000F894DEBF0FBECDBFCF91DF910895CF931C
:10534000DF93CAECD3E0FE01949108C08091C000C5
:1053500085FFFCCF9093C600319694919923B1F7C5
:10536000E4ECF5E0949108C08091C00085FFFCCF8B
:105370009093C600319694919923B1F78091C00023
:1053800085FFFCCF8AE08093C600FE019491EAEC91
:10539000F3E008C08091C00085FFFCCF9093C60069
:1053A000319694919923B1F74091590A50915A0A34
:1053B00060915B0A70915C0A8CEB95E00E9411345D
:1053C00040915D0A50915E0A60915F0A7091600A97
:1053D00089EB95E00E9411344091610A5091620A74
:1053E0006091630A7091640A86EB95E00E94113423
:1053F0004091650A5091660A6091670A7091680A47
:1054000083EB95E00E941134E6E1F2E007C0809161
:10541000C00085FFFCCF31969093C6009081992300
:10542000B1F78091C00085FFFCCF8AE08093C60071
:10543000FE019491EAECF3E008C08091C00085FF82
:10544000FCCF9093C600319694919923B1F7E9E986
:10545000F5E0949108C08091C00085FFFCCF909347
:10546000C600319694919923B1F78091C00085FFD1
:10547000FCCF8AE08093C600FE019491EAECF3E051
:1054800008C08091C00085FFFCCF9093C600319684
:1054900094919923B1F74091490A50914A0A609139
:1054A0004B0A70914C0A80E995E00E9411344091BA
:1054B0004D0A50914E0A60914F0A7091500A8DE842
:1054C00095E00E9411344091510A5091520A609126
:1054D000530A7091540A8AE895E00E941134409171
:1054E000550A5091560A6091570A7091580A87E8F8
:1054F00095E00E941134E6E1F2E007C08091C0001F
:1055000085FFFCCF31969093C60090819923B1F727
:105510008091C00085FFFCCF8AE08093C600FE0129
:105520009491EAECF3E008C08091C00085FFFCCFC5
:105530009093C600319694919923B1F7E9E6F5E08E
:10554000949108C08091C00085FFFCCF9093C60065
:10555000319694919923B1F78091C00085FFFCCFDB
:105560008AE08093C600FE019491EAECF3E008C063
:105570008091C00085FFFCCF9093C6003196949136
:105580009923B1F740916D0A50916E0A60916F0AAC
:105590007091700A80E695E00E9424344091710A6F
:1055A0005091720A6091730A7091740A8DE595E0CA
:1055B0000E9424344091750A5091760A6091770ACE
:1055C0007091780A8AE595E00E9424344091790A26
:1055D00050917A0A60917B0A70917C0A87E595E088
:1055E0000E942434E6E1F2E007C08091C00085FF0C
:1055F000FCCF31969093C60090819923B1F78091AA
:10560000C00085FFFCCF8AE08093C600FE01949124
:10561000EAECF3E008C08091C00085FFFCCF9093D6
:10562000C600319694919923B1F7E2E2F5E09491A6
:1056300008C08091C00085FFFCCF9093C6003196D2
:1056400094919923B1F78091C00085FFFCCF8AE047
:105650008093C600FE019491EAECF3E008C08091CB
:10566000C00085FFFCCF9093C6003196949199239A
:10567000B1F74091810A5091820A6091830A70913A
:10568000840A89E195E00E9411344091850A509185
:10569000860A6091870A7091880A86E195E00E94E7
:1056A0001134E6E1F2E007C08091C00085FFFCCF35
:1056B00031969093C60090819923B1F78091C000F4
:1056C00085FFFCCF8AE08093C600FE019491EAEC4E
:1056D000F3E008C08091C00085FFFCCF9093C60026
:1056E000319694919923B1F7E3E6F4E0949108C0E0
:1056F0008091C00085FFFCCF9093C60031969491B5
:105700009923B1F78091C00085FFFCCF8AE0809398
:10571000C600FE019491EAECF3E008C08091C0005D
:1057200085FFFCCF9093C600319694919923B1F7F1
:1057300040917D0A50917E0A60917F0A7091800AA3
:105740008AE594E00E9411344091950A5091960A9E
:105750006091970A7091980A87E594E00E9411344D
:105760004091450A5091460A6091470A7091480A53
:1057700084E594E00E9424344091890A50918A0A79
:1057800060918B0A70918C0A81E594E00E9411343B
:1057900040918D0A50918E0A60918F0A7091900A03
:1057A0008EE494E00E9411344091910A5091920A43
:1057B0006091930A7091940A8BE494E00E941134F2
:1057C000E6E1F2E007C08091C00085FFFCCF319692
:1057D0009093C60090819923B1F78091C00085FF16
:1057E000FCCF8AE08093C600FE019491EAECF3E0DE
:1057F00008C08091C00085FFFCCF9093C600319611
:1058000094919923B1F7E9E3F4E0949108C0809171
:10581000C00085FFFCCF9093C600319694919923E8
:10582000B1F78091C00085FFFCCF8AE08093C6006D
:10583000FE019491EAECF3E008C08091C00085FF7E
:10584000FCCF9093C600319694919923B1F7409183
:10585000440650914506609146067091470680E3E4
:1058600094E0DFD7409148065091490660914A067E
:1058700070914B068DE294E0D4D740914C06509144
:105880004D0660914E0670914F068AE294E0C9D7AA
:10589000E6E1F2E007C08091C00085FFFCCF3196C1
:1058A0009093C60090819923B1F78091C00085FF45
:1058B000FCCF8AE08093C600FE019491EAECF3E00D
:1058C00008C08091C00085FFFCCF9093C600319640
:1058D00094919923B1F7ECE1F4E0949108C08091A0
:1058E000C00085FFFCCF9093C60031969491992318
:1058F000B1F78091C00085FFFCCF8AE08093C6009D
:10590000FE019491EAECF3E008C08091C00085FFAD
:10591000FCCF9093C600319694919923B1F74091B2
:10592000850350918603609187037091880382E11B
:1059300094E077D76091890370918A0380918B03FB
:1059400090918C030E947287AB01BC018FE094E0C0
:1059500068D760918D0370918E0380918F03909131
:1059600090030E947E87AB01BC018CE094E059D784
:10597000E6E1F2E007C08091C00085FFFCCF3196E0
:105980009093C60090819923B1F78091C00085FF64
:10599000FCCF8AE08093C600DF91CF910895EF920B
:1059A000FF921F93CF93DF93EC017B01142F88812B
:1059B00099810E94B1DBF70181937F0188819981F0
:1059C000019699838883115091F7DF91CF911F91B0
:1059D000FF90EF900895EF92FF920F931F93DF9344
:1059E000CF93CDB7DEB766970FB6F894DEBF0FBE84
:1059F000CDBF84E690E09A838983809117029091CD
:105A00001802A0911902B0911A028B8B9C8BAD8B5E
:105A1000BE8B8E01015F1F4F7E010894E11CF11CBB
:105A2000C701B80144E0BBDFCE014396B80143E0B3
:105A300050E00E94DAD4009709F0A6C0C70169E5DA
:105A40007AE040E1ACDFC70169E47AE040E1A7DF3A
:105A5000C7016DE67AE040E1A2DF0E94A85AC701C3
:105A600061E87AE044E09BDFC70165E87AE044E062
:105A700096DFC7016DE77AE044E091DFC70165E991
:105A80007AE044E08CDFC70165E47AE044E087DF38
:105A9000C70169E87AE044E082DFC7016DE87AE097
:105AA00044E07DDFC70161E97AE044E078DFC701C7
:105AB00064E476E04CE073DFC701BE016D5F7F4FA9
:105AC00042E06DDFC701BE016B5F7F4F42E067DFE1
:105AD000C701BE01695F7F4F42E061DFC701BE01C0
:105AE000675F7F4F42E05BDFC701BE01655F7F4FAD
:105AF00042E055DFC701BE01635F7F4F42E04FDFE9
:105B0000C70165E873E044E04ADFC70169E873E074
:105B100044E045DFC7016DE873E044E040DFC701C2
:105B20006AE773E046E03BDFC70169EA73E041E002
:105B300036DFC70168E672E141E031DF0E9460862E
:105B4000EAECF3E0949108C08091C00085FFFCCF9F
:105B50009093C600319694919923B1F7E2EFF3E068
:105B6000949108C08091C00085FFFCCF9093C6003F
:105B7000319694919923B1F78091C00085FFFCCFB5
:105B80008AE08093C60001C03CDAD9DB66960FB686
:105B9000F894DEBF0FBECDBFCF91DF911F910F9163
:105BA000FF90EF900895EF92FF921F93CF93DF93B2
:105BB000EC017B01142F88819981F70161917F01AC
:105BC0000E94CCDB8881998101969983888311504A
:105BD00091F7DF91CF911F91FF90EF900895EF9291
:105BE000FF920F931F93DF93CF93CDB7DEB76697E6
:105BF0000FB6F894DEBF0FBECDBF80911B0290910F
:105C00001C02A0911D02B0911E028F87988BA98B58
:105C1000BA8B84E6E82EF12CFA82E9828E010F5FBE
:105C20001F4FC801BE01615F7F4F44E0BCDFC80168
:105C300069E57AE040E1B7DFC80169E47AE040E174
:105C4000B2DFC8016DE67AE040E1ADDFC80161E88E
:105C50007AE044E0A8DFC80165E87AE044E0A3DF29
:105C6000C8016DE77AE044E09EDFC80165E97AE0AB
:105C700044E099DFC80165E47AE044E094DFC801BC
:105C800069E87AE044E08FDFC8016DE87AE044E03B
:105C90008ADFC80161E97AE044E085DFC80164E495
:105CA00076E04CE080DF84EB90E09C838B8386E49D
:105CB00090E09E838D8318861F8280EF90E09A8704
:105CC0008987FC86EB861E861D86C801BE016D5F36
:105CD0007F4F42E068DFC801BE016B5F7F4F42E04B
:105CE00062DFC801BE01695F7F4F42E05CDFC8012F
:105CF000BE01675F7F4F42E056DFC801BE01655FAE
:105D00007F4F42E050DFC801BE01635F7F4F42E03A
:105D10004ADFC80165E873E044E045DFC80169E88F
:105D200073E044E040DFC8016DE873E044E03BDF2E
:105D3000C8016AE773E046E036DFC80169EA73E04C
:105D400041E031DFC80168E672E141E02CDF80917B
:105D5000170290911802A0911902B0911A028B8B30
:105D60009C8BAD8BBE8BFA82E982C801BE016D5E51
:105D70007F4F44E018DFEAECF3E0949108C0809193
:105D8000C00085FFFCCF9093C60031969491992373
:105D9000B1F7E4EDF5E0949108C08091C00085FF73
:105DA000FCCF9093C600319694919923B1F78091DE
:105DB000C00085FFFCCF8AE08093C60066960FB6D0
:105DC000F894DEBF0FBECDBFCF91DF911F910F9131
:105DD000FF90EF900895DF93CF930F920F92CDB77E
:105DE000DEB72091531730915417CE01019621153B
:105DF000310519F48955974102C0821B930B9A8390
:105E0000898389819A810F900F90CF91DF910895B6
:105E1000089520E08091BA099091BB0918161906DF
:105E20000CF421E0822F0895EF92FF920F931F93BD
:105E3000CF93DF93EC01E0905006F0905106009173
:105E4000520610915306688179818A819B81A8014D
:105E500097010E9421D6882324F4E882F9820A83DC
:105E60001B83E0905406F090550600915606109161
:105E700057066C817D818E819F81A80197010E94C8
:105E800021D6882324F4EC82FD820E831F83E090C8
:105E90005806F090590600915A0610915B066885E5
:105EA00079858A859B85A80197010E9421D6882340
:105EB00024F4E886F9860A871B87E0905003F09067
:105EC00051030091520310915303688179818A81B3
:105ED0009B81A80197010E9424D8181624F4E88217
:105EE000F9820A831B83E0905403F09055030091DC
:105EF0005603109157036C817D818E819F81A8018B
:105F000097010E9424D8181624F4EC82FD820E8397
:105F10001F83E0905803F090590300915A031091A9
:105F20005B03688579858A859B85A80197010E9416
:105F300024D8181624F4E886F9860A871B87DF918F
:105F4000CF911F910F91FF90EF90089580916D0672
:105F5000811181E0089580916D060895CF93DF93BC
:105F60008130910541F46F5F7F4FF9F482E394E053
:105F70000E946B271AC0892BC1F46F5F7F4FA9F471
:105F80008DEF95E00E94181DC9EBD5E0CE010E946F
:105F9000181D6F9784E0C338D807C1F7CE010E945F
:105FA000181DCE0181970E94181DDF91CF91089591
:105FB00080E090E06FEF7FEFD1CF81E090E06FEF76
:105FC0007FEFCCCF1F93182F0E94498780916D06D9
:105FD000882309F035C010936D0680916F0690916B
:105FE0007006A0917106B09172068093730690932B
:105FF0007406A0937506B0937606EAEEF5E09491E8
:1060000008C08091C00085FFFCCF9093C6003196F8
:1060100094919923B1F7E1EFF5E0949108C0809154
:10602000C00085FFFCCF9093C600319694919923D0
:10603000B1F78091C00085FFFCCF8AE08093C60055
:106040001F910895F8940E944987159A469A439A99
:10605000409A8CE060E00E94A11BEAEEF5E094918A
:1060600008C08091C00085FFFCCF9093C600319698
:1060700094919923B1F7E7E6F6E0949108C08091F6
:10608000C00085FFFCCF9093C60031969491992370
:10609000B1F78091C00085FFFCCF8AE08093C600F5
:1060A000FFCF0E94531A609377067093780680930F
:1060B000790690937A06E091A006F091A106EE553C
:1060C000F94F80818823A9F4E6E8F6E0949108C0AE
:1060D0008091C00085FFFCCF9093C60031969491CB
:1060E0009923B1F78091C00085FFFCCF8AE08093AF
:1060F000C6000895EF92FF920F931F930E94531AC8
:10610000E0907B06F0907C0600917D0610917E0663
:1061100020917706309178064091790650917A0661
:10612000621B730B840B950BE616F706080719071D
:1061300030F4E114F1040105110509F083DF8091C9
:106140006D0390916E03A0916F03B091700300975F
:10615000A105B105F9F00E94531A209177063091FC
:1061600078064091790650917A06621B730B840B76
:10617000950B20916D0330916E0340916F03509108
:106180007003261737074807590720F48091890FB5
:1061900080918A0F069B02C08AE014DF0E94335D63
:1061A0001F910F91FF90EF9008956F927F928F92C1
:1061B0009F92AF92BF92CF92DF92EF92FF920F9396
:1061C0001F93F82E60917F06709180068091810662
:1061D0009091820620918306309184064091850635
:1061E000509186060E9431D83B014C0100D000D06E
:1061F0000DB71EB70F5F1F4F60914C0370914D0399
:10620000882777FD8095982F0E94C3D6209171032F
:106210003091720340917303509174030E94F6D839
:1062200020E030E040E752E40E9428D620E030E051
:1062300048EC52E40E9428D65B016C01F8016082B0
:10624000718282829382F48280915C06858384E3EA
:1062500096E06BE876E04FE756E020E001E032E0C0
:10626000E32E0E941B5780918B0690918C06A09183
:106270008D06B0918E068093340690933506A093D8
:106280003606B093370680918F0690919006A091C4
:106290009106B09192068093380690933906A093A8
:1062A0003A06B0933B068091930690919406A09194
:1062B0009506B091960680933C0690933D06A09378
:1062C0003E06B0933F068091970690919806A09164
:1062D0009906B0919A068093400690934106A09348
:1062E0004206B09343068DB79EB706960FB6F89454
:1062F0009EBF0FBE8DBF0E94531A609377067093A6
:1063000078068093790690937A061F910F91FF90FB
:10631000EF90DF90CF90BF90AF909F908F907F9045
:106320006F900895CF92DF92EF92FF920F931F9399
:106330008BE896E079DD0E94531A6093770670939C
:1063400078068093790690937A066091340670916E
:106350003506809136069091370620918B06309154
:106360008C0640918D0650918E060E9421D688237E
:1063700009F07AC0609138067091390680913A062A
:1063800090913B0620918F063091900640919106A6
:10639000509192060E9421D6882309F065C0609131
:1063A000710370917203809173039091740320E0E4
:1063B00030E040E752E40E9428D67B018C018BE854
:1063C00096E06FE876E043E956E027E936E0ECE551
:1063D000CE2EE6E0DE2E0E945C6080918B069091CE
:1063E0008C06A0918D06B0918E0680933406909312
:1063F0003506A0933606B093370680918F069091AC
:106400009006A0919106B0919206809338069093E1
:106410003906A0933A06B0933B068091930690917B
:106420009406A0919506B091960680933C069093B1
:106430003D06A0933E06B0933F068091970690914B
:106440009806A0919906B0919A0680934006909381
:106450004106A0934206B09343061F910F91FF900F
:10646000EF90DF90CF90089560914C0370914D03B1
:10647000882777FD8095982F0E94C3D620917103BD
:106480003091720340917303509174030E94F6D8C7
:1064900020E030E040E752E40E9428D620E030E0DF
:1064A00048EC52E488CF84E49AE00E945755E9E82A
:1064B000F6E0949108C08091C00085FFFCCF9093D6
:1064C000C600319694919923B1F740916F0650918F
:1064D000700660917106709172064F5F5F4F6F4F4B
:1064E0007F4F84E49AE02AE030E00E9413568091C6
:1064F000C00085FFFCCF8AE08093C600D2CD2F92EA
:106500003F924F925F926F927F928F929F92AF9243
:10651000BF92CF92DF92EF92FF920F931F93DF9380
:10652000CF9300D000D0CDB7DEB78C01833091057A
:1065300008F040C13C01660C771C660C771C930187
:106540002C5C394F3A83298380E090E0A0E0B0E0F2
:10655000F90180839183A283B38384E396E068E3A7
:1065600076E04CE356E020E436E00E94FF5AF30167
:10657000EF5DF74F6591759185919491075C174F89
:10658000F801E49093012557394F3E832D8320E095
:1065900030E040EC5FE30E94F6D85B016C01FF2421
:1065A000E7FCF0940F2D1F2DC801B7010E94C3D640
:1065B0001B012C01C601B501A20191010E94F6D870
:1065C000AD81BE816D937D938D939C931397F30161
:1065D000E45CFC4FFC83EB83608171818281938159
:1065E00060937103709372038093730390937403A9
:1065F00020E030E040E752E40E9428D67B018C0185
:106600008BE896E06FE876E043E956E027E936E06C
:10661000FCE5CF2EF6E0DF2E0E945C600E94497FF1
:1066200080E090E0A0E0B0E0E981FA81808391838E
:10663000A283B38384E396E068E376E04CE356E01C
:1066400020E436E00E94FF5AF301E35DF74F8590A6
:106650009590A590B490C501B4019058A201910104
:106660000E94F6D8AD81BE816D937D938D939C93EE
:1066700013976091710370917203809173039091ED
:10668000740320E030E040E752E40E9428D67B010A
:106690008C018BE896E06FE876E043E956E027E965
:1066A00036E00E945C600E94497FC501B401A501EB
:1066B00094010E9448D5A20191010E94F6D8ED8173
:1066C000FE816083718382839383AB81BC816D91F2
:1066D0007D918D919C9120E030E040E450E40E9457
:1066E00028D6609371037093720380937303909321
:1066F000740320E030E040E752E40E9428D67B019A
:106700008C018BE896E06FE876E043E956E027E9F4
:1067100036E00E945C600E94497FF301E350F84F2D
:106720006591759185919491F301EC5BF94F20810E
:106730003181428153810E9448D59B01AC01E9819E
:10674000FA812083318342835383F301E75FF74F5C
:106750002591359145915491F301E05BF94F2083E8
:10676000318342835383F301EB5EF74F25913591DB
:1067700045915491A0E5B3E06A0E7B1EF30120839E
:10678000318342835383AC01CB01DA01ED81FE8179
:1067900080839183A283B38380E090E0A0E0B0E0A7
:1067A0008093710390937203A0937303B093740367
:1067B0000E94D87D26960FB6F894DEBF0FBECDBFDF
:1067C000CF91DF911F910F91FF90EF90DF90CF90CD
:1067D000BF90AF909F908F907F906F905F904F9001
:1067E0003F902F900895682F2091A0063091A10628
:1067F00080E690E0AC01249FC001259F900D349F5E
:10680000900D11248055994F70E00E94C8D49C01CE
:106810009093AF068093AE0680E0232B09F081E0D1
:106820000895FC01949108C08091C00085FFFCCFC1
:106830009093C600319694919923B1F784E49AE03D
:1068400022E030E00C941957FC01949108C080912B
:10685000C00085FFFCCF9093C60031969491992398
:10686000B1F784E49AE02AE030E00C94F755809187
:10687000AE069091AF06019660E070E04AE050E00D
:106880000C94CDD28091AE069091AF06019660E057
:1068900070E00C9467D1CF93DF93EC0180915C069C
:1068A00080936E0684E59FDF882309F46EC0EADFDB
:1068B0000E9495D6262F60936E06662309F465C064
:1068C000E4EEF5E0949108C08091C00085FFFCCF14
:1068D0009093C600319694919923B1F7C936D105AA
:1068E00099F0CA36D10524F4C836D105F1F50FC0A8
:1068F000CD36D10531F0CA3DD105B9F5EFE1F2E071
:1069000031C0E6E3F2E023C0EDE4F2E015C0E4E6D6
:10691000F2E007C08091C00085FFFCCF31969093D4
:10692000C60090819923B1F720C08091C00085FFF7
:10693000FCCF31969093C60090819923B1F715C092
:106940008091C00085FFFCCF31969093C600908166
:106950009923B1F70AC08091C00085FFFCCF319622
:106960009093C60090819923B1F784E49AE0622F56
:1069700040E050E00E9402568091C00085FFFCCFAD
:106980008AE08093C60081E001C080E0DF91CF9172
:1069900008955F926F927F928F929F92AF92BF9273
:1069A000CF92DF92EF92FF920F931F93DF93CF93DB
:1069B00000D00F92CDB7DEB719821A821B821C82DB
:1069C00014E3C12E16E0D12EBBE8EB2EB6E0FB2E71
:1069D00000E010E03E010894611C711C55245394A2
:1069E000F801E652FC4F8081FEDE882359F14ADF30
:1069F0004B015C01F801E25DF94F8081882311F0C1
:106A000061E002C060919B0670E0882777FD809569
:106A1000982F0E94C3D6F601208131814281538193
:106A20000E94F6D89B01AC01C501B4010E9448D573
:106A3000F7016083718382839383F301E00FF11F79
:106A400050820AC0F60180819181A281B381F70151
:106A500080839183A283B3830F5F1F4F84E090E014
:106A6000C80ED91EE80EF91E0430110509F0B8CF82
:106A700086E4B9DE8823D9F005DF7B018C016093C1
:106A80009C0670939D0680939E0690939F0620E03F
:106A900030E040E050E00E9424D8181644F4E09220
:106AA0007103F09272030093730310937403809147
:106AB0005E06882309F4C1C08981882309F0BDC01E
:106AC0008A81882309F0B9C08B81882309F0B5C079
:106AD0008C81882309F4B1C0A0904006B090410693
:106AE000C0904206D0904306609197067091980638
:106AF0008091990690919A06A60195010E9447D52A
:106B00007B018C012DEC3CEC4CEC5DEB0E9421D622
:106B100088230CF04EC080915F06882309F08DC059
:106B200060919306709194068091950690919606D7
:106B3000209165033091660340916703509168038B
:106B40000E9448D5609393067093940680939506AF
:106B500090939606C801B701905820915D0330913B
:106B60005E0340915F03509160030E9447D59B01F3
:106B7000AC01C601B5010E9447D5609340067093F1
:106B80004106809342069093430680916103909161
:106B90006203A0916303B0916403809371039093A7
:106BA0007203A0937303B093740381E080935F0634
:106BB00044C0C801B7012DEC3CEC4CEC5DE30E94F5
:106BC00024D81816D4F580915F068823B1F160911E
:106BD0005D0370915E0380915F0390916003A80153
:106BE00097010E9447D5209160063091610640913F
:106BF0006206509163060E9448D59B01AC01C60114
:106C0000B5010E9448D56093400670934106809379
:106C10004206909343068091690390916A03A09184
:106C20006B03B0916C038093710390937203A093F4
:106C30007303B093740310925F060F900F900F9040
:106C40000F90CF91DF911F910F91FF90EF90DF9008
:106C5000CF90BF90AF909F908F907F906F905F90FC
:106C6000089597DE89E4BFDD882351F00BDE609341
:106C70007F067093800680938106909382060CC0F5
:106C800080E090E0A0E0B0E080937F0690938006E3
:106C9000A0938106B09382068AE4A5DD882351F093
:106CA000F1DD60938306709384068093850690934C
:106CB0008606089580E090E0A0E0B0E0809383062F
:106CC00090938406A0938506B093860608952F922C
:106CD0003F924F925F926F927F928F929F92AF926C
:106CE000BF92CF92DF92EF92FF920F931F93DF93A9
:106CF000CF93CDB7DEB76E970FB6F894DEBF0FBE59
:106D0000CDBF1092640687E46EDD882309F44DC67A
:106D1000B9DD0E9490D66A30710509F48BC06B30E2
:106D200071059CF46230710599F16330710524F4AA
:106D3000772334F50C94054D6330710581F164308F
:106D4000710511F00C94054D33C06A35710509F4D5
:106D5000D7C56B35710554F46B30710509F405C165
:106D60006C31710511F00C94054D74C16B357105D2
:106D700009F4CAC56C35710511F00C94054DC9C5EF
:106D800080916D06882321F404DECCDA0C94284D22
:106D900080916D06882319F464DF81E006C080913C
:106DA0006D06882329F45DDF80E0FFD90C94284D1F
:106DB00080E519DD882321F4EE24FF24870105C036
:106DC00061DD0E9495D67B018C0183E50CDD882373
:106DD00059F058DD20E030E04AE754E40E94F6D84C
:106DE0000E9495D67B018C010E94497F0E94531A14
:106DF0005B016C01AE0CBF1CC01ED11E0E94531A59
:106E000060937706709378068093790690937A065C
:106E100081E08093640605C00E94798B6BD90E9443
:106E2000CB940E94531A6A157B058C059D05A0F32F
:106E30000C94054D80915F06882311F00C94054D4C
:106E40008091340690913506A0913606B0913706B0
:106E500080938B0690938C06A0938D06B0938E063C
:106E60008091380690913906A0913A06B0913B0680
:106E700080938F0690939006A0939106B09392060C
:106E800080913C0690913D06A0913E06B0913F0650
:106E90008093930690939406A0939506B0939606DC
:106EA000E0915C06F0E0EE0FFF1FEE0FFF1FE759C9
:106EB000F54F60915D0370915E0380915F03909147
:106EC000600320813181428153810E9428D69B0139
:106ED000AC0160914006709141068091420690910C
:106EE00043060E9447D59B01AC01609397067093BF
:106EF00098068093990690939A06E0907103F0901B
:106F00007203009173031091740380916103909157
:106F10006203A0916303B091640380937103909323
:106F20007203A0937303B093740360914006709151
:106F3000410680914206909143060E9447D5609396
:106F4000600670936106809362069093630681E009
:106F500080935F06E7D9E0927103F0927203009389
:106F60007303109374030C94054D80915F0688237E
:106F700011F40C94054D8091340690913506A09142
:106F80003606B091370680938B0690938C06A093BB
:106F90008D06B0938E068091380690913906A091A7
:106FA0003A06B0913B0680938F0690939006A0938B
:106FB0009106B093920680913C0690913D06A09177
:106FC0003E06B0913F068093930690939406A0935B
:106FD0009506B093960660914006709141068091A7
:106FE00042069091430620916006309161064091DF
:106FF0006206509163060E9448D56093970670938D
:1070000098068093990690939A06E0907103F09009
:10701000720300917303109174038091690390913E
:107020006A03A0916B03B0916C03809371039093FA
:107030007203A0937303B093740310925F0672D926
:10704000E0927103F0927203009373031093740340
:107050000C94054D85E080936406809171039091B6
:107060007203A0917303B09174038093AA06909366
:10707000AB06A093AC06B093AD0680914C03909103
:107080004D03909333068093320684E690E090930C
:107090004D0380934C030E94531A609377067093BC
:1070A00078068093790690937A0681E00E94DF7DCE
:1070B0008091340690913506A0913606B09137063E
:1070C00080938B0690938C06A0938D06B0938E06CA
:1070D0008091380690913906A0913A06B0913B060E
:1070E00080938F0690939006A0939106B09392069A
:1070F00080913C0690913D06A0913E06B0913F06DE
:107100008093930690939406A0939506B093960669
:107110008091400690914106A0914206B0914306AD
:107120008093970690939806A0939906B0939A0639
:1071300080E090E0A0E0B0E0809371039093720350
:10714000A0937303B093740388E54DDB882351F457
:1071500089E549DB882331F48AE545DB882311F48E
:1071600081E001C080E080937503882309F4A2C107
:107170000F2EF0E08F2EF0E09F2EF0E0AF2EF0E02B
:10718000BF2EF02D8092340690923506A0923606DE
:10719000B09237068092380690923906A0923A064D
:1071A000B0923B0680923C0690923D06A0923E062D
:1071B000B0923F0684E396E068E376E04CE356E065
:1071C00020E436E00E94FF5A80E090E8ACEAB3EC9D
:1071D00080938B0690938C06A0938D06B0938E06B9
:1071E00080E090E8ACEAB3E480938F069093900639
:1071F000A0939106B0939206809393069093940681
:10720000A0939506B093960660913C0370913D0360
:1072100080913E0390913F036093710370937203DA
:10722000809373039093740320E030E040E752E4CE
:107230000E9428D67B018C018BE896E06FE876E00F
:1072400043E956E027E936E0FCE5CF2EF6E0DF2EF5
:107250000E945C600E94497F0E94D87DEDEFF7E0BC
:1072600065917591859194912091440630914506E0
:1072700040914606509147060E9448D560933406D7
:10728000709335068093360690933706E9E0F8E070
:1072900085919591A591B491809350069093510654
:1072A000A0935206B0935306E5E1F8E085919591DD
:1072B000A591B4918093500390935103A0935203EE
:1072C000B0935303E1E0F8E0659175918591949155
:1072D000209148063091490640914A0650914B064C
:1072E0000E9448D5609338067093390680933A0619
:1072F00090933B06EDE0F8E085919591A591B491CE
:107300008093540690935506A0935606B093570663
:10731000E9E1F8E085919591A591B49180935403AA
:1073200090935503A0935603B0935703E5E0F8E01C
:10733000659175918591949120914C0630914D06FF
:1073400040914E0650914F060E9448D560933C06EE
:1073500070933D0680933E0690933F06E1E1F8E08E
:1073600085919591A591B491809358069093590673
:10737000A0935A06B0935B06EDE1F8E085919591F4
:10738000A591B4918093580390935903A0935A0305
:10739000B0935B0384E396E068E376E04CE356E069
:1073A00020E436E00E94FF5A809134069091350621
:1073B000A0913606B091370680938B0690938C0689
:1073C000A0938D06B0938E06809138069091390671
:1073D000A0913A06B0913B0680938F069093900659
:1073E000A0939106B093920680913C0690913D0641
:1073F000A0913E06B0913F06809393069093940629
:10740000A0939506B09396066091710370917203F4
:10741000809173039091740320E030E040E752E4E0
:107420000E9428D67B018C018BE896E06FE876E01D
:1074300043E956E027E936E00E945C6080927103E0
:1074400090927203A0927303B09274030E94497FDA
:107450000E94D87D80918B0690918C06A0918D061C
:10746000B0918E068093340690933506A09336062D
:10747000B093370680918F0690919006A091910667
:10748000B09192068093380690933906A0933A06FD
:10749000B0933B068091930690919406A091950637
:1074A000B091960680933C0690933D06A0933E06CD
:1074B000B0933F0680917503882321F48AE593D920
:1074C000882319F082E090E01AD880917503882310
:1074D00051F488E588D9882309F46DC189E583D9F9
:1074E000882309F468C180E090E0A0E0B0E08093D8
:1074F000340690933506A0933606B09337068093F2
:10750000380690933906A0933A06B0933B0684E37D
:1075100096E068E376E04CE356E020E436E00E9433
:10752000FF5A80E090E8ACEAB3EC80938B0690932E
:107530008C06A0938D06B0938E0680E090E8ACEAAE
:10754000B3E480938F0690939006A0939106B09336
:10755000920620913C0330913D0340913E035091AF
:107560003F0320937103309372034093730350934E
:107570007403E0904003F0904103009142031091A6
:107580004303C801B7010E9421D6882344F4E09246
:107590007103F0927203009373031093740360916C
:1075A000710370917203809173039091740320E0D2
:1075B00030E040E752E40E9428D67B018C018BE842
:1075C00096E06FE876E043E956E027E936E0ECE53F
:1075D000CE2EE6E0DE2E0E945C600E94497FEDEF39
:1075E000F7E06591759185919491209144063091D1
:1075F000450640914606509147060E9448D5609343
:107600003406709335068093360690933706E9E08A
:10761000F8E085919591A591B4918093500690934F
:107620005106A0935206B0935306E5E1F8E0859128
:107630009591A591B4918093500390935103A09399
:107640005203B0935303E1E0F8E0659175918591A1
:107650009491209148063091490640914A065091F4
:107660004B060E9448D56093380670933906809384
:107670003A0690933B06EDE0F8E085919591A5914F
:10768000B4918093540690935506A0935606B093F8
:107690005706E9E1F8E085919591A591B491809321
:1076A000540390935503A0935603B093570384E378
:1076B00096E068E376E04CE356E020E436E00E9492
:1076C000FF5A8091340690913506A0913606B0910C
:1076D000370680938B0690938C06A0938D06B0930B
:1076E0008E068091380690913906A0913A06B091A5
:1076F0003B0680938F0690939006A0939106B093DB
:10770000920660917103709172038091730390915E
:10771000740320E030E040E752E40E9428D67B0169
:107720008C018BE896E06FE876E043E956E027E9C4
:1077300036E00E945C6080E090E0A0E0B0E08093E2
:10774000710390937203A0937303B09374030E9428
:10775000497F0E94D87D80918B0690918C06A091E4
:107760008D06B0918E068093340690933506A093D3
:107770003606B093370680918F0690919006A091BF
:107780009106B09192068093380690933906A093A3
:107790003A06B0933B068091930690919406A0918F
:1077A0009506B091960680933C0690933D06A09373
:1077B0003E06B0933F0680917503882321F488E547
:1077C00012D8882321F080E090E00E947F328091DF
:1077D0007503882321F489E506D8882321F081E008
:1077E00090E00E947F3288E50E94F3338823C9F03D
:1077F0003ED8611571058105910599F043D8209116
:1078000044063091450640914606509147060E9435
:1078100048D560933406709335068093360690936E
:10782000370689E50E94F3338823C9F020D8611513
:1078300071058105910599F025D820914806309170
:10784000490640914A0650914B060E9448D56093E4
:1078500038067093390680933A0690933B068AE582
:107860000E94F3338823C9F002D8611571058105A0
:10787000910599F007D820914C0630914D06409122
:107880004E0650914F060E9448D560933C06709377
:107890003D0680933E0690933F0684E396E068E3BE
:1078A00076E04CE356E020E436E00E94FF5A80E0A8
:1078B0000E94DF7D8091AA069091AB06A091AC0654
:1078C000B091AD068093710390937203A0937303FC
:1078D000B0937403809132069091330690934D03D8
:1078E00080934C030E94531A609377067093780636
:1078F0008093790690937A060E94D87D0C94054D6A
:1079000010929B060C94054D81E080939B060C948D
:10791000054D85E40E94F333882311F40E94497FCA
:1079200044E3E42E46E0F42E34E4C32E36E0D32EB6
:1079300000E010E0F801E652FC4F80810E94F33332
:10794000882331F1033061F40E944234F7016083EF
:1079500071838283938380E496E00E94D35A18C097
:107960000E944234F60120813181428153810E947C
:1079700048D5F701608371838283938384E396E023
:1079800068E376E04CE356E020E436E00E94FF5ADC
:107990000F5F1F4F24E030E0E20EF31EC20ED31E35
:1079A0000430110539F60C94054D8DE40E94F33333
:1079B000882311F40C94274C0E9442340E9490D6E4
:1079C0006937710511F40C9497466A3771050CF00C
:1079D0009CC06135710509F495C7623571050CF0DD
:1079E00048C06931710509F4D1C16A317105F4F4F7
:1079F0006531710509F493C16631710574F4623122
:107A0000710509F48CC76431710509F458C16131FD
:107A1000710511F00C94054D4CC16731710509F4E5
:107A20008AC1683171050CF0A1C17FC16E31710549
:107A300009F419C26F31710574F46B31710509F4E1
:107A4000D0C16B3171050CF4A7C16C31710511F017
:107A50000C94054DCCC16A32710509F434C360350C
:107A6000710509F44BC76F31710511F00C94054D88
:107A7000A9C26A36710509F4C4C66B367105F4F4FF
:107A80006535710509F49CC7663571054CF463359D
:107A9000710509F43FC7643571050CF040C736C75E
:107AA0006836710509F457C3693671050CF084C353
:107AB0006C35710511F00C94054D9DC76337710548
:107AC00011F40C948045643771057CF46D367105B2
:107AD00009F441C46237710511F40C949F456B366B
:107AE000710511F00C94054D05C76737710509F450
:107AF000DCC06837710514F00C9493466537710546
:107B000011F00C94054D0C948F4531E060337307F0
:107B100011F40C94B14941E0613374070CF057C083
:107B20006F3C710511F40C94FE47603D71051CF526
:107B30006B3C710511F40C9444476C3C71057CF46A
:107B40006E3B710509F49AC5693C710511F40C94FA
:107B500022476C38710511F00C94054D1CC36D3C27
:107B6000710511F40C9482476E3C710514F00C946D
:107B7000E0470C9462476D3D710511F40C94C348C5
:107B80006E3D71058CF4613D710511F40C944D4806
:107B9000613D710514F40C942D486C3D710511F094
:107BA0000C94054D0C94B44851E06E32750711F4F5
:107BB0000C945F4A81E06F32780714F00C946E4A9F
:107BC0006D52714011F00C94054D0C94D948E3E0CE
:107BD000603A7E0709F4BBC1F3E0613A7F077CF5A8
:107BE00021E0663F720711F40C94B74A31E0673F19
:107BF00073079CF441E0643F740711F40C94B14A9C
:107C000051E0653F750714F00C94B44A6059714017
:107C100011F00C94054D0C94AE4A93E06B38790743
:107C200011F40C94BD4AE3E06B397E0709F466C198
:107C3000675F714011F00C94054D0C94BA4A27E22D
:107C40006231720711F40C94294B37E263317307E8
:107C50009CF447E26031740711F40C94014B57E235
:107C60006131750714F00C94044B675E734011F09A
:107C70000C94054D0C94EC4A97E26431790711F4A9
:107C80000C947E4BE7E264317E0714F40C944E4B67
:107C9000F7E265317F0711F40C94AE4B6A517742DD
:107CA00011F00C94054D0C94DE4BEBE7F2E00C94D4
:107CB000A24615984698439840980C94054DEDEED1
:107CC000F7E0949108C08091C00085FFFCCF9093AD
:107CD000C600319694919923B1F78091C00085FF39
:107CE000FCCF8AE08093C60082E394E00E941F27C5
:107CF000EFEDF7E0949108C08091C00085FFFCCFC4
:107D00009093C600319694919923B1F78091C00069
:107D100085FFFCCF8AE08093C6000C94054D82E37A
:107D200094E00E94AB220C94054D82E394E00E9403
:107D30009A1C0C94054D8091AE069091AF06049666
:107D40006AE270E00E94C8D4FC01009711F03197FC
:107D500010826091AE067091AF066C5F7F4F82E338
:107D600094E041E00E94181F0C94054D82E394E0DA
:107D70000E949E1C0E94531A6093650670936606CB
:107D800080936706909368060C94054D82E394E017
:107D90000E94A51C0C94054D80916104882311F468
:107DA0000C94054D8091DB05882311F00C94054D52
:107DB00083E50E94F333882311F40C94054D0E944F
:107DC0003734AB01BC0140932406509325068093C1
:107DD00026067093270681E096E00E94BD6F0C9402
:107DE000054D82E394E00E949B1E0C94054D80910A
:107DF000AE069091AF0604966AE270E00E94C8D485
:107E00008C01009719F12091A0063091A10680E61F
:107E100090E0AC01249FC001259F900D349F900DF0
:107E200011248055994F6EE470E00E94C8D460E23E
:107E300070E00E94C8D49C012F5F3F4F3093AF0683
:107E40002093AE0601501040F80110826091AE06FA
:107E50007091AF066C5F7F4F82E394E040E00E9438
:107E6000181F0C94054D80916104882311F40C9423
:107E7000054D8091DB05882311F00C94054D82E3BC
:107E800094E00E940A1E8091AE069091AF0604967F
:107E90006AE270E00E94C8D48C01009719F1209129
:107EA000A0063091A10680E690E0AC01249FC001BD
:107EB000259F900D349F900D11248055994F6EE4AD
:107EC00070E00E94C8D460E270E00E94C8D49C01B7
:107ED0002F5F3F4F3093AF062093AE060150104006
:107EE000F80110826091AE067091AF066C5F7F4F13
:107EF00082E394E00E943A210C94054D8091AE06F5
:107F00009091AF0604966AE270E00E94C8D4FC012A
:107F1000009711F0319710826091AE067091AF0614
:107F20006C5F7F4F82E394E041E00E94181F82E380
:107F300094E00E949E1C0E94531A60936506709301
:107F4000660680936706909368060C94054D8091B1
:107F5000AE069091AF0605966AE270E00E94C8D422
:107F60008C01009719F12091A0063091A10680E6BE
:107F700090E0AC01249FC001259F900D349F900D8F
:107F800011248055994F6EE470E00E94C8D460E2DD
:107F900070E00E94C8D49C012F5F3F4F3093AF0622
:107FA0002093AE0601501040F80110826091AE0699
:107FB0007091AF066B5F7F4F82E394E00E943421A3
:107FC0000C94054D0E94531A6093690670936A06DB
:107FD00080936B0690936C0620916506309166063F
:107FE0004091670650916806621B730B840B950BDA
:107FF00028EE33E040E050E00E94EFDCF22EE32E6A
:10800000D42EC52E2DB73EB7285030400FB6F89469
:108010003EBF0FBE2DBF0DB71EB70F5F1F4FCE0166
:108020000196EDB7FEB79283818380ED97E0F8016A
:10803000938382836F2D7E2D842F952F2CE330E048
:1080400040E050E00E94EFDCF801358324836F2D7F
:108050007E2D8D2D9C2D2CE330E040E050E00E94E1
:10806000EFDCF801778366830E9417D5E4EEF5E034
:1080700094912DB73EB7285F3F4F0FB6F8943EBF9F
:108080000FBE2DBF08C08091C00085FFFCCF90932C
:10809000C600319694919923B1F7FE01319607C03D
:1080A0008091C00085FFFCCF31969093C6009081EF
:1080B0009923B1F78091C00085FFFCCF8AE08093BF
:1080C000C6000C94054D83E50E94F333882311F418
:1080D0000C94054D0E9442340E9490D67B018C0185
:1080E0006B0180E50E94F333882369F0F7FC0BC035
:1080F0003FEFE316F10409F034F40E9442340E9489
:1081000090D68B0102C008E010E0EEEDF3E0808134
:1081100091818017910711F40C94054D329644E03B
:10812000EE34F407A1F70730110519F4C0925D068B
:1081300004C017FF02C00C94054D802F61E00E941F
:10814000A11B802F6C2D0E94541C802FB6010E9411
:10815000C31A0C94054D88E690E00E944B348823A6
:1081600011F00C94054D83E50E94F333882379F0D8
:108170000E94423420916E06022F10E0000F111F62
:1081800008501E4E0E9490D6F801718360830E94B1
:1081900048870C94054D83E50E94F333882311F43E
:1081A0000C94054D0E9442340E9490D67093FB11AE
:1081B0006093FA110C94054D89E690E00E944B34CF
:1081C000882311F00C94054DEAECF7E0949108C077
:1081D0008091C00085FFFCCF9093C60031969491AA
:1081E0009923B1F7E0916E06F0E0EE0FFF1FEE0F5E
:1081F000FF1FE250FE4E408151816281738184E411
:108200009AE021E030E00E941957E7ECF7E0949102
:1082100008C08091C00085FFFCCF9093C6003196C6
:1082200094919923B1F7E0916E06F0E0EE0FFF1FF5
:10823000E850FE4E60817181882777FD8095982FE8
:108240000E94C3D6AB01BC0184E49AE021E030E097
:108250000E941957E3ECF7E0949108C08091C000A8
:1082600085FFFCCF9093C600319694919923B1F786
:1082700040910412509105126091061270910712FC
:1082800084E49AE021E030E00E941957E0ECF7E046
:10829000949108C08091C00085FFFCCF9093C600E8
:1082A000319694919923B1F76091FA117091FB1175
:1082B000882777FD8095982F0E94C3D6AB01BC011B
:1082C00084E49AE021E030E00E941957ECEBF7E0FB
:1082D000949108C08091C00085FFFCCF9093C600A8
:1082E000319694919923B1F780916E060E948D8604
:1082F000BC0184E49AE04AE050E00E944656E7EB75
:10830000F7E0949108C08091C00085FFFCCF909366
:10831000C600319694919923B1F78FEF9FEF0E9499
:108320008D86BC0184E49AE04AE050E00E94465603
:10833000E4E9F2E007C08091C00085FFFCCF3196F0
:108340009093C60090819923B1F78091C00085FF7A
:10835000FCCF0C94234C8DE690E00E944B34882394
:1083600011F00C94054D83E08093640683E50E9430
:10837000F333882379F00E94423420916E06022F55
:1083800010E0000F111F08501E4E0E9490D6F801F9
:10839000718360830E9448870E94531A4B015C01DD
:1083A00020916E06022F10E07724000F111FF801B4
:1083B000E850FE4E60817181882777FD8095982F67
:1083C0000E94C3D6000F111F02501E4EF8012081DB
:1083D0003181428153810E9424D8181614F47724E5
:1083E0007394CC24CA94DC2C7601E4EBF7E044903F
:1083F000E0EBF7E05490ECEAF7E064907AE0372E97
:1084000030C1942DE4EBF7E008C08091C00085FFF7
:10841000FCCF9093C600319694919923B1F7E091E7
:108420006E06F0E0EE0FFF1FEE0FFF1FE250FE4E54
:10843000408151816281738184E49AE021E030E0DF
:108440000E941957952DE0EBF7E008C08091C0001D
:1084500085FFFCCF9093C600319694919923B1F794
:1084600060916E0684E49AE070E04AE050E00E9479
:108470004656962DECEAF7E008C08091C00085FFD3
:10848000FCCF9093C600319694919923B1F7F7FEF3
:1084900003C0E5E9F2E028C00E94531AA701960143
:1084A0002854344F4F4F5F4F261B370B480B590B47
:1084B000CA01B90128EE33E040E050E00E94EFDC51
:1084C00084E49AE0BA01A9012AE030E00E94F7555D
:1084D0008091C00085FFFCCF0EC08091C00085FF59
:1084E000FCCF31969093C60090819923B1F780918B
:1084F000C00085FFFCCF3092C6000E94531A4B018A
:108500005C010E94798B0E947A300E94CB94FFEF2D
:10851000CF16FFEFDF06FFEFEF06FFEFFF0609F0D4
:1085200050C0E0916E06772031F1F0E08F01000F2E
:10853000111F000F111F02501E4EEE0FFF1FE850BB
:10854000FE4E60817181882777FD8095982F0E946B
:10855000C3D620E030E040E050E40E9447D59B01C4
:10856000AC01F80160817181828193810E9424D8DD
:1085700087FF5AC060C0F0E08F01000F111F000F8D
:10858000111F02501E4EEE0FFF1FE850FE4E60817D
:108590007181882777FD8095982F0E94C3D620E0AF
:1085A00030E040E050E40E9448D59B01AC01F80166
:1085B00060817181828193810E9421D61816A4F571
:1085C0003AC0F7FC38C0E0916E06F0E08F01000F72
:1085D000111F000F111F02501E4EEE0FFF1FE8501B
:1085E000FE4E60817181882777FD8095982F0E94CB
:1085F000C3D69B01AC01F8016081718182819381B6
:108600000E9447D50E9490D697FF07C0909580950D
:10861000709561957F4F8F4F9F4F64307105810535
:1086200091054CF0772039F40E94531AAC01CB012C
:10863000DA016C017D01FFEFCF16FFEFDF06FFEFE0
:10864000EF06FFEFFF0669F0F7FE02C00C94084D3D
:108650000E94531A6C197D09685B7B4010F00C94E2
:10866000084D0E94531A681979098A099B09695EA5
:1086700073408040904008F0C4CE43CF84E08093A4
:10868000640683E50E94F333882341F00E9442345C
:108690000E9490D67093FB116093FA110E94531AB6
:1086A0007B018C01E9EAF7E0B490E5EAF7E0C490D9
:1086B000E1EAF7E0D490BAE0AB2E7DC00E94531AF5
:1086C0006E197F09800B910B695E7340804090406A
:1086D00008F46BC0E0915C06F0E0EE0FFF1FEE0FB8
:1086E000FF1FE250FE4E40815181628173819B2DBC
:1086F000E9EAF7E008C08091C00085FFFCCF9093C5
:10870000C600319694919923B1F784E49AE022E06F
:1087100030E00E9419579C2DE5EAF7E008C08091EF
:10872000C00085FFFCCF9093C600319694919923A9
:10873000B1F760915C0684E49AE070E04AE050E0B2
:108740000E9446569D2DE1EAF7E008C08091C000E6
:1087500085FFFCCF9093C600319694919923B1F791
:108760004091041250910512609106127091071207
:1087700084E49AE021E030E00E941957E4E9F2E055
:1087800007C08091C00085FFFCCF31969093C60052
:1087900090819923B1F78091C00085FFFCCFA09212
:1087A000C6000E94531A7B018C010E94798B0E94A3
:1087B0007A300E94CB946091FA117091FB11625053
:1087C0007040882777FD8095982F0E94C3D69B0123
:1087D000AC01609104127091051280910612909183
:1087E00007120E9421D687FD69CF0E94531A609319
:1087F0007706709378068093790690937A060C94A6
:10880000054D83E50E94F333882309F465C00E9477
:1088100042347B018C0160915C0370E0882777FD16
:108820008095982F0E94C3D69B01AC01C801B70167
:108830000E94F6D820E030E048EC52E40E9428D6AE
:1088400020E030E040E050E00E9421D6882314F47C
:1088500060E03EC00E9442347B018C0160915C0369
:1088600070E0882777FD8095982F0E94C3D69B01E2
:10887000AC01C801B7010E94F6D820E030E048EC16
:1088800052E40E9428D620E030E04FE753E40E94F3
:1088900024D8181614F46FEF1BC00E9442347B01D9
:1088A0008C0160915C0370E0882777FD8095982F9C
:1088B0000E94C3D69B01AC01C801B7010E94F6D843
:1088C00020E030E048EC52E40E9428D60E9495D681
:1088D00060935D060C94054D80915C039FEF899F2A
:1088E000C001112464E670E00E94DCDC60935D0648
:1088F0000C94054D10925D060C94054D269A2E9809
:108900000C94054D269A2E9A0C94054D1092310622
:108910000C94054D81E0809331060C94054D83E560
:108920000E94F3338823A1F00E94423420E030E01B
:108930004AE754E40E94F6D80E9495D660936D03EE
:1089400070936E0380936F03909370030C94054DA6
:1089500088E50E94F333882311F00C941D4D89E5BE
:108960000E94F333882311F00C941D4D8AE50E9478
:10897000F333882311F00C941D4D85E40E94F333EA
:10898000882311F00C941D4D0E94497F409A0E944B
:10899000577F0C94054D159A89E50E94F333811198
:1089A000469A8AE50E94F3338111439A85E40E9436
:1089B000F333882311F40C94054D409A0C94054D23
:1089C00083E50E94F333882311F40C94054D0E9433
:1089D000423420E030E04AE754E40E94F6D80E9496
:1089E00095D660937B0670937C0680937D0690936A
:1089F0007E060C94054DE9E56E2EEAE07E2E79E4C4
:108A0000272E7AE0372E69E9462E6AE0562E882412
:108A10009924F401E652FC4F80810E94F3338823AD
:108A200009F45DC053E0851609F052C00E9442343B
:108A30005B016C0120E030E040EA51E40E9421D665
:108A400088230CF03FC0F3016081718182819381A2
:108A5000A60195010E9428D67B018C016091910AA4
:108A60007091920A8091930A9091940AA8019701BB
:108A70000E94F6D86093910A7093920A8093930AA9
:108A80009093940AF1016081718182819381A801A0
:108A900097010E94F6D8F1016083718382839383EA
:108AA000F20160817181828193810E94C1D6A80107
:108AB00097010E94F6D80E9495D6F20160837183D7
:108AC00082839383F301A082B182C282D38207C0E2
:108AD0000E944234F30160837183828393830894FC
:108AE000811C911C24E030E0620E731E220E331EA6
:108AF000420E531E34E08316910409F08ACF85C7D5
:108B0000E1E0F7E0949108C08091C00085FFFCCFC0
:108B10009093C600319694919923B1F776C78091CE
:108B2000AE069091AF0605966AE270E00E94C8D446
:108B3000FC01009709F469C73197108266C7EEEF10
:108B4000F6E0949108C08091C00085FFFCCF90931F
:108B5000C600319694919923B1F740913406509113
:108B60003506609136067091370684E49AE022E07B
:108B700030E00E941957EBEFF6E0949108C0809125
:108B8000C00085FFFCCF9093C60031969491992345
:108B9000B1F7409138065091390660913A067091CC
:108BA0003B0684E49AE022E030E00E941957E8EFA7
:108BB000F6E0949108C08091C00085FFFCCF9093AF
:108BC000C600319694919923B1F740913C0650919B
:108BD0003D0660913E0670913F0684E49AE022E0F3
:108BE00030E00E941957E5EFF6E0949108C08091BB
:108BF000C00085FFFCCF9093C600319694919923D5
:108C0000B1F7409140065091410660914206709143
:108C1000430684E49AE022E030E00E941957EAEE2D
:108C2000F6E0949108C08091C00085FFFCCF90933E
:108C3000C600319694919923B1F780E00E94337E6B
:108C40000E94C3D62091590A30915A0A40915B0A7A
:108C500050915C0A0E9428D6AB01BC0184E49AE0E2
:108C600022E030E00E941957E7EEF6E0949108C048
:108C70008091C00085FFFCCF9093C60031969491FF
:108C80009923B1F781E00E94337E0E94C3D62091E0
:108C90005D0A30915E0A40915F0A5091600A0E941D
:108CA00028D6AB01BC0184E49AE022E030E00E94C7
:108CB0001957E4EEF6E0949108C08091C00085FF5A
:108CC000FCCF9093C600319694919923B1F782E03E
:108CD0000E94337E0E94C3D62091610A3091620ABD
:108CE0004091630A5091640A0E9428D6AB01BC01EE
:108CF00084E49AE022E030E00E941957E4E9F2E0CF
:108D000007C08091C00085FFFCCF31969093C600CC
:108D100090819923B1F78091C00085FFFCCF8AE054
:108D20008093C60072C680E00E94DF7D6EC681E03F
:108D30000E94DF7D6AC68091C00085FFFCCF31961E
:108D40009093C60090819923B1F78091C00085FF70
:108D5000FCCF8AE08093C600ECEDF6E0949108C069
:108D60008091C00085FFFCCF9093C600319694910E
:108D70009923B1F7009B03C0E7E9F2E00AC0ECE9F0
:108D8000F2E007C08091C00085FFFCCF3196909340
:108D9000C60090819923B1F78091C00085FFFCCF78
:108DA0008AE08093C600E4EDF6E0949108C08091DB
:108DB000C00085FFFCCF9093C60031969491992313
:108DC000B1F7049B03C0E7E9F2E00AC0ECE9F2E086
:108DD00007C08091C00085FFFCCF31969093C600FC
:108DE00090819923B1F78091C00085FFFCCF8AE084
:108DF0008093C600ECECF6E0949108C08091C0002E
:108E000085FFFCCF9093C600319694919923B1F7DA
:108E1000079B03C0E7E9F2E00AC0ECE9F2E007C013
:108E20008091C00085FFFCCF31969093C600908161
:108E30009923B1F78091C00085FFFCCF8AE0809331
:108E4000C600E3C50AED13E05DE6E52E5AE0F52E17
:108E5000F80180810E94F333882349F00E94423454
:108E60000E9495D6F70160837183828393830F5F9D
:108E70001F4F24E030E0E20EF31E33E00E3D1307F7
:108E800039F70E94A85AC1C50AED13E049E4E42E5F
:108E90004AE0F42EF80180810E94F333882339F0F0
:108EA0000E944234F70160837183828393830F5F52
:108EB0001F4F24E030E0E20EF31E33E00E3D1307B7
:108EC00049F7A3C583E50E94F333882351F00E943C
:108ED00042346093810A7093820A8093830A90934C
:108EE000840A84E50E94F333882309F48EC50E9426
:108EF00042346093850A7093860A8093870A909320
:108F0000880A83C583E50E94F333882351F00E94C9
:108F1000423460937D0A70937E0A80937F0A909317
:108F2000800A84E50E94F333882351F00E94423482
:108F30006093950A7093960A8093970A9093980A83
:108F400082E40E94F333882361F00E9442340E943D
:108F500095D66093450A7093460A8093470A90938A
:108F6000480A88E50E94F333882351F00E94423476
:108F70006093890A70938A0A80938B0A90938C0A73
:108F80008AE50E94F333882351F00E9442346093B3
:108F90008D0A70938E0A80938F0A9093900A85E4CD
:108FA0000E94F333882309F430C50E944234609351
:108FB000910A7093920A8093930A9093940A25C51C
:108FC0000AED13E034E4E32E36E0F32EF80180815D
:108FD0000E94F333882339F00E944234F701608302
:108FE0007183828393830F5F1F4F24E030E0E20E92
:108FF000F31E33E00D3D130749F707C583E50E94D3
:10900000F333882351F00E94423460935D037093E0
:109010005E0380935F039093600386E40E94F333C2
:10902000882351F00E94423460936103709362037D
:1090300080936303909364038AE50E94F33388234B
:1090400009F4E3C40E94423460936503709366039D
:109050008093670390936803D8C483E50E94F33339
:10906000882351F00E944234609360067093610639
:10907000809362069093630686E40E94F33388230C
:1090800009F4C3C40E9442346093690370936A0375
:1090900080936B0390936C03B8C483E50E94F33311
:1090A000882309F4B2C40E9442340E9490D6672BF0
:1090B00021F06130710561F405C010925E061092D6
:1090C0005F06A3C481E080935E0610925F069DC494
:1090D000E4EEF5E0949108C08091C00085FFFCCFDC
:1090E0009093C600319694919923B1F7E9EBF6E09D
:1090F000949108C08091C00085FFFCCF9093C6007A
:10910000319694919923B1F72091A0063091A10650
:1091100080E690E0289FF001299FF00D389FF00D28
:109120001124E055F94F07C08091C00085FFFCCFA6
:1091300031969093C60090819923B1F7E7EBF6E062
:10914000949108C08091C00085FFFCCF9093C60029
:10915000319694919923B1F78091C00085FFFCCF9F
:109160008AE08093C60051C483E50E94F3338823CC
:1091700009F44BC40E9442340E9490D670934D0370
:1091800060934C0342C483E50E94F333882309F4BF
:109190003CC480915C06082F10E00E944234000F0E
:1091A000111F025B1C4F0E9490D6F80171836083EF
:1091B0002CC480E50E94F333882351F00E9442348E
:1091C000609385037093860380938703909388034D
:1091D00089E40E94F333882361F00E9442340E94A4
:1091E0006C876093890370938A0380938B039093B9
:1091F0008C0384E40E94F333882361F00E9442349C
:109200000E94788760938D0370938E0380938F0301
:109210009093900383E40E94F333882351F00E94DB
:1092200042346093910370939203809393039093DD
:1092300094030E946086E6EAF2E007C08091C000D5
:1092400085FFFCCF31969093C60090819923B1F7AA
:10925000E9EAF2E007C08091C00085FFFCCF3196BB
:109260009093C60090819923B1F740918503509166
:109270008603609187037091880384E49AE022E07A
:1092800030E00E941957EDEAF2E007C08091C0007B
:1092900085FFFCCF31969093C60090819923B1F75A
:1092A0006091890370918A0380918B0390918C0364
:1092B0000E947287AB01BC0184E49AE022E030E0B6
:1092C0000E941957E1EBF2E007C08091C00085FFD2
:1092D000FCCF31969093C60090819923B1F76091AD
:1092E0008D0370918E0380918F03909190030E9463
:1092F0007E87AB01BC0184E49AE022E030E00E946A
:109300001957E5EBF2E007C08091C00085FFFCCF64
:1093100031969093C60090819923B1F740919103C3
:1093200050919203609193037091940384E49AE0C6
:1093300022E030E00E941957E4E9F2E007C0809192
:10934000C00085FFFCCF31969093C6009081992391
:10935000B1F78091C00085FFFCCF8AE08093C60002
:1093600054C380E50E94F333882351F00E944234B5
:10937000609395037093960380939703909398035B
:1093800089E40E94F333882361F00E9442340E94F2
:109390006C876093990370939A0380939B039093D7
:1093A0009C0384E40E94F333882361F00E944234DA
:1093B0000E94788760939D0370939E0380939F0320
:1093C0009093A0030E946086E6EAF2E007C08091D5
:1093D000C00085FFFCCF31969093C6009081992301
:1093E000B1F7E9EAF2E007C08091C00085FFFCCF49
:1093F00031969093C60090819923B1F740919503DF
:1094000050919603609197037091980384E49AE0D9
:1094100022E030E00E941957EDEAF2E007C08091A7
:10942000C00085FFFCCF31969093C60090819923B0
:10943000B1F76091990370919A0380919B03909189
:109440009C030E947287AB01BC0184E49AE022E095
:1094500030E00E941957E1EBF2E007C08091C000B4
:1094600085FFFCCF31969093C60090819923B1F788
:1094700060919D0370919E0380919F039091A00342
:109480000E947E87AB01BC0184E49AE022E030E0D8
:109490000E941957E4E9F2E007C08091C00085FFFF
:1094A000FCCF31969093C60090819923B1F78091BB
:1094B000C00085FFFCCF8AE08093C600A6C283E58A
:1094C0000E94F333882329F460E070E080E090E0AC
:1094D00002C00E9442340E949F5A97C285E40E94B3
:1094E000F333882319F4CC24DD2412C00E944234C3
:1094F0000E9490D66B0177FF0BC00F2EF0E0EF2E8D
:10950000F0E0FF2EFCE80F2FF2E41F2FF02D0AC031
:109510000F2EF0E0EF2EF0E0FF2EF6E10F2FF3E438
:109520001F2FF02D83E50E94F333882321F00E9442
:1095300042347B018C0183E40E94F333882319F4C5
:1095400025E030E005C00E9442340E9490D69B0185
:10955000C801B701A6010E940D8E57C20E94497F23
:1095600054C20E94EF2D51C20E94EB2C4EC20E94A9
:1095700001284BC20E949F2948C288E50E94F3330C
:10958000882351F00E9442340E9490D69B01AC0186
:1095900080E0B9010E94687E8AE50E94F333882347
:1095A00051F00E9442340E9490D69B01AC0181E0B0
:1095B000B9010E94687E85E40E94F333882309F490
:1095C00024C20E9442340E9490D69B01AC0182E0EA
:1095D000B9010E94687E19C210926D0680917306CF
:1095E00090917406A0917506B091760680936F06EF
:1095F00090937006A0937106B09372060E94533246
:1096000004C20E944BA501C288E50E94F33388235F
:1096100011F400E003C00E943734062F89E50E9450
:10962000F333882311F410E003C00E943734162F5F
:1096300083E50E94F333882309F4E7C14091AE0625
:109640005091AF064F5F5F4F802F612F0E943D9B6F
:10965000DCC188E50E94F333882311F400E003C0E5
:109660000E943734062F89E50E94F333882311F4D2
:1096700010E003C00E943734162F83E50E94F333B5
:10968000882309F4C2C14091AE065091AF064F5FE6
:109690005F4F802F612F0E941F9CB7C188E50E94F9
:1096A000F333882311F4FF2403C00E943734F62ECD
:1096B00089E50E94F333882311F400E003C00E947F
:1096C0003734062F87E50E94F333882311F411E025
:1096D00003C00E943734162F88E40E94F333882396
:1096E00011F421E003C00E943734262F1F0D200FF4
:1096F0008F2D602F412F0E9472A087C188E50E94A4
:10970000F333882311F4FF2403C00E943734F62E6C
:1097100089E50E94F333882311F400E003C00E941E
:109720003734062F87E50E94F333882311F411E0C4
:1097300003C00E943734162F88E40E94F333882335
:1097400011F421E003C00E943734262F1F0D200F93
:109750008F2D602F412F0E94759F57C188E50E9471
:10976000F333882311F4FF2403C00E943734F62E0C
:1097700089E50E94F333882311F400E003C00E94BE
:109780003734062F87E50E94F333882311F411E064
:1097900003C00E943734162F88E40E94F3338823D5
:1097A00011F421E003C00E943734262F1F0D200F33
:1097B0008F2D602F412F0E94759F27C1E1EBF6E0AE
:1097C000949108C08091C00085FFFCCF9093C600A3
:1097D000319694919923B1F760918716709188160C
:1097E00084E49AE04AE050E00E94465610928816BF
:1097F0001092871680918A16882399F0ECEAF6E099
:10980000949108C08091C00085FFFCCF9093C60062
:10981000319694919923B1F78091C00085FFFCCFD8
:1098200012C0E7EAF6E0949108C08091C00085FF7D
:10983000FCCF9093C600319694919923B1F7809113
:10984000C00085FFFCCF8AE08093C60001C184E59B
:109850000E94F333882309F48DC00E9442340E9491
:1098600095D6262F60936E066623B9F1E4EEF5E0F7
:10987000949108C08091C00085FFFCCF9093C600F2
:10988000319694919923B1F7E9EBF2E007C080910A
:10989000C00085FFFCCF31969093C600908199233C
:1098A000B1F784E49AE0622F40E050E00E94025653
:1098B000EBEBF2E007C08091C00085FFFCCF319652
:1098C0009093C60090819923B1F78091C00085FFE5
:1098D000FCCF8AE08093C60098C086E40E94F333F0
:1098E0008823E1F00E9442347B018C0160939C0646
:1098F00070939D0680939E0690939F0620E030E033
:1099000040E050E00E9424D8181644F4E09271031D
:10991000F09272030093730310937403E4EEF5E086
:10992000949108C08091C00085FFFCCF9093C60041
:10993000319694919923B1F7ECECF2E007C0809155
:10994000C00085FFFCCF31969093C600908199238B
:10995000B1F760915C0684E49AE070E04AE050E080
:109960000E9446568091C00085FFFCCF8AE080931C
:10997000C6004BC0E4EEF5E0949108C08091C000B1
:1099800085FFFCCF9093C600319694919923B1F74F
:10999000E4E9F6E0949108C08091C00085FFFCCF17
:1099A0009093C600319694919923B1F72091A00627
:1099B0003091A10680E690E0289FF001299FF00DEC
:1099C000389FF00D1124E055F94F07C08091C00079
:1099D00085FFFCCF31969093C60090819923B1F713
:1099E000E2E9F6E0949108C08091C00085FFFCCFC9
:1099F0009093C600319694919923B1F78091C0005D
:109A000085FFFCCF8AE08093C6000E94513020C0C1
:109A10000E94531A609365067093660680936706EA
:109A2000909368060E94531A6093770670937806A5
:109A30008093790690937A06E8CF0E94497F88E563
:109A40000E94F333882311F00C94CB440C94CC4443
:109A50006E960FB6F894DEBF0FBECDBFCF91DF91EB
:109A60001F910F91FF90EF90DF90CF90BF90AF903C
:109A70009F908F907F906F905F904F903F902F902E
:109A800008952F923F924F925F926F927F928F92A2
:109A90009F92AF92BF92CF92DF92EF92FF920F937D
:109AA0001F93DF93CF93CDB7DEB76E970FB6F894C1
:109AB000DEBF0FBECDBF90E6A92EB12CE3E6F8E0E5
:109AC00084908AE0782EE9EDF8E09490662463941F
:109AD00040C22D3071F02A3321F48091B1098823DE
:109AE00041F08091B2099091B3098F3591050CF442
:109AF0000CC2E091B209F091B309309709F45DC34B
:109B0000A091B409B091B509AA9D7001AB9DF00C6C
:109B1000BA9DF00C1124EE0DFF1DE055F94F108297
:109B20008091B109882309F0EBC11092B109AE55BB
:109B3000B94F1C9287010055194FC8016EE470E0BF
:109B40000E94C8D49C01009709F4F5C09093AF0619
:109B50008093AE062F5F3F4F201B310B2E0D3F1D14
:109B6000C9018055994F60E070E04AE050E00E94E2
:109B7000CDD26093B6097093B7098093B8099093DA
:109B8000B909C0906F06D0907006E0907106F09011
:109B90007206A70196012F5F3F4F4F4F5F4F62172D
:109BA00073078407950709F4BAC38091B4099091AB
:109BB000B5099C012A9DC0012B9D900D3A9D900DE9
:109BC00011248055994F62E879E00E948DD4892B49
:109BD00009F0A5C3EAEEF5E0949108C08091C000B9
:109BE00085FFFCCF9093C600319694919923B1F7ED
:109BF000EFE4F9E0949108C08091C00085FFFCCFAC
:109C00009093C600319694919923B1F784E49AE039
:109C1000B701A6012AE030E00E9413568091C000EF
:109C200085FFFCCF71C0FE264F5FFC01E40FF11DE4
:109C3000E055F94FE081EA32B1F73093AF06209357
:109C4000AE06C901019660E070E00E9467D10E94F3
:109C500090D62F2D30E02617370709F45BC0EAEEC7
:109C6000F5E0949108C08091C00085FFFCCF9093EF
:109C7000C600319694919923B1F7E0E3F9E094910D
:109C800008C08091C00085FFFCCF9093C60031963C
:109C900094919923B1F740916F06509170066091AD
:109CA00071067091720684E49AE02AE030E0BBD736
:109CB0008091C00085FFFCCF27C0EAEEF5E09491CB
:109CC00008C08091C00085FFFCCF9093C6003196FC
:109CD00094919923B1F7E6E0F9E0949108C080915E
:109CE000C00085FFFCCF9093C600319694919923D4
:109CF000B1F784E49AE0B701A6012AE030E093D7F7
:109D00008091C00085FFFCCF8AE08093C6000E944E
:109D1000533249C08091B6099091B709A091B80912
:109D2000B091B90980936F0690937006A093710665
:109D3000B09372063DC0C8016AE270E00E94C8D4C8
:109D4000009709F435C0EAEEF5E0949108C08091DF
:109D5000C00085FFFCCF9093C60031969491992363
:109D6000B1F7ECEDF8E0949108C08091C00085FF58
:109D7000FCCF9093C600319694919923B1F740910E
:109D80006F0650917006609171067091720684E4BE
:109D90009AE02AE030E047D78091C00085FFFCCFF1
:109DA0008AE08093C6001092B3091092B209D6C21D
:109DB0008091B4099091B5098A9D70018B9DF00C3A
:109DC0009A9DF00C112487010055194FC80167E4D2
:109DD00070E00E94C8D49C01009709F445C090939C
:109DE000AF068093AE062F5F3F4F201B310B2E0D29
:109DF0003F1DC9018055994F60E070E00E9467D116
:109E00000E9490D66430710578F580916D068823A4
:109E1000B9F480913204882339F5992DE9EDF8E001
:109E200008C08091C00085FFFCCF9093C60031969A
:109E300094919923B1F78091C00085FFFCCF12C0A7
:109E4000982DE3E6F8E008C08091C00085FFFCCFC4
:109E50009093C600319694919923B1F78091C000F8
:109E600085FFFCCF7092C6008091B4099091B5092E
:109E70008A9D70018B9DF00C9A9DF00C1124870136
:109E80000055194FC8016DE470E00E94C8D49C01D0
:109E90009093AF068093AE062F5F3F4F201B310B90
:109EA0002E0D3F1DC9018055994F60E070E04AE0DA
:109EB00050E00E94CDD2693671058105910551F0BF
:109EC0000E94531A60936312709364128093651218
:109ED000909366128091B4099091B509019668E05B
:109EE00070E00E94DCDC9093B5098093B409809106
:109EF000BA099091BB0901969093BB098093BA0966
:109F00001092B3091092B20924C02B3311F460925D
:109F1000B1098091B1098823E1F42091B20930910F
:109F2000B3098091B4099091B5098A9DF0018B9D88
:109F3000F00D9A9DF00D1124E20FF31FE055F94F3B
:109F40008091B00980832F5F3F4F3093B3092093F6
:109F5000B2098091400A9091410A2091420A3091C1
:109F6000430A821B930B8F779070892B09F4F1C100
:109F70008091BA099091BB0908970CF0EAC184E47A
:109F80009AE077D5282F8093B0098A3009F0A1CDC7
:109F9000B0CD8091B2099091B309892B09F473C1B6
:109FA000DDC180913504882329F482E394E00E9486
:109FB0009A1CF9CE1092DB051092B3091092B209E7
:109FC0004091BC095091BD096091BE097091BF09D3
:109FD00080911C0690911D06A0911E06B0911F064F
:109FE00080509240A040B04084179507A607B7075D
:109FF00018F410923404B2C14093240650932506FD
:10A00000609326067093270681E096E00E94BD6F5C
:10A01000A5C1262F6093B0096A30A1F06D3091F090
:10A020006A3321F48091B109882361F08091B209EB
:10A030009091B3098F3591052CF43FEF6F3F730773
:10A0400009F0FCC020912406309125064091260697
:10A050005091270680911C0690911D06A0911E0626
:10A06000B0911F06281739074A075B0720F46F5F76
:10A070007F4F09F09BC0962DE0E5F8E008C0809185
:10A08000C00085FFFCCF9093C60031969491992330
:10A09000B1F78091C00085FFFCCF3092C6000E94CE
:10A0A000531A6093690670936A0680936B069093C7
:10A0B0006C062091650630916606409167065091C6
:10A0C0006806621B730B840B950B28EE33E040E0AF
:10A0D00050E00E94EFDCF22EE32ED42EC52EEDB719
:10A0E000FEB738970FB6F894FEBF0FBEEDBF0DB7A1
:10A0F0001EB70F5F1F4FB282A182F80153824282C6
:10A10000622F732F842F952F20E13EE040E050E036
:10A110000E94EFDCF801358324836F2D7E2D8D2D79
:10A120009C2D2CE330E040E050E00E94EFDCCA01BF
:10A13000B9012CE330E040E050E00E94EFDCF80190
:10A14000778366830E9417D5972DE4EEF5E02DB74F
:10A150003EB7285F3F4F0FB6F8943EBF0FBE2DBFEE
:10A1600008C08091C00085FFFCCF9093C600319657
:10A1700094919923B1F7F50107C08091C00085FF44
:10A18000FCCF31969093C60090819923B1F78091CE
:10A19000C00085FFFCCF3092C60082E394E00E94AD
:10A1A000251D82E394E061E00E948B232091B20997
:10A1B0003091B3092115310519F41092B109CEC0BF
:10A1C0008091B4099091B509889DF001899DF00DA9
:10A1D000989DF00D1124E20FF31FE055F94F108206
:10A1E000FC01EE55F94F20822091BA093091BB094C
:10A1F0002F5F3F4F3093BB092093BA09019668E067
:10A2000070E00E94DCDC9093B5098093B409109251
:10A21000B1091092B3091092B2098091240690916D
:10A220002506A0912606B09127068093BC0990933D
:10A23000BD09A093BE09B093BF093AC02B3311F4F6
:10A240002092B1098091B109882391F52091B2093A
:10A250003091B3098091B4099091B509889DF001BE
:10A26000899DF00D989DF00D1124E20FF31FE0552C
:10A27000F94F8091B00980832F5F3F4F3093B3092E
:10A280002093B20915C000E6802E912C222423943D
:10A29000E0E5F8E064901AE0312E5E010894A11C1C
:10A2A000B11CBCE34B2EB8E05B2EE4EEF5E07490FD
:10A2B00020912406309125064091260650912706CC
:10A2C00080911C0690911D06A0911E06B0911F065C
:10A2D000281739074A075B0708F040C08091BA0980
:10A2E0009091BB090897D4F58091090690910A06D0
:10A2F000A0910B06B0910C0680932406909325063E
:10A30000A0932606B093270681E096E00E945B7337
:10A31000BC018091DB05882309F47BCE42CE80917D
:10A32000B4099091B5098A9D80018B9D100D9A9D6D
:10A33000100D1124C8018055994F6AE270E00E9407
:10A34000C8D49C01009709F4B8CCFF2440E0C801B0
:10A350006CCC80913404882309F01BCE6E960FB626
:10A36000F894DEBF0FBECDBFCF91DF911F910F914B
:10A37000FF90EF90DF90CF90BF90AF909F908F9025
:10A380007F906F905F904F903F902F900895CF9364
:10A39000DF938091BA099091BB0907970CF471DBA8
:10A3A00082E394E060E00E948B238091BA0990914F
:10A3B000BB09892B09F46CC080913204882309F40D
:10A3C0004CC02091A0063091A10680E690E0289F25
:10A3D000E001299FD00D389FD00D1124C055D94FD1
:10A3E000CE016CE979E00E948DD4892BE1F482E3FF
:10A3F00094E0BE010E94231E80913304882369F5F6
:10A40000E9E9F9E0949108C08091C00085FFFCCF94
:10A410009093C600319694919923B1F78091C00032
:10A4200085FFFCCF16C082E394E00E940A1EE7E895
:10A43000F9E0949108C08091C00085FFFCCF909313
:10A44000C600319694919923B1F78091C00085FFA1
:10A45000FCCF8AE08093C60002C00E9467368091DC
:10A46000BA099091BB091816190694F401979093B4
:10A47000BB098093BA098091A0069091A10601962C
:10A4800068E070E00E94DCDC9093A1068093A00657
:10A490000E94798B0E947A300E94C2850E94CB94E0
:10A4A000DF91CF910895269A2E9884E49AE040E9AE
:10A4B00050ED63E070E0A9D2E5E7FAE0949108C0BE
:10A4C0008091C00085FFFCCF9093C6003196949197
:10A4D0009923B1F78091C00085FFFCCF8AE080937B
:10A4E000C60044EE55E0FA01949108C08091C00086
:10A4F00085FFFCCF9093C600319694919923B1F7D4
:10A5000084B7282F80FF15C0EDE6FAE0949108C0CB
:10A510008091C00085FFFCCF9093C6003196949146
:10A520009923B1F78091C00085FFFCCF8AE080932A
:10A53000C60021FF15C0EDE5FAE0949108C08091B6
:10A54000C00085FFFCCF9093C6003196949199236B
:10A55000B1F78091C00085FFFCCF8AE08093C600F0
:10A5600022FF15C0ECE4FAE0949108C08091C0008D
:10A5700085FFFCCF9093C600319694919923B1F753
:10A580008091C00085FFFCCF8AE08093C60023FF46
:10A5900015C0ECE3FAE0949108C08091C00085FFFB
:10A5A000FCCF9093C600319694919923B1F7809196
:10A5B000C00085FFFCCF8AE08093C60025FF15C050
:10A5C000ECE2FAE0949108C08091C00085FFFCCFD6
:10A5D0009093C600319694919923B1F78091C00071
:10A5E00085FFFCCF8AE08093C60014BEE4E2FAE067
:10A5F000949108C08091C00085FFFCCF9093C60065
:10A60000319694919923B1F7EEE1FAE0949108C064
:10A610008091C00085FFFCCF9093C6003196949145
:10A620009923B1F78091C00085FFFCCF8AE0809329
:10A63000C600FA019491E4EEF5E008C08091C000F4
:10A6400085FFFCCF9093C600319694919923B1F782
:10A65000EEE0FAE0949108C08091C00085FFFCCF45
:10A660009093C600319694919923B1F7E9EFF9E000
:10A67000949108C08091C00085FFFCCF9093C600E4
:10A68000319694919923B1F7EDEEF9E0949108C0D9
:10A690008091C00085FFFCCF9093C60031969491C5
:10A6A0009923B1F7EDEDF9E0949108C08091C000D5
:10A6B00085FFFCCF9093C600319694919923B1F712
:10A6C0008091C00085FFFCCF8AE08093C600E2ED58
:10A6D000F9E0949108C08091C00085FFFCCF909371
:10A6E000C600319694919923B1F7E6ECF9E0949184
:10A6F00008C08091C00085FFFCCF9093C6003196C2
:10A7000094919923B1F78091C00085FFFCCF8AE036
:10A710008093C600FA019491E4EEF5E008C08091C0
:10A72000C00085FFFCCF9093C60031969491992389
:10A73000B1F7E7EBF9E0949108C08091C00085FF84
:10A74000FCCF9093C600319694919923B1F70E9463
:10A75000EB2EBC0184E49AE04AE050E097D2E0EAB4
:10A76000F9E0949108C08091C00085FFFCCF9093E0
:10A77000C600319694919923B1F784E49AE060ED94
:10A7800074E04AE050E082D28091C00085FFFCCFA7
:10A790008AE08093C600E2EAF6E0119286E0EA3AA7
:10A7A000F807D9F70E94EB2C0E948D8A0E94935DD6
:10A7B0000E9459D10E94D27E0C947695BC01809162
:10A7C000BA099091BB0908970CF070C02091B409A8
:10A7D0003091B50980E690E0AC01249FC001259F2F
:10A7E000900D349F900D11248055994F0E9448D4AC
:10A7F000E4EEF5E0949108C08091C00085FFFCCFA5
:10A800009093C600319694919923B1F7EDE7FAE061
:10A81000949108C08091C00085FFFCCF9093C60042
:10A82000319694919923B1F72091B4093091B509EB
:10A8300080E690E0289FF001299FF00D389FF00DF1
:10A840001124E055F94F07C08091C00085FFFCCF6F
:10A8500031969093C60090819923B1F7EBE7FAE027
:10A86000949108C08091C00085FFFCCF9093C600F2
:10A87000319694919923B1F78091C00085FFFCCF68
:10A880008AE08093C600C901019668E070E00E94EA
:10A89000DCDC9093B5098093B4098091BA0990915A
:10A8A000BB0901969093BB098093BA090895BC0136
:10A8B0008091BA099091BB0908970CF070C0209163
:10A8C000B4093091B50980E690E0AC01249FC00145
:10A8D000259F900D349F900D11248055994F0E9413
:10A8E000D3D4E4EEF5E0949108C08091C00085FFD8
:10A8F000FCCF9093C600319694919923B1F7EAE882
:10A90000FAE0949108C08091C00085FFFCCF90933D
:10A91000C600319694919923B1F72091B4093091F2
:10A92000B50980E690E0289FF001299FF00D389F3F
:10A93000F00D1124E055F94F07C08091C00085FF4C
:10A94000FCCF31969093C60090819923B1F7E8E847
:10A95000FAE0949108C08091C00085FFFCCF9093ED
:10A96000C600319694919923B1F78091C00085FF7C
:10A97000FCCF8AE08093C600C901019668E070E0D0
:10A980000E94DCDC9093B5098093B4098091BA09E8
:10A990009091BB0901969093BB098093BA090895E1
:10A9A0001F920F920FB60F920BB60F9211242F9396
:10A9B0003F934F938F939F93EF93FF934091C600E4
:10A9C000E091400AF091410A31969F012F77307053
:10A9D00031978091420A9091430A2817390739F03C
:10A9E000E054F64F40833093410A2093400AFF9190
:10A9F000EF919F918F914F913F912F910F900BBEAF
:10AA00000F900FBE0F901F9018959A01AB01203048
:10AA100081EE380780E0480780E0580729F182E09E
:10AA20008093C00060E079E08DE390E00E94EFDC6D
:10AA300021503040404050405695479537952795D6
:10AA40003093C5002093C4008091C1008061809341
:10AA5000C1008091C10088608093C1008091C100D5
:10AA600080688093C10008951092C00020E130E01A
:10AA7000E7CF2091420A3091430A8091400A909199
:10AA8000410A8217930719F42FEF3FEF0EC0F90127
:10AA9000E054F64F80812F5F3F4F2F773070309317
:10AAA000430A2093420A282F30E0C901089580917B
:10AAB000420A9091430A9093410A8093400A089574
:10AAC00008952F923F924F925F926F927F928F9252
:10AAD0009F92AF92BF92CF92DF92EF92FF920F932D
:10AAE0001F93DF93CF93CDB7DEB7A0970FB6F8943F
:10AAF000DEBF0FBECDBF1C016A017B0141155105B0
:10AB00006105710541F440E350E060E070E020E051
:10AB100030E089D053C0882499245401422E552412
:10AB20006624772401E010E00C0F1D1F080D191D8D
:10AB3000C701B601A30192010E94EFDCF801608316
:10AB40000894811C911CA11CB11CC701B601A30172
:10AB500092010E94EFDCC901DA016C017D01C11490
:10AB6000D104E104F104F1F691E0E92EF12CEC0EB0
:10AB7000FD1EE80CF91C3E010894611C711CD501F6
:10AB8000C4010197A109B1096C01C818D90813C003
:10AB9000F601EE0DFF1D40814A3010F4405D01C00A
:10ABA000495C50E060E070E0C10120E030E03BD063
:10ABB0000894E108F1086E147F0451F7A0960FB6CF
:10ABC000F894DEBF0FBECDBFCF91DF911F910F91E3
:10ABD000FF90EF90DF90CF90BF90AF909F908F90BD
:10ABE0007F906F905F904F903F902F900895211528
:10ABF000310539F48091C00085FFFCCF4093C60039
:10AC000008955FCFEF92FF920F931F939A01E62E64
:10AC1000FF2400E010E0B801A701E9DF1F910F91C8
:10AC2000FF90EF900895EF92FF920F931F93CF93B1
:10AC3000DF93EC017A018B012115310539F4809104
:10AC4000C00085FFFCCFE092C60019C02A30310554
:10AC5000A9F477FF0FC04DE250E060E070E020E023
:10AC600030E0E1DF10950095F094E094E11CF11CD8
:10AC7000011D111DCE01B801A7012AE022DFDF91DD
:10AC8000CF911F910F91FF90EF900895EF92FF9257
:10AC90000F931F937B019A010027F7FC0095102F5B
:10ACA000B801A701C0DF1F910F91FF90EF900895A9
:10ACB0000F931F938C014DE050E060E070E020E0C6
:10ACC00030E0B1DFC8014AE050E060E070E020E031
:10ACD00030E0A9DF1F910F910895CF92DF92EF929C
:10ACE000FF920F931F938C019A016B01EE24FF24B6
:10ACF000B701A6017CDFC801DBDF1F910F91FF9038
:10AD0000EF90DF90CF9008959F92AF92BF92CF9235
:10AD1000DF92EF92FF920F931F93CF93DF93EC019B
:10AD20007A018B01922ECB01BA0120E030E040E0A5
:10AD300050E00E9421D6882364F4CE014DE250E019
:10AD400060E070E020E030E06EDF17FB109517F94F
:10AD5000109520E030E040E05FE3AA240BC0CA0178
:10AD6000B90120E030E040E251E40E9428D69B0186
:10AD7000AC01A394A91498F3C801B7010E9448D567
:10AD80007B018C010E9495D65B016C010E94C1D6AB
:10AD90009B01AC01C801B7010E9447D57B018C0122
:10ADA000CE01B601A5012AE030E021DF992099F11A
:10ADB000EEEDF2E007C08091C00085FFFCCF319638
:10ADC0009093C60090819923B1F725C0C801B701BF
:10ADD00020E030E040E251E40E94F6D87B018C0193
:10ADE0000E9490D65B016C01CC24B7FCC094DC2C93
:10ADF000CE01B601A5012AE030E015DFC601B5019C
:10AE00000E94C3D69B01AC01C801B7010E9447D57F
:10AE10007B018C019A949920C9F6DF91CF911F9103
:10AE20000F91FF90EF90DF90CF90BF90AF909F90E9
:10AE300008956ACF08952F923F924F925F926F923A
:10AE40007F928F929F92AF92BF92CF92DF92EF92BA
:10AE5000FF920F931F93DF93CF93CDB7DEB7CD55FE
:10AE6000D0400FB6F894DEBF0FBECDBF2F969FAF78
:10AE70008EAF2F9761967FAF6EAF61972A01629672
:10AE80002FAF629763960FAF63976496EFAE6497A8
:10AE90006896ACAEBDAECEAEDFAE6897E22EFF24B4
:10AEA000EE0CFF1CEE0CFF1C9A012E0D3F1D2D9683
:10AEB0003FAF2EAF2D97D9016D907D908D909C90D6
:10AEC000FC01EE0DFF1DC401B301208131814281DF
:10AED00053810E9448D569AF7AAF8BAF9CAF10E029
:10AEE000000F111F000F111FF201E00FF11F2B9631
:10AEF000FFAFEEAF2B97A080B180C280D3802F969A
:10AF0000EEADFFAD2F97E00FF11FC601B501208117
:10AF10003181428153810E9448D56DAB7EAB8FABAE
:10AF200098AF64962FAD6497E22FF0E0EE0FFF1F0D
:10AF3000EE0FFF1F2F96AEADBFAD2F97AE0FBF1F09
:10AF40004D915D916D917C9129964CAF5DAF6EAF47
:10AF50007FAF299761966EAD7FAD6197E60FF71FC2
:10AF6000608171818281938129962CAD3DAD4EAD7A
:10AF70005FAD29970E9447D569AB7AAB8BAB9CAB91
:10AF80006196AEADBFAD61971C968D919D910D9070
:10AF9000BC91A02D25968CAF9DAFAEAFBFAF2597CE
:10AFA0002F96AEADBFAD2F971C962D913D914D9133
:10AFB0005C911F9721962CAF3DAF4EAF5FAF2197AD
:10AFC000A401930150582DA73EA74FA758ABB60137
:10AFD000A501705849A75AA76BA77CA761966EADCB
:10AFE0007FAD6197E60EF71ED7016D917D918D9132
:10AFF0009C9129AD3AAD4BAD5CAD0E9447D53B016C
:10B000004C016196EEADFFAD61970E0F1F1FD80189
:10B010006D917D918D919C912DA93EA94FA958AD1F
:10B020000E9447D55B016C016DA57EA58FA598A9EF
:10B03000A60195010E94F6D87B018C0169A57AA52D
:10B040008BA59CA5A40193010E94F6D89B01AC019D
:10B05000C801B7010E9447D51B012C016DA57EA533
:10B060008FA598A9A40193010E94F6D87B018C01B9
:10B0700069A57AA58BA59CA5A60195010E94F6D885
:10B080009B01AC01C801B7010E9448D59B01AC01EE
:10B09000C201B1010E94BBD55B016C0120E030E030
:10B0A00040E050E00E9421D6882354F4C601B50147
:10B0B0002BED3FE049EC50E40E9448D55B016C0168
:10B0C000E8968FADE897882351F0C601B5012BEDC6
:10B0D0003FE049EC50E40E9447D55B016C01C6019A
:10B0E000B501E7962CAD3DAD4EAD5FADE7970E9443
:10B0F000F6D829A93AA94BA95CA95F770E9431D853
:10B100007B018C012FE632E143E85AE30E9421D60D
:10B1100087FDF4C1C801B7010E94FED60E9495D6F2
:10B1200078A76FA3672B21F4E1E0F0E0F8A7EFA385
:10B130002FA138A5B90180E090E00E94C1D67B0123
:10B140008C01C601B501A80197010E9428D66BA306
:10B150007CA38DA39EA369A97AA98BA99CA9A80108
:10B1600097010E9428D66F8F78A389A39AA325966A
:10B170006CAD7DAD8EAD9FAD259721962CAD3DADCF
:10B180004EAD5FAD21970E9447D5A80197010E945F
:10B1900028D66B8F7C8F8D8F9E8F6BA17CA18DA10C
:10B1A0009EA120E030E040E05FEB0E94F6D82BA1AA
:10B1B0003CA14DA15EA10E94F6D820E030E040E81D
:10B1C0005FE30E9448D56F8B788F898F9A8F649642
:10B1D0003FAD6497E32FF0E0EE0FFF1FEE0FFF1F70
:10B1E0009E012F5F3F4FE20FF31F29964CAD5DADDF
:10B1F0006EAD7FAD299740835183628373832F9611
:10B20000AEADBFAD2F971C964D915D916D917C9128
:10B210001F974D875E876F87788B41E050E05A8B90
:10B22000498B662462967FAD6297672F70E0660F48
:10B23000771F660F771FC901860F971F6A969FAF0A
:10B240008EAF6A976396BFAD6397AB2FB0E0AA0F3E
:10B25000BB1FAA0FBB1F21E030E02C0F3D1F2A0FA0
:10B260003B1F6C963FAF2EAF6C976E96FFAFEEAF65
:10B270006E9719C138E136150CF446C06DA57EA550
:10B280008FA598A92BA13CA14DA15EA10E94F6D843
:10B290007B018C0169A57AA58BA59CA52F89388D8A
:10B2A000498D5A8D0E94F6D89B01AC01C801B701A7
:10B2B0000E9448D57B018C016DA57EA58FA598A91C
:10B2C0002F89388D498D5A8D0E94F6D85B016C010B
:10B2D00069A57AA58BA59CA52BA13CA14DA15EA13A
:10B2E0000E94F6D89B01AC01C601B5010E9447D56A
:10B2F0006DA77EA78FA798AB6394C701D80189A7D4
:10B300009AA7ABA7BCA765C049895A89BA0180E052
:10B3100090E00E94C1D62BA13CA14DA15EA10E944C
:10B32000F6D87B018C01C8010E9425D66B8B7C8BE3
:10B330008D8B9E8BB701C8010E9459D93B014C01EE
:10B340002D96AEADBFAD2D97ED90FD900D911C915A
:10B3500017FB109517F910952B96EEADFFAD2B97B7
:10B360002080318042805380C801B7012B893C89FD
:10B370004D895E890E94F6D85B016C01C201B10162
:10B38000A40193010E94F6D89B01AC01C601B5014E
:10B390000E9448D56DA77EA78FA798ABC801B701BB
:10B3A000A40193010E94F6D87B018C01C201B10176
:10B3B0002B893C894D895E890E94F6D89B01AC019E
:10B3C000C801B7010E9447D569A77AA78BA79CA798
:10B3D000662469AD7AAD8BAD9CAD2DA53EA54FA57C
:10B3E00058A90E9448D56A96AEADBFAD6A976D93D5
:10B3F0007D938D939C9313976DA97EA98FA998AD8A
:10B4000029A53AA54BA55CA50E9448D56C96EEAD42
:10B41000FFAD6C9760837183828393836E96AEAD2C
:10B42000BFAD6E976D917D918D919C912F8D38A1BF
:10B4300049A15AA10E9448D56E96EEADFFAD6E9718
:10B4400060837183828393836D857E858F859889E0
:10B450002B8D3C8D4D8D5E8D0E9448D56D877E87EE
:10B460008F87988BCE0101960E94142FCE010196F2
:10B47000BE016B5F7F4FAE01475F5F4F9E01235F51
:10B480003F4F6896ECACFDAC0EAD1FAD6897F8E78A
:10B49000CF2ED12CCC0EDD1E0FD629893A892F5FF5
:10B4A0003F4F3A8B298B49895A896FA178A5461756
:10B4B000570708F4DFCE61964EAD5FAD6197485FE8
:10B4C0005F4F61962EAD3FAD6197245F3F4F619610
:10B4D0008EAD9FAD6197DC0114966196BFAFAEAFA4
:10B4E0006197BD016896ECACFDAC0EAD1FAD6897E1
:10B4F000E8E7CE2ED12CCC0EDD1EDED5C35ADF4FB1
:10B500000FB6F894DEBF0FBECDBFCF91DF911F9174
:10B510000F91FF90EF90DF90CF90BF90AF909F90F2
:10B520008F907F906F905F904F903F902F900895F5
:10B530008091890F90918A0F891B8F700895609375
:10B54000760370937703809378039093790308953B
:10B550000F931F93CF93DF93C0E0D0E08E01075687
:10B56000154FFE01E359F54F60817181828193810E
:10B570000E94C1D6FE01E75AF54F208131814281F8
:10B5800053810E94F6D80E9495D6F801608371839A
:10B59000828393832496C031D10501F7DF91CF9147
:10B5A0001F910F910895FC016081718182819381C7
:10B5B0002091650A3091660A4091670A5091680AA5
:10B5C0000E94F6D8E0915C06F0E0EE0FFF1FEE0F50
:10B5D000FF1FE759F54F20813181428153810E943D
:10B5E000F6D80E94C6D86093B50A7093B60A8093C5
:10B5F000B70A9093B80A85EB9AE00C94227E8F925A
:10B600009F92AF92BF92CF92DF92EF92FF920F93F1
:10B610001F93FC018B015A01490160817181828174
:10B6200093812091590A30915A0A40915B0A5091B6
:10B630005C0A0E94F6D80E94C6D859EAC52E5AE084
:10B64000D52E6093A90A7093AA0A8093AB0A9093AF
:10B65000AC0AF801608171818281938120915D0A39
:10B6600030915E0A40915F0A5091600A0E94F6D8BC
:10B670000E94C6D844E0E42EF12CEC0CFD1C609333
:10B68000AD0AF701718382839383F5016081718133
:10B69000828193812091610A3091620A4091630A0C
:10B6A0005091640A0E94F6D80E94C6D88601085FAD
:10B6B0001F4F6093B10AF801718382839383F40171
:10B6C00060817181828193812091650A3091660A3F
:10B6D0004091670A5091680A0E94F6D8E0915C0692
:10B6E000F0E0EE0FFF1FEE0FFF1FE759F54F20812F
:10B6F0003181428153810E94F6D80E94C6D8F6015A
:10B700003C966093B50A718382839383C601B70127
:10B71000A8019F010E94E87D80E090E0A0E0B0E0F9
:10B7200080938B0F90938C0FA0938D0FB0938E0FFF
:10B7300080938F0F9093900FA093910FB093920FDF
:10B740008093930F9093940FA093950FB093960FBF
:10B750008093970F9093980FA093990FB0939A0F9F
:10B7600080939B0F90939C0FA0939D0FB0939E0F7F
:10B770001F910F91FF90EF90DF90CF90BF90AF900F
:10B780009F908F9008958F929F92AF92BF92CF9289
:10B79000DF92EF92FF920F931F93CF93DF93EC0111
:10B7A0006B01009709F45CC08FA9882309F058C089
:10B7B000EEA0FFA008A519A5FB01B6A0A7A090A424
:10B7C00081A4C801B7012B2D3A2D492D582D0E9477
:10B7D00021D688230CF044C0C801B701A801970105
:10B7E0000E94F6D87B018C016AA97BA98CA99DA92E
:10B7F000905820E030E040E050EC0E94F6D82EA5B2
:10B800003FA548A959A90E94F6D89B01AC01C801DF
:10B81000B7010E9448D50E9463D97B018C016B2D32
:10B820007A2D892D982D9701A8010E9421D6882371
:10B8300024F4EB2CFA2C092D182D6B2D7A2D892D43
:10B84000982D9701A8010E9421D6882349F0C701AD
:10B85000D801F60186A397A3A0A7B1A781E086AB84
:10B86000DF91CF911F910F91FF90EF90DF90CF90DC
:10B87000BF90AF909F908F900895EF92FF920F939B
:10B880001F93CF93DF93F0908A0F00E010E020E049
:10B8900030E06DE4E62E11C0FE9CE0011124C75497
:10B8A000D54FC901B801AE016EDF8F2D8F5F80319A
:10B8B00009F480E0F82E98018E018091890FF81626
:10B8C00059F7C901B80140E050E05DDFDF91CF9149
:10B8D0001F910F91FF90EF900895AF92BF92CF927A
:10B8E000DF92EF92FF920F931F93CF93DF93EB01C1
:10B8F0008A016115710509F466C04115510509F405
:10B9000062C0DAA4CBA4BCA4ADA46EA17FA188A51B
:10B9100099A52D2D3C2D4B2D5A2D0E9421D68823E3
:10B9200009F451C08FA9882309F043C0F801E6A0AB
:10B93000F7A000A511A56D2D7C2D8B2D9A2DA801AA
:10B9400097010E9424D81816A4F5C801B701A801D0
:10B9500097010E94F6D87B018C016AA97BA98CA96A
:10B960009DA9905820E030E040E050EC0E94F6D8CD
:10B970002EA53FA548A959A90E94F6D89B01AC0164
:10B98000C801B7010E9448D50E9463D97B018C0190
:10B990006D2D7C2D8B2D9A2D9701A8010E9421D60B
:10B9A000882324F4ED2CFC2C0B2D1A2DC701D80173
:10B9B00004C08D2D9C2DAB2DBA2D8EA39FA3A8A7BF
:10B9C000B9A781E08EABDF91CF911F910F91FF90CE
:10B9D000EF90DF90CF90BF90AF900895CF92DF921D
:10B9E000EF92FF920F93DF93CF930F920F92CDB709
:10B9F000DEB78091890F8FB7F894F0908A0F8FBFD0
:10BA00008091890F90E040968F1991098F70907006
:10BA10000497FCF00091890F03500F70CC24DD24B3
:10BA200040E050E07DE4E72E12C0802F002309F4AF
:10BA300080E1082F01500E9DC00111248754954FBD
:10BA40009A838983B60149DFA601C980DA800F1580
:10BA500061F70F900F90CF91DF910F91FF90EF90D2
:10BA6000DF90CF900895DF92EF92FF920F931F9394
:10BA7000D0905D0690918A0F8091890F9817C1F040
:10BA800040918A0F242F30E08DE490E0289FF00150
:10BA9000299FF00D389FF00D1124EF5FF44F608166
:10BAA00002C04F5F4F708091890F4817D1F7D62E93
:10BAB000DD2031F1E0909F0FF090A00F0091A10FD9
:10BAC0001091A20FE114F1040105110579F40E940F
:10BAD000531A6C597F4F8F4F9F4F60939F0F7093F6
:10BAE000A00F8093A10F9093A20F07C00E94531A3A
:10BAF0006E157F058007910758F4DD24DA9408C09D
:10BB000010929F0F1092A00F1092A10F1092A20FEF
:10BB100087E06D2D70E00E94C31A1F910F91FF9076
:10BB2000EF90DF9008951092890F10928A0F80E1B4
:10BB3000E9EAFAE0DF011D928A95E9F780E090E0FA
:10BB4000A0E0B0E080938F0F9093900FA093910F9F
:10BB5000B093920F8093930F9093940FA093950FAF
:10BB6000B093960F8093970F9093980FA093990F8F
:10BB7000B0939A0F80939B0F90939C0FA0939D0F6F
:10BB8000B0939E0F80938B0F90938C0FA0938D0F8B
:10BB9000B0938E0F80E090E0A0E8BFE38093690A45
:10BBA00090936A0AA0936B0AB0936C0A08952F923F
:10BBB0003F924F925F926F927F928F929F92AF923D
:10BBC000BF92CF92DF92EF92FF920F931F93DF937A
:10BBD000CF93CDB7DEB766970FB6F894DEBF0FBE32
:10BBE000CDBF9E8B8D8B6A017B0148015901DC0121
:10BBF000D8966D917D918D919C91DB970E94C1D6D5
:10BC0000698B7A8B8B8B9C8BA70196010E94F6D84F
:10BC10000E940ED60E9495D66D837E838F8398876F
:10BC200069897A898B899C89A50194010E94F6D83B
:10BC30000E940ED60E9495D669837A838B839C835B
:10BC40002D813E814F8158852837310541055105A9
:10BC500040F448E750E060E070E04D835E836F831E
:10BC6000788769817A818B819C816837710581052C
:10BC7000910540F488E790E0A0E0B0E089839A83E2
:10BC8000AB83BC83AD89BE89AC5BBF4FAD90BD902B
:10BC9000CD90DC901397A454B040BE8BAD8B6D81DA
:10BCA0007E818F8198850E94C1D66D877E878F8720
:10BCB000988BC601B5010E94C3D61B012C0120E060
:10BCC00030E040E050E00E9421D6882321F4E0E0FB
:10BCD00070E060E028C069897A898B899C899B0122
:10BCE000AC010E94F6D87B018C016D857E858F8525
:10BCF00098899B01AC010E94F6D89B01AC01C80158
:10BD0000B7010E9447D57B018C01C201B101A2019C
:10BD100091010E9448D59B01AC01C801B7010E9466
:10BD200028D6E62F692F2E2F372F482F562FB901EF
:10BD3000CA010E940ED60E9490D63B014C01698137
:10BD40007A818B819C810E94C1D669877A878B8793
:10BD50009C8766277727CB016A197B098C099D0987
:10BD60000E94C3D65B016C0120E030E040E050E06F
:10BD70000E9421D6882321F4E0E070E060E028C032
:10BD800069857A858B859C859B01AC010E94F6D8DC
:10BD90007B018C0169897A898B899C899B01AC0123
:10BDA0000E94F6D89B01AC01C801B7010E9447D59B
:10BDB0007B018C01C601B501A60195010E9448D501
:10BDC0009B01AC01C801B7010E9428D6E62F692F5C
:10BDD0002E2F372F482F562FB901CA010E94FED6A9
:10BDE000ED89FE89A088B188C288D3888601750153
:10BDF000E618F708080919090E9490D6A8019701CA
:10BE0000261B370B480B590B57FF71C0C201B101FC
:10BE100020E030E040E050E00E9421D6882321F469
:10BE2000E0E070E060E044C0C201B101A201910114
:10BE30000E9448D57B018C01C601B5010E94C1D684
:10BE40009B01AC01C801B7010E94F6D87B018C01AF
:10BE50006D857E858F8598899B01AC010E94F6D8FF
:10BE60009B01AC01C801B7010E9447D57B018C0141
:10BE700069857A858B859C859B01AC010E94F6D8EB
:10BE80009B01AC01C801B7010E9448D57B018C0120
:10BE9000C201B10120E030E040E850E40E94F6D851
:10BEA0009B01AC01C801B7010E9428D6E62F692F7B
:10BEB0002E2F372F482F562FB901CA010E940ED6B8
:10BEC0000E9490D6AC01CB01DA013C014D0197FEF6
:10BED00003C06624772443016A147B048C049D0408
:10BEE00010F03501460120E030E040E050E09FB71F
:10BEF000F8946D897E89645B7F4FDB018C91AC5433
:10BF0000B040BE8BAD8B882321F5FD01648A758A14
:10BF1000868A978A260D371D481D591D58962D93E0
:10BF20003D934D935C935B972D813E814F81588566
:10BF3000DC962D933D934D935C93DF97A05CBF4FB0
:10BF400029813A814B815C812D933D934D935C9384
:10BF500013979FBF66960FB6F894DEBF0FBECDBF96
:10BF6000CF91DF911F910F91FF90EF90DF90CF90D5
:10BF7000BF90AF909F908F907F906F905F904F9009
:10BF80003F902F9008954F925F927F928F929F9251
:10BF9000AF92BF92CF92DF92EF92FF920F931F93D7
:10BFA000CF93DF9370908A0FC0E0D0E0EDE44E2E87
:10BFB000512C45C02097A9F18EA9882361F4849C57
:10BFC000F001859CF00D949CF00D1124E754F54F81
:10BFD00086A9882331F1EAA0FBA00CA11DA16EA1C6
:10BFE0007FA188A599A5A80197010E9428D65B0189
:10BFF0006C01849CF001859CF00D949CF00D112443
:10C00000E754F54F66A177A180A591A5A8019701F6
:10C010000E9428D68B019C01CE01B601A501C7DD87
:10C020001EAA739480E1781609F47724849CE001B9
:10C03000859CD00D949CD00D1124C754D54F872CCE
:10C04000992487FC90948091890F90E08816990636
:10C0500009F0B0CF2097E9F0EAA0FBA00CA11DA148
:10C060006EA17FA188A599A5A80197010E9428D655
:10C070005B016C016DEC7CEC8CE49DE3A801970105
:10C080000E9428D68B019C01CE01B601A5018FDD4F
:10C090001EAADF91CF911F910F91FF90EF90DF903B
:10C0A000CF90BF90AF909F908F907F905F904F9078
:10C0B000089594DCE2DB67CF2F923F924F925F921C
:10C0C0006F927F928F929F92AF92BF92CF92DF92A8
:10C0D000EF92FF920F931F93DF93CF93CDB7DEB70D
:10C0E000C659D0400FB6F894DEBF0FBECDBF5C017D
:10C0F0004B013A012901CD56DF4FE882C359D040A8
:10C10000CC56DF4FF882C459D040CB56DF4F08835E
:10C11000C559D040CA56DF4F1883C659D040E19662
:10C12000DFAECEAEE1978091890F8F5F803109F449
:10C1300080E0282F332727FD30953CA72BA706C08A
:10C140000E94798B0E947A300E94CB9480918A0F52
:10C1500090E04BA55CA58417950791F36091590A6F
:10C1600070915A0A80915B0A90915C0AAF966CAF0D
:10C170007DAF8EAF9FAFAF97D5012D913D914D9182
:10C180005C910E94F6D80E94C6D8EE966FAFEE97EB
:10C19000EF967FAFEF97C158DF4F8883CF57D040DE
:10C1A000C058DF4F9883C058D04020915D0A30912D
:10C1B0005E0A40915F0A5091600AAB962CAF3DAF8A
:10C1C0004EAF5FAFAB97CA01B901D4012D913D913C
:10C1D0004D915C910E94F6D80E94C6D8CF57DF4F90
:10C1E0006883C158D040CE57DF4F7883C258D040C3
:10C1F000CD57DF4F8883C358D040CC57DF4F98834B
:10C20000C458D0402091610A3091620A4091630A7B
:10C210005091640AA7962CAF3DAF4EAF5FAFA79782
:10C22000CA01B901D3012D913D914D915C910E94BC
:10C23000F6D80E94C6D8CB57DF4F6883C558D04088
:10C24000CA57DF4F7883C658D040C957DF4F88831D
:10C25000C758D040C857DF4F9883C858D040209166
:10C26000650A3091660A4091670A5091680AA39660
:10C270002CAF3DAF4EAF5FAFA397E196AEADBFAD74
:10C28000E1978C91082F10E0CA01B901F2012081D9
:10C290003181428153810E94F6D8000F111F000F97
:10C2A000111FF801E759F54F2081318142815381F7
:10C2B0000E94F6D80E94C6D8C757DF4F6883C95876
:10C2C000D040C657DF4F7883CA58D040C557DF4F9C
:10C2D0008883CB58D040C457DF4F9883CC58D04088
:10C2E0008091B50A9091B60AA091B70AB091B80AA8
:10C2F000C757DF4F288139814A815B81C958D040B7
:10C30000281739074A075B0709F4B2C002501E4ECE
:10C31000D8016D917D918D919C9120917603309102
:10C32000770340917803509179030E9421D68823A6
:10C330000CF033C0C757DF4F288139814A815B81B8
:10C34000C958D0402093B50A3093B60A4093B70A33
:10C350005093B80AE5E9FAE0949108C08091C000D2
:10C3600085FFFCCF9093C600319694919923B1F745
:10C37000E9EBFAE0949108C08091C00085FFFCCF02
:10C380009093C600319694919923B1F78091C000A3
:10C3900085FFFCCF8AE08093C6008091B50A90911A
:10C3A000B60AA091B70AB091B80AC757DF4F2881E3
:10C3B00039814A815B81C958D040281B390B4A0B0F
:10C3C0005B0BCA01B90157FF07C090958095709526
:10C3D00061957F4F8F4F9F4F0E94C3D67B018C0189
:10C3E000A3966CAD7DAD8EAD9FADA39720E030E000
:10C3F00046EE53E40E94F6D89B01AC01C801B70198
:10C400000E9424D818160CF033C0C757DF4F48815C
:10C4100059816A817B81C958D0404093B50A5093B5
:10C42000B60A6093B70A7093B80AE5E9FAE0949106
:10C4300008C08091C00085FFFCCF9093C600319664
:10C4400094919923B1F7EBE9FAE0949108C08091B7
:10C45000C00085FFFCCF9093C6003196949199233C
:10C46000B1F78091C00085FFFCCF8AE08093C600C1
:10C470008091890F682F70E06F967FAF6EAF6F97D6
:10C480008DE490E0689FF001699FF00D789FF00DBA
:10C490001124E754F54FE45BFF4F1082EC54F04059
:10C4A0008091A90A9091AA0AA091AB0AB091AC0A16
:10C4B0006D968CAF9DAFAEAFBFAF6D97C358DF4FDA
:10C4C000288139814A815B81CD57D040281B390BA7
:10C4D0004A0B5B0B69962CAF3DAF4EAF5FAF6997D0
:10C4E000208331834283538357FF0DC0DA01C90192
:10C4F000B095A095909581959F4FAF4FBF4F80838A
:10C500009183A283B3834091AD0A5091AE0A6091AA
:10C51000AF0A7091B00A65964CAF5DAF6EAF7FAF5A
:10C520006597CF57DF4F88819981AA81BB81C15818
:10C53000D040841B950BA60BB70B61968CAF9DAFBB
:10C54000AEAFBFAF61978DE490E06F96AEADBFAD7B
:10C550006F97A89FF001A99FF00DB89FF00D1124CF
:10C56000E754F54F61962CAD3DAD4EAD5FAD619793
:10C57000248335834683578357FF0DC0DA01C901F1
:10C58000B095A095909581959F4FAF4FBF4F8483F5
:10C590009583A683B7834091B10A5091B20A609106
:10C5A000B30A7091B40A2D964CAF5DAF6EAF7FAFFA
:10C5B0002D97CB57DF4F88819981AA81BB81C558C0
:10C5C000D040841B950BA60BB70B29968CAF9DAF63
:10C5D000AEAFBFAF29978DE490E06F96AEADBFAD23
:10C5E0006F97A89FF001A99FF00DB89FF00D11243F
:10C5F000E754F54F29962CAD3DAD4EAD5FAD299773
:10C60000208731874287538757FF0DC0DA01C90160
:10C61000B095A095909581959F4FAF4FBF4F808764
:10C620009187A287B3872090B50A3090B60A4090D0
:10C63000B70A5090B80AC757DF4F488159816A81BD
:10C640007B81C958D04042195309640975094DA32B
:10C650005EA36FA378A79A01AB0157FF07C050955F
:10C660004095309521953F4F4F4F5F4F8DE490E0BF
:10C670006F966EAD7FAD6F97689F8001699F100DBB
:10C68000789F100D11240754154F7CE0E72EF12CF4
:10C69000E00EF11EE196AEADBFADE197EC91F0E09A
:10C6A000EE0FFF1FE25BFC4F60817181882777FDF1
:10C6B0008095982F0E949DDC24E630E040E050E019
:10C6C0000E9411DDF8012487D70111963C93119740
:10C6D00012964C93129713965C93608071808280BF
:10C6E0009380A480B580C680D780E084F1840285E1
:10C6F0001385C901DA018E159F05A007B10714F44F
:10C70000D801C7018A159B05AC05BD0514F4D601F7
:10C71000C5019C01AD0186159705A805B90514F45E
:10C72000A40193018DE490E06F96EEADFFAD6F979D
:10C73000E89FB001E99F700DF89F700D11246754B8
:10C74000754FDB0150962D933D934D935C9353971A
:10C75000263031054105510510F40C949A6CFB010B
:10C76000E85BFF4F80915D0690E0A0E0B0E0808341
:10C770009183A283B383FB0110A2C358DF4F2881AA
:10C7800039814A815B81CD57D0406D968CAD9DAD8E
:10C79000AEADBFAD6D97281739074A075B0714F494
:10C7A00081E080A3CF57DF4F288139814A815B81A7
:10C7B000C158D04065966CAD7DAD8EAD9FAD65978F
:10C7C000261737074807590794F48DE490E06F96D1
:10C7D000AEADBFAD6F97A89FF001A99FF00DB89FB8
:10C7E000F00D1124E754F54F80A1826080A3CB5750
:10C7F000DF4F288139814A815B81C558D0402D9611
:10C800006CAD7DAD8EAD9FAD2D97261737074807D0
:10C81000590794F48DE490E06F96AEADBFAD6F977D
:10C82000A89FF001A99FF00DB89FF00D1124E754C7
:10C83000F54F80A1846080A3C757DF4F28813981DD
:10C840004A815B81C958D0402215330544055505FE
:10C8500094F48DE490E06F964EAD5FAD6F97489F76
:10C86000F001499FF00D589FF00D1124E754F54F4A
:10C8700080A1886080A38DE490E06F966EAD7FAD5F
:10C880006F97689FF001699FF00D789FF00D11245C
:10C89000E754F54FE196AEADBFADE1978C9181A322
:10C8A000208131814281538125962CAF3DAF4EAF1F
:10C8B0005FAF2597211531054105510509F0159800
:10C8C0008DE490E06F964EAD5FAD6F97489FF0019D
:10C8D000499FF00D589FF00D1124E754F54F6480E7
:10C8E000758086809780611471048104910409F039
:10C8F00046988DE490E06F966EAD7FAD6F97689F20
:10C90000F001699FF00D789FF00D1124E754F54F69
:10C91000A084B184C284D384A114B104C104D1041D
:10C9200009F043988DE490E06F96AEADBFAD6F9780
:10C93000A89FF001A99FF00DB89FF00D1124E754B6
:10C94000F54F84859585A685B7850097A105B10526
:10C9500051F0409820907D0A30907E0A40907F0AE6
:10C960005090800A08C02090950A3090960A409016
:10C97000970A5090980ACD56DF4F6881C359D0402E
:10C98000CC56DF4F7881C459D040CB56DF4F8881D9
:10C99000C559D040CA56DF4F9881C659D040A20130
:10C9A00091010E9421D687FD16C0CD56DF4F8881A8
:10C9B000C359D040CC56DF4F9881C459D040CB5694
:10C9C000DF4FA881C559D040CA56DF4FB881C6593C
:10C9D000D0401C012D0169966CAD7DAD8EAD9FAD33
:10C9E00069970E94C3D6AF962CAD3DAD4EAD5FADFD
:10C9F000AF970E9428D6EA966FAFEA97EB967FAF83
:10CA0000EB97EC968FAFEC97ED969FAFED97AC015F
:10CA1000CB01DA0189839A83AB83BC8361966CADC9
:10CA20007DAD8EAD9FAD61970E94C3D6AB962CAD08
:10CA30003DAD4EAD5FADAB970E9428D6E6966FAF89
:10CA4000E697E7967FAFE797E8968FAFE897E99686
:10CA50009FAFE997AC01CB01DA018D839E83AF8351
:10CA6000B88729966CAD7DAD8EAD9FAD29970E949C
:10CA7000C3D6A7962CAD3DAD4EAD5FADA7970E9436
:10CA800028D6E2966FAFE297E3967FAFE397E496FE
:10CA90008FAFE497E5969FAFE597AC01CB01DA0144
:10CAA00089879A87AB87BC876DA17EA18FA198A546
:10CAB0000E94C3D6A3962CAD3DAD4EAD5FADA397FE
:10CAC0000E9428D67B018C01E196AEADBFADE19707
:10CAD000EC91F0E0EE0FFF1FE25BFC4F6081718193
:10CAE000882777FD8095982F0E94C3D69B01AC01C3
:10CAF000C801B7010E94F6D820E030E048EC52E4CB
:10CB00000E9428D69B01AC016D877E878F87988B0A
:10CB100025966CAD7DAD8EAD9FAD259766307105C8
:10CB2000810591051CF576E0671671048104910476
:10CB3000ECF486E0A816B104C104D104BCF48DE481
:10CB400090E06F96AEADBFAD6F97A89FF001A99F23
:10CB5000F00DB89FF00D1124E754F54FDA01C9012B
:10CB6000BF7786A797A7A0ABB1AB55C0EA962FAD0C
:10CB7000EA97EB963FADEB97EC964FADEC97ED96C1
:10CB80005FADED97B901CA010E94A1D93B014C01EB
:10CB9000E6962FADE697E7963FADE797E8964FAD5F
:10CBA000E897E9965FADE997B901CA010E94A1D95A
:10CBB0005B016C01E2962FADE297E3963FADE39700
:10CBC000E4964FADE497E5965FADE597B901CA01EC
:10CBD0000E94A1D97B018C01C401B301A60195017A
:10CBE0000E9448D5A80197010E9448D50E9463D9A8
:10CBF0002DE430E06F964EAD5FAD6F97429FF00130
:10CC0000439FF00D529FF00D1124E754F54F66A796
:10CC100077A780AB91AB8DE490E06F966EAD7FAD62
:10CC20006F97689FF001699FF00D789FF00D1124B8
:10CC3000E754F54F86A597A5A0A9B1A921968CAF79
:10CC40009DAFAEAFBFAF219760E070E080E89FE39B
:10CC500021962CAD3DAD4EAD5FAD21970E9428D6FB
:10CC60009B01AC01C201B1010E94F6D82B013C012D
:10CC70008091890F90918A0FA82FB0E05096A91B40
:10CC8000B109AF70B070BAA7A9A7A230B1050CF472
:10CC900051C05D01CC24B7FCC094DC2CC601B501A9
:10CCA0000E94C3D620E030E040E051E40E9421D64B
:10CCB00088230CF03FC060E074E284E799E4A301AC
:10CCC00092010E9428D60E94C6D87B018C016091F7
:10CCD000450A7091460A8091470A9091480AE616E3
:10CCE000F7060807190730F56E197F09800B910BBD
:10CCF000660F771F881F991FA60195010E94EFDC20
:10CD0000CA01B9010E94C1D60E94C6D89B01AC01DC
:10CD10002E0D3F1D401F511FCA01B9010E94C1D6EF
:10CD20009B01AC0160E074E284E799E40E9428D69C
:10CD30002B013C018DE490E06F96EEADFFAD6F9757
:10CD4000E89F8001E99F100DF89F100D11240754F2
:10CD5000154F21966CAD7DAD8EAD9FAD2197A30192
:10CD600092010E94F6D8D80192966D937D938D938F
:10CD70009C93959750966D917D918D919C91539731
:10CD80000E94C1D6A30192010E94F6D80E940ED63D
:10CD90000E9495D6F80160AF71AF82AF93AFC357D1
:10CDA000DF4F1882CD58D040C257DF4F1882CE587F
:10CDB000D04020E8222E9FE3392E88249924E1E0F8
:10CDC000F0E0EC0FFD1FE80DF91DC301B201208159
:10CDD0003181428153810E94F6D8E1E1F0E0EC0F0D
:10CDE000FD1FE80DF91D60837183828393835B01CE
:10CDF0006C01E894D7F8F401E75BF54FE080F1802F
:10CE000002811381C601B501A80197010E9424D8AF
:10CE10001816CCF4C801B701A60195010E9428D6C6
:10CE20006B017C01C357DF4F6881CD58D040C2579A
:10CE3000DF4F7881CE58D040C101A70196010E94F2
:10CE400021D688236CF4C357DF4F8881CD58D0405A
:10CE5000C257DF4F9881CE58D040D1016C017D017F
:10CE600024E030E0820E931E30E18316910471F0CD
:10CE7000D701C601C357DF4FC882CD58D040C25733
:10CE8000DF4F9883CE58D0401D0199CFC701B6011E
:10CE900020E030E040E85FE30E9421D688230CF0D8
:10CEA0004CC08E010F5E1F4F81E2A82EB12CAC0E3C
:10CEB000BD1ED8016D917D918D919C91A701960128
:10CEC0000E94F6D8F80161937193819391938F0139
:10CED000EA15FB0571F78DE490E06F962EAD3FAD3E
:10CEE0006F97289F8001299F100D389F100D1124E6
:10CEF0000754154FD80192966D917D918D919C911B
:10CF00009597A70196010E94F6D8F80162A373A332
:10CF100084A395A360AD71AD82AD93AD0E94C1D6DF
:10CF2000A70196010E94F6D80E9495D6D801D896FE
:10CF30006D937D938D939C93DB978DE490E06F963A
:10CF4000EEADFFAD6F97E89F8001E99F100DF89F50
:10CF5000100D11240754154FD80150966D917D91F5
:10CF60008D919C9153970E94C1D6F80126A537A5B3
:10CF700040A951A90E9428D61B012C01F8018081EB
:10CF80009181A281B3810097A105B10549F5848102
:10CF90009581A681B7810097A105B10509F5808526
:10CFA0009185A285B3850097A105B105C9F4C20199
:10CFB000B1012091850A3091860A4091870A5091EB
:10CFC000880A0E94F6D80E940ED60C5B1F4F0E9462
:10CFD00095D6D8016D937D938D939C93139771C1D2
:10CFE000C201B1012091810A3091820A4091830AE5
:10CFF0005091840A0E94F6D80E940ED60E9495D6BF
:10D000002DE430E06F96EEADFFAD6F97E29F6001CB
:10D01000E39FD00CF29FD00C112429EB3AE0C20E12
:10D02000D31E14E4612E712C6C0C7D1CD3016D9306
:10D030007D938D939C9313978090990A90909A0A70
:10D04000A0909B0AB0909C0A0E94C1D67B018C01E3
:10D05000F60160817181828193810E94C3D69B0118
:10D06000AC01C801B7010E94F6D87B018C01D60142
:10D0700050966D917D918D919C9153970E94C1D650
:10D080009B01AC01C801B7010E9428D67B018C012D
:10D09000C501B4010E94C1D69B01AC01C801B70112
:10D0A0000E9424D818162CF4F30180829182A28267
:10D0B000B38280909D0A90909E0AA0909F0AB090A3
:10D0C000A00A8DE490E06F962EAD3FAD6F97289F3C
:10D0D0006001299FD00C389FD00C112449EB5AE0F5
:10D0E000C40ED51EB4E46B2E712C6C0C7D1CD301C8
:10D0F0006D917D918D919C910E94C1D67B018C0197
:10D10000F60164817581868197810E94C3D69B0157
:10D11000AC01C801B7010E94F6D87B018C01D60191
:10D1200050966D917D918D919C9153970E94C1D69F
:10D130009B01AC01C801B7010E9428D67B018C017C
:10D14000C501B4010E94C1D69B01AC01C801B70161
:10D150000E9424D818162CF4F30180829182A282B6
:10D16000B3828090A50A9090A60AA090A70AB090DA
:10D17000A80A8DE490E06F962EAD3FAD6F97289F83
:10D180006001299FD00C389FD00C112449EB5AE044
:10D19000C40ED51EA4E46A2E712C6C0C7D1CD30128
:10D1A0006D917D918D919C910E94C1D67B018C01E6
:10D1B000F60164857585868597850E94C3D69B0197
:10D1C000AC01C801B7010E94F6D87B018C01D601E1
:10D1D00050966D917D918D919C9153970E94C1D6EF
:10D1E0009B01AC01C801B7010E9428D67B018C01CC
:10D1F000C501B4010E94C1D69B01AC01C801B701B1
:10D200000E9424D818162CF4F30180829182A28205
:10D21000B3828090A10A9090A20AA090A30AB09035
:10D22000A40A8DE490E06F962EAD3FAD6F97289FD6
:10D230006001299FD00C389FD00C112449EB5AE093
:10D24000C40ED51EF4E46F2E712C6C0C7D1CD30122
:10D250006D917D918D919C910E94C1D67B018C0135
:10D26000F60160857185828593850E94C3D69B01F6
:10D27000AC01C801B7010E94F6D87B018C01D60130
:10D2800050966D917D918D919C9153970E94C1D63E
:10D290009B01AC01C801B7010E9428D67B018C011B
:10D2A000C501B4010E94C1D69B01AC01C801B70100
:10D2B0000E9424D818162CF4F30180829182A28255
:10D2C000B3828DE490E06F962EAD3FAD6F97289FAF
:10D2D0006001299FD00C389FD00C112449EB5AE0F3
:10D2E000C40ED51EF601EC5BFF4F60817181828117
:10D2F00093810E94C1D67B018C01A20191010E9401
:10D3000028D6D601D2966D937D938D939C93D59715
:10D31000C801B7012DEB37E346E051E40E94F6D88F
:10D320000E9490D6F601648F758F868F978F6090DC
:10D33000890A70908A0A80908B0A90908C0AC401A6
:10D34000B30120E030E040E05FE30E94F6D85B01EB
:10D350006C01298D3A8D4B8D5C8D29AF3AAF4BAF67
:10D360005CAF40918D0A50918E0A60918F0A709146
:10D37000900A4DAB5EAB6FAB78AFCB01BA0120E04A
:10D3800030E040E05FE30E94F6D87B018C0169AD9C
:10D390007AAD8BAD9CAD9F77A80197010E9424D8F0
:10D3A000181644F4C601B501A80197010E9421D6C0
:10D3B000882314F4860175016D8D7E8D8F8D98A163
:10D3C00069AB7AAB8BAB9CAB8091910A9091920A3E
:10D3D000A091930AB091940A8DA79EA7AFA7B8AB6E
:10D3E000BC01CD0120E030E040E05FE30E94F6D8D0
:10D3F0001B012C0169A97AA98BA99CA99F77A2017D
:10D4000091010E9424D8181644F4C801B701A20162
:10D4100091010E9421D6882314F4170128018DE47C
:10D4200090E06F96AEADBFAD6F97A89FF001A99F3A
:10D43000F00DB89FF00D1124E754F54F22A133A150
:10D4400044A155A129A33AA34BA35CA3C201B101F6
:10D450000E9421D687FD04C029A03AA04BA05CA061
:10D4600049A55AA5423051050CF401C150918B0FCA
:10D47000C157DF4F5883CF58D04060918C0FC057B1
:10D48000DF4F6883C059D04070918D0FCF56DF4F6A
:10D490007883C159D04080918E0FCE56DF4F88835C
:10D4A000C259D040652FC057DF4F7881C059D04056
:10D4B000CF56DF4F8881C159D040CE56DF4F98817B
:10D4C000C259D04027E137EB41ED58E30E9424D800
:10D4D00018160CF0CCC069897A898B899C892091B7
:10D4E0008F0F3091900F4091910F5091920F0E94A9
:10D4F00047D50E94A1D97B018C016D897E898F89D6
:10D50000988D2091930F3091940F4091950F5091E9
:10D51000960F0E9447D50E94A1D99B01AC01C8017A
:10D52000B7010E9448D50E9463D97B018C01A401F8
:10D5300093010E9424D818165CF00F2EF0E06F2E95
:10D54000F0E07F2EF0E88F2EFFE39F2EF02D08C035
:10D55000C401B301A80197010E9428D63B014C01E8
:10D5600069AD7AAD8BAD9CAD2091970F3091980F3E
:10D570004091990F50919A0F0E9447D57B018C01E1
:10D58000E89417F9C801B7012DA93EA94FA958ADD4
:10D590000E9424D8181694F46DA97EA98FA998AD7D
:10D5A000A80197010E9428D65B016C01C401B30158
:10D5B000A60195010E9421D6882314F46401530129
:10D5C00069A97AA98BA99CA920919B0F30919C0FE6
:10D5D00040919D0F50919E0F0E9447D57B018C0179
:10D5E000E89417F9C801B7012DA53EA54FA558A984
:10D5F0000E9424D8181694F46DA57EA58FA598A92D
:10D60000A80197010E9428D67B018C01C601B501B3
:10D61000A80197010E9421D6882314F48601750180
:10D6200069A17AA18BA19CA1A80197010E94F6D8BB
:10D630007B018C01C157DF4F6881CF58D040C05764
:10D64000DF4F7881C059D040CF56DF4F8881C15914
:10D65000D040CE56DF4F9881C259D040A8019701E3
:10D660000E9421D687FD19C0D801C70102C0D2018E
:10D67000C101C157DF4F8883CF58D040C057DF4F1B
:10D680009883C059D040CF56DF4FA883C159D040AE
:10D69000CE56DF4FB883C259D0408DE490E06F96EC
:10D6A000AEADBFAD6F97A89F8001A99F100DB89F29
:10D6B000100D11240754154FC157DF4F8881CF58E3
:10D6C000D040C057DF4F9881C059D040CF56DF4F70
:10D6D000A881C159D040CE56DF4FB881C259D04041
:10D6E000F80182A793A7A4A7B5A762A973A984A9E3
:10D6F00095A9905820E030E040E050EC0E94F6D828
:10D70000D8019E962D913D914D915C91D1970E94AB
:10D71000F6D82BE037ED43E25BE30E9448D50E9448
:10D7200063D9F62EE72ED82EC92EC157DF4F688158
:10D73000CF58D040C057DF4F7881C059D040CF5626
:10D74000DF4F8881C159D040CE56DF4F9881C259F2
:10D75000D0402F2D3E2D4D2D5C2D0E9421D687FDD2
:10D7600014C0C157DF4FF882CF58D040C057DF4FA9
:10D77000E882C059D040CF56DF4FD882C159D0403F
:10D78000CE56DF4FC882C259D0408DE490E06F96EC
:10D79000EEADFFAD6F97E89F8001E99F100DF89FF8
:10D7A000100D11240754154FC157DF4F8881CF58F2
:10D7B000D040C057DF4F9881C059D040CF56DF4F7F
:10D7C000A881C159D040CE56DF4FB881C259D04050
:10D7D000F80186A397A3A0A7B1A762A173A184A112
:10D7E00095A12F2D3E2D4D2D5C2D0E9421D6181672
:10D7F0002CF081E0D801D7968C9302C0F80117AACB
:10D800008DE490E06F962EAD3FAD6F97289FF001AD
:10D81000299FF00D389FF00D1124E754F54F81E05A
:10D8200086ABAFE8BFE0FE01719680E101900D92FA
:10D830008150E1F78DE490E06F964EAD5FAD6F974C
:10D84000489F6001499FD00C589FD00C112469EB70
:10D850007AE0C60ED71ED6019296ED90FD900D91FE
:10D860001C919597E0928B0FF0928C0F00938D0F87
:10D8700010938E0F96966D917D918D919C919997B5
:10D88000A80197010E9428D64B015C01C201B10199
:10D89000A80197010E9428D68B019C01C601B50101
:10D8A000A4010E94D75DBBA5B093890FC757DF4F76
:10D8B000288139814A815B81C958D0402093B50ABB
:10D8C0003093B60A4093B70A5093B80ACB57DF4F4C
:10D8D000488159816A817B81C558D0404093B10A03
:10D8E0005093B20A6093B30A7093B40ACF57DF4FD4
:10D8F000688179818A819B81C158D0406093AD0A4B
:10D900007093AE0A8093AF0A9093B00AC358DF4F6A
:10D9100088819981AA81BB81CD57D0408093A90A83
:10D920009093AA0AA093AB0AB093AC0A0E945960E4
:10D930000E94E27DCA56DF4F0FB6F894DEBF0FBEDD
:10D94000CDBFCF91DF911F910F91FF90EF90DF90AE
:10D95000CF90BF90AF909F908F907F906F905F908F
:10D960004F903F902F900895FF920F931F93CF9366
:10D97000DF938B010E94531AEB01FF24FA9409C034
:10D980000E94531A6C1B7D0B6017710710F080E02A
:10D9900008C0FEBC0DB407FEFDCF8EB58F3F81F7EA
:10D9A00081E0DF91CF911F910F91FF900895FC01CD
:10D9B0004281242F30E0C9019595879580658CBD03
:10D9C00040FF02C080E004C080E0463009F081E002
:10D9D0008DBD808160E00C94541CDF92EF92FF9229
:10D9E0000F931F93CF93DF93EC01D62E79018A0119
:10D9F000DEDFCE016CE271E0B7DF8D2D80648EBD7D
:10DA00000DB407FEFDCF28E130E0D801C701022E9A
:10DA100004C0B695A795979587950A94D2F78EBDC1
:10DA20000DB407FEFDCF285030408FEF283F380758
:10DA300061F7DD2011F485E906C088E0D81611F4FD
:10DA400087E801C08FEF8EBD0DB407FEFDCF8CE0DF
:10DA5000D81631F48FEF8EBD0DB407FEFDCF8EB515
:10DA60009FEF2FEF2EBD0DB407FEFDCF8EB587FFC4
:10DA700004C0992311F09150F5CF8B83DF91CF91A2
:10DA80001F910F91FF90EF90DF900895FC0180812E
:10DA900061E00C94541CDC016EBDFA0120E030E022
:10DAA0000DB407FEFDCF80818EBD0DB407FEFDCF06
:10DAB00081818EBD2E5F3F4F329682E02030380745
:10DAC00079F70DB407FEFDCF8FEF8EBD0DB407FEC5
:10DAD000FDCF8FEF8EBD0DB407FEFDCF8FEF8EBD56
:10DAE0000DB407FEFDCF8EB513968C9313978F71EF
:10DAF000853011F481E0089583E111968C9311979C
:10DB0000CD01C4DF80E00895CF92DF92EF92FF92C3
:10DB10000F931F93CF93DF93EC017A018B0169017F
:10DB20008C81833039F059E0EE0CFF1C001F111F6F
:10DB30005A95D1F7CE0168E1A80197014EDF8823FD
:10DB400011F086E020C0CE016EEFA601A4DF88238D
:10DB5000D9F0CE0168E572E007DF882311F487E190
:10DB600012C0CE016DE020E030E040E050E035DF53
:10DB7000882341F48FEF8EBD0DB407FEFDCF8EB527
:10DB8000882371F086E18983CE0180DF80E0DF9118
:10DB9000CF911F910F91FF90EF90DF90CF9008955C
:10DBA000CE0174DF81E0F3CFBF92CF92DF92EF928C
:10DBB000FF920F931F93CF93DF93EC016B018A01C8
:10DBC0000E94531A7B01BB24BA9409C00E94531AC5
:10DBD0006E197F096D52714010F081E15FC0BEBCCB
:10DBE0000DB407FEFDCF8EB58B838F3F79F38E3F4B
:10DBF00011F08FE053C0D801119701151105D9F02C
:10DC00008FEF8EBD20E030E09FEF0BC00DB407FE1C
:10DC1000FDCF8EB5F601E20FF31F80839EBD2F5F0F
:10DC20003F4F2A173B0790F30DB407FEFDCF8EB58B
:10DC3000AC0DBD1D8C9340E050E060E070E016C07C
:10DC4000272F3327F601E40FF51F808190E0282766
:10DC50003927220F331F2D52354FF90185919491A9
:10DC6000762F6627682779274F5F5F4F4017510748
:10DC700038F38FEF8EBD0DB407FEFDCF3EB58FEFAD
:10DC80008EBD0DB407FEFDCF2EB5932F80E030E0A2
:10DC9000822B932B6817790731F080E28983CE01BC
:10DCA000F5DE80E003C0CE01F1DE81E0DF91CF91AF
:10DCB0001F910F91FF90EF90DF90CF90BF9008954C
:10DCC000AF92BF92CF92DF92EF92FF920F931F938A
:10DCD000CF93DF93EC017A018B0159018C81833062
:10DCE00039F029E0EE0CFF1C001F111F2A95D1F717
:10DCF00093E0D92E84E0C82EDA94CE0161E1A80128
:10DD000097016BDE882311F0C98209C0CE01B501ED
:10DD100040E052E049DF882311F081E010C0DD20AF
:10DD200059F0CE01B3DECE016CE020E030E040E0FF
:10DD300050E053DE1982E0CFCE01A8DE80E0DF9113
:10DD4000CF911F910F91FF90EF90DF90CF90BF90F8
:10DD5000AF900895BF92CF92DF92EF92FF920F9310
:10DD60001F93CF93DF93EC01B62E1C821982488358
:10DD70000E94531A6B01888161E00E94A11BCE01B1
:10DD800085DE82E360E00E94A11B83E361E00E94E4
:10DD9000A11B84E361E00E94A11B85E361E00E9476
:10DDA000A11B85E361E00E94541C85E08A8382E523
:10DDB0008CBD1DBC80E09FEF9EBD0DB407FEFDCF66
:10DDC0008F5F8A30C9F709C00E94531A6C197D0908
:10DDD000615D774010F081E059C0CE0160E020E045
:10DDE00030E040E050E0F9DD182F8B83813061F79F
:10DDF000CE0168E02AEA31E040E050E0EEDD82FF4B
:10DE000002C01C8311C080E02FEF2EBD0DB407FEB1
:10DE1000FDCF9EB58F5F8430C1F79B839A3A11F096
:10DE200082E034C082E08C838C81823021F0EE2449
:10DE3000FF2487010FC0E12CF12C012D50E4152F98
:10DE400009C00E94531A6C197D09615D774010F07A
:10DE50008AE01CC0CE0167E320E030E040E050E003
:10DE6000BCDDCE0169E2A8019701B7DD8B83882371
:10DE700041F78C81823019F5CE016AE320E030E071
:10DE800040E050E0AADD882329F088E08983CE01B4
:10DE9000FDDD20C08FEF8EBD0DB407FEFDCF8EB52A
:10DEA000807C803C11F483E08C8380E09FEF9EBDFA
:10DEB0000DB407FEFDCF2EB58F5F8330C1F7CE01C5
:10DEC000E5DD86E08B1518F488E1898303C0BA820A
:10DED00081E001C080E0DF91CF911F910F91FF9011
:10DEE000EF90DF90CF90BF900895CF93DF93DC0148
:10DEF000EB01BA0180E090E020E2FE01E80FF91F9B
:10DF0000208301968B309105C1F757E040E022C095
:10DF10002E3219F083ED9CE007C05A3049F15AE0E7
:10DF200048E017C0321721F1FC01019634913323E8
:10DF3000C9F75417E8F02132D8F02F37C8F4822FF0
:10DF400081568A3108F42052FE01E40FF11D20832E
:10DF50004F5F11962C91222311F02F32C9F6FB014D
:10DF6000B183A08390E08881803219F091E001C0F4
:10DF700090E0892FDF91CF9108956F927F928F92D9
:10DF80009F92AF92BF92CF92DF92EF92FF920F9348
:10DF90001F93CF93DF93EC017A018B012B81222316
:10DFA00009F480C089899A89AB89BC89841795074F
:10DFB000A607B70708F476C085C0E114F10401058F
:10DFC000110551F41C821D821E821F82188619863B
:10DFD0001A861B8681E067C0288539854A855B855E
:10DFE000E98DFA8D858590E00996215030404040BA
:10DFF000504039014A01082E04C0969487947794C2
:10E0000067940A94D2F72F5F3F4F4F4F5F4F0894AA
:10E01000E108F108010911095701680104C0D6940B
:10E02000C794B794A7948A95D2F70894E11CF11C81
:10E03000011D111DA614B704C804D90428F0211528
:10E0400031054105510549F48D899E89AF89B88D07
:10E050008C839D83AE83BF8316C0A618B708C808FB
:10E06000D90811C04C815D816E817F81898D9A8D27
:10E0700094010E94917B0894A108B108C108D108BD
:10E08000882331F40FC084E0882E912C8C0E9D1EC5
:10E09000A114B104C104D10429F7E886F9860A87DE
:10E0A0001B8798CF80E0DF91CF911F910F91FF9058
:10E0B000EF90DF90CF90BF90AF909F908F907F9028
:10E0C0006F900895223009F078CFE7CFCF93DF9398
:10E0D000EC018C859D85AE85BF8540E0611141E0F6
:10E0E000BC01CD010E945F79882319F420E030E063
:10E0F0000AC08889282F30E095E0220F331F9A95B7
:10E10000E1F72755304FC901DF91CF9108950F9363
:10E110001F93CF93DF938C01FC0183818823E9F166
:10E12000818187FF37C0C80161E0D0DFEC01009733
:10E13000A1F18881853E89F1F8018381823040F424
:10E1400081899289A389B4898C8F9D8FAE8FBF8F6F
:10E15000F801858996899B8F8A8F85899689A789F9
:10E16000B08DCD01AA27BB279D8B8C8BE091A30F8F
:10E17000F091A40F309751F0BE016A5E7F4FCE013F
:10E1800048961995888D998D9B8B8A8BF801818192
:10E190008F7781830E94247904C081E0F801808315
:10E1A00080E0DF91CF911F910F9108950F931F93FE
:10E1B0008C01ADDFF80113821F910F910895FC01CE
:10E1C0008381882311F0CF01F1CF08956F927F9260
:10E1D0008F929F92AF92BF92CF92DF92EF92FF9277
:10E1E0000F931F93DF93CF9300D00F92CDB7DEB77D
:10E1F0007C015A016B01DC0113968C9113978130DD
:10E2000009F08EC011968C9181FF8AC09DC0009745
:10E21000A105B10511F481E084C0F7016084718427
:10E2200082849384C701B601A501A7DE882309F47F
:10E2300077C0D70159968D919C915A97A114B1043A
:10E24000C104D10489F455964D915D916D917C91F5
:10E2500058970E94067C882309F462C0F701158A4A
:10E26000168A178A108E44C0D70114964D915D917D
:10E270006D917C9117979E012F5F3F4F0E94917B7C
:10E28000882309F44DC0D7015996ED91FC915A9716
:10E2900049815A816B817C818789803149F4483F6B
:10E2A000BFEF5B07B0E06B07B0E07B0748F020C032
:10E2B000483F8FEF58078FEF68078FE07807C0F46B
:10E2C000CF010E94067C882359F1D70114964D9105
:10E2D0005D916D917C91179759968D919C915A976C
:10E2E0000FEF1FEF2FEF3FE00E940B7B8823C1F061
:10E2F000F701A18AB28AC38AD48A81818068818326
:10E30000C70105DF882361F0B601A5016A147B040B
:10E310008C049D0410F4B401A301C7012EDE01C0DA
:10E3200080E00F900F900F900F90CF91DF911F9191
:10E330000F91FF90EF90DF90CF90BF90AF909F90A4
:10E340008F907F906F900895F70181899289A389BA
:10E35000B48984179507A607B70708F058CFE0CF10
:10E36000CF93DF93EC0140E050E060E070E02EDFFF
:10E37000882359F0CE0161E0A9DEFC01009729F065
:10E3800085EE80831B8260D701C080E0DF91CF9152
:10E3900008952F923F924F925F926F927F928F9249
:10E3A0009F92AF92BF92CF92DF92EF92FF920F9324
:10E3B0001F93CF93DF93EC012A018B81882309F40B
:10E3C000B5C0898180FFB2C0C7C025014E185F0863
:10E3D0003B0174E0272E312C2C0E3D1E4201A0C0C3
:10E3E000288539854A855B856FEFA62E61E0B62EBC
:10E3F000A222B3228B8179018A0199E016950795B3
:10E40000F794E7949A95D1F7E98DFA8D823049F423
:10E41000428D538D648D758D4E0D5F1D601F711F74
:10E420003FC0D480DA94DE20A114B104D9F4DD20F9
:10E43000C9F4211531054105510549F48D899E899D
:10E44000AF89B88D8C839D83AE83BF830BC04C8115
:10E450005D816E817F81CF0191010E94917B882334
:10E4600009F464C0E98DFA8D4C815D816E817F81F4
:10E470004250504060407040058404C0440F551F16
:10E48000661F771F0A94D2F786859785A089B18980
:10E49000480F591F6A1F7B1F4D0D511D611D711DB6
:10E4A00080E092E08A199B0984018815990508F497
:10E4B0008C0182E00030180709F066C08091A50F3A
:10E4C0009091A60FA091A70FB091A80F48175907D8
:10E4D0006A077B0709F458C08091A9119091AA118D
:10E4E0009301EEDB882349F421C095012755304F75
:10E4F000C301B901A8010E94B4D4600E711E980135
:10E5000040E050E088859985AA85BB85820F931FDE
:10E51000A41FB51F88879987AA87BB87801A910A8D
:10E520008114910409F05CCFA20102C04FEF5FEFAC
:10E53000CA01DF91CF911F910F91FF90EF90DF9073
:10E54000CF90BF90AF909F908F907F906F905F9093
:10E550004F903F902F900895A988BA88CB88DC8887
:10E56000E884F9840A851B859A0140E050E0D601D1
:10E57000C5018E199F09A00BB10B281739074A074F
:10E580005B0708F022CF24CFCB01BA0140E097D639
:10E59000882309F0AACFCACFCF92DF92EF92FF92E1
:10E5A0000F931F93CF93DF937C01EB018A01FC0152
:10E5B0008381823008F46EC080859185A285B38501
:10E5C0008F719070A070B0700097A105B10509F02F
:10E5D00061C06CC0F8011082EDE0CE2ED12CC701D5
:10E5E000BE0140E250E0D5DE9C018032910521F071
:10E5F000009709F04FC050C04881442309F44CC033
:10E60000453E69F34E3259F38B858F738F30E9F5B0
:10E6100001151105D1F18A8D9B8D892BB1F5842FC0
:10E6200090E08F719070009781F1833091056CF5C7
:10E630008C9D90018D9D300D9C9D300D11242D5091
:10E640003040F801E20FF31F898180838B81818341
:10E650008D8182838F818383898584838E85858361
:10E66000888986838A8987838C8980878E89818738
:10E67000888D82878C8D83878E8D8487888186FFA5
:10E6800004C0F801E20FF31F15868B8583FDA7CF29
:10E69000822F03C08FEF01C080E0DF91CF911F91E7
:10E6A0000F91FF90EF90DF90CF90089541155105A5
:10E6B00009F090CF91CFDF93CF930F92CDB7DEB714
:10E6C000BE016F5F7F4F41E050E063DE019719F0BC
:10E6D0002FEF3FEF03C08981282F30E0C9010F9051
:10E6E000CF91DF910895EF92FF920F931F93CF93F5
:10E6F000DF93EC018B81823030F1E884F9840A8564
:10E700001B85CE01D8DF97FD1EC088859985AA8517
:10E71000BB854F96A11DB11D88879987AA87BB87A6
:10E72000A5E016950795F794E794AA95D1F72E2DB5
:10E7300030E02F703070F5E0220F331FFA95E1F7CB
:10E740002755304F02C020E030E0C901DF91CF9162
:10E750001F910F91FF90EF9008950F931F93CF9308
:10E76000DF93EC018B018B81882309F040C0FB0112
:10E770008789803109F041C082E08B831D8A1E8A1F
:10E780001F8A188E808D918DA0E0B0E045E0880F43
:10E79000991FAA1FBB1F4A95D1F7898B9A8BAB8B08
:10E7A000BC8B13C083E08B83F801428D538D648D45
:10E7B000758D4D8B5E8B6F8B788F9E012F5E3F4FDB
:10E7C000C8010E94627C882391F01A8F098F81E032
:10E7D00089831C821D821E821F82188619861A86D2
:10E7E0001B861C861D861E861F86188A01C080E037
:10E7F000DF91CF911F910F9108958032C1F7D2CF51
:10E800001F93CF93DF93EC01142F262F30E0F901F3
:10E8100075E0EE0FFF1F7A95E1F7E755F04F83851E
:10E82000817121F0842F827109F067C08091A50F5A
:10E830009091A60FA091A70FB091A80F8C879D87EC
:10E84000AE87BF87688BF90165E0EE0FFF1F6A9501
:10E85000E1F7E755F04F84899589A0E0B0E0DC014D
:10E86000992788278D8B9E8BAF8BB88F228D338D08
:10E87000A90160E070E0482B592B6A2B7B2B4D8B54
:10E880005E8B6F8B788F838590E088719070009796
:10E8900051F4848D958DA68DB78D898B9A8BAB8B1A
:10E8A000BC8B81E00CC0409741F59E012F5E3F4F2D
:10E8B000898D9A8D0E94627C8823F9F084E08B8395
:10E8C000812F8F7089831C821D821E821F82188671
:10E8D00019861A861B8614FF16C0CE0140E050E050
:10E8E00060E070E073DC882371F409C049895A89BB
:10E8F0006B897C89CE0141DB02C01B8280E0DF9105
:10E90000CF911F91089515FDF1CF81E0F8CF2F929F
:10E910003F924F925F926F927F928F929F92AF92AF
:10E92000BF92CF92DF92EF92FF920F931F93DF93EC
:10E93000CF930F92CDB7DEB72C015B013A014901AD
:10E9400000E010E0EE24EA94FE2C1E010894211C45
:10E95000311C11C00A0D1B1DF80160838114910444
:10E9600019F46A3039F41BC0C40170E00E94C8D4A5
:10E970000097A9F4860168010894C11CD11CC61433
:10E98000D7043CF5C201B10141E050E002DD7C0159
:10E9900081309105F1F469816D30E1F6ECCF8601AB
:10E9A000A00EB11EF5011082C8010F90CF91DF912A
:10E9B0001F910F91FF90EF90DF90CF90BF90AF909D
:10E9C0009F908F907F906F905F904F903F902F908F
:10E9D0000895F7FEE5CF0FEF1FEFE6CFCF93DF935C
:10E9E000EC019C012C5F3F4F898D9A8D41E050E0F6
:10E9F00060E070E0D2D78823A1F08D899E89AF892D
:10EA0000B88D0097A105B10559F48C819D81AE8127
:10EA1000BF818D8B9E8BAF8BB88F898180688983F6
:10EA200081E0DF91CF9108952F923F924F925F92B4
:10EA30007F928F929F92AF92BF92CF92DF92EF928E
:10EA4000FF920F931F93DF93CF9300D000D0CDB7E9
:10EA5000DEB76C01162F072F5E834D83DC01139602
:10EA60008C911397813009F069C111968C9181FFC7
:10EA700065C182C1F60141895289638974898085A3
:10EA80009185A285B38584179507A607B70729F056
:10EA9000C60173DA882309F451C1812F902F9C019C
:10EAA00019014D805E800FC1D6015996ED91FC9100
:10EAB0005A97DA01C90149E0B695A79597958795C8
:10EAC0004A95D1F774807A9478228FEF882E81E06E
:10EAD000982E82229322772009F051C0811491044C
:10EAE00009F04DC0D60114964D915D916D917C91C8
:10EAF0001797411551056105710581F455968D9162
:10EB00009D910D90BC91A02D0097A105B10559F1E3
:10EB1000F60184839583A683B78331C0CF019E011C
:10EB20002F5F3F4FFED5882309F408C129813A8120
:10EB30004B815C81D6015996ED91FC915A9787895A
:10EB4000803149F4283FBFEF3B07B0E04B07B0E00E
:10EB50005B0770F008C0283FEFEF3E07EFEF4E076E
:10EB6000EFE05E0728F0C60139DF882341F4E6C0F4
:10EB7000D60114962D933D934D935C93179780E0A7
:10EB800092E08819990952018415950508F45C01F1
:10EB9000D6015996ED91FC915A971496ED90FD90FF
:10EBA0000D911C9117978EEF9FEFAFEFBFEFE80E1F
:10EBB000F91E0A1F1B1F058404C0EE0CFF1C001F5A
:10EBC000111F0A94D2F786859785A089B189E80E2E
:10EBD000F91E0A1F1B1FE70CF11C011D111D90E0FF
:10EBE000A91692E0B90639F58091A50F9091A60F6C
:10EBF000A091A70FB091A80F8E159F05A007B10790
:10EC000071F41092AB118FEF9FEFAFEFBFEF8093D6
:10EC1000A50F9093A60FA093A70FB093A80F809174
:10EC2000A9119091AA11B801A70191010E94846DC8
:10EC30008823A9F583C08114910411F5D601189693
:10EC40002D913D914D915C911B9751968D919D9188
:10EC50000D90BC91A02D281739074A075B0780F05B
:10EC6000F3D2882309F46AC081E08093AB11E0926B
:10EC7000A50FF092A60F0093A70F1093A80F07C03F
:10EC8000C801B70141E01BD3882309F457C09401A0
:10EC90002755304FC901B101A5010E94B4D4950197
:10ECA00040E050E0F60180859185A285B385820F12
:10ECB000931FA41FB51F80879187A287B3872A0C53
:10ECC0003B1C4A185B08D60118962D913D914D9139
:10ECD0005C911B974114510409F0E6CE51968D9139
:10ECE0009D910D90BC91A02D82179307A407B507A5
:10ECF00048F4F601218B328B438B548B81818068E1
:10ED0000818311C08091A30F9091A40F892B59F09A
:10ED10008D819E81892B39F0D60111968C911197A6
:10ED2000806811968C93F601818183FF04C0C6012F
:10ED3000EED9882319F04D815E8105C081E0D601AE
:10ED40008C934FEF5FEFCA0126960FB6F894DEBFA3
:10ED50000FBECDBFCF91DF911F910F91FF90EF902C
:10ED6000DF90CF90BF90AF909F908F907F905F90FB
:10ED70004F903F902F90089582FD7CCE8ECEDF92F3
:10ED8000EF92FF920F931F93CF93DF93EC0189894A
:10ED90009A89AB89BC89805E9F4FAF41B04008F033
:10EDA0006FC0CE011BDE882309F46AC04DD28823D0
:10EDB00009F466C0E98DFA8DEC80FD800E811F811B
:10EDC0008EEF9FEFAFEFBFEFE80EF91E0A1F1B1F7C
:10EDD000058404C0EE0CFF1C001F111F0A94D2F71B
:10EDE00086859785A089B189E80EF91E0A1F1B1F29
:10EDF00081E08093AB11E092A50FF092A60F0093F3
:10EE0000A70F1093A80F80E092E0E9EAFFE0DF018E
:10EE10009C011D9221503040E1F7DD24D39411C0B4
:10EE2000B801A7014D0D511D611D711D8091A911E2
:10EE30009091AA1129EA3FE00E94846D882301F194
:10EE4000D394E98DFA8D8481D81650F320E032E016
:10EE500040E050E0058404C0220F331F441F551FBB
:10EE60000A94D2F789899A89AB89BC89820F931F4A
:10EE7000A41FB51F898B9A8BAB8BBC8B81E001C023
:10EE800080E0DF91CF911F910F91FF90EF90DF9085
:10EE900008958F929F92AF92BF92CF92DF92EF929E
:10EEA000FF920F931F93CF93DF936C01EB01942E8E
:10EEB000852EA22E898D9A8DD6015A969C938E937B
:10EEC0005997CB0140E050E060E070E056D8BB2499
:10EED00037C0CE0108DCFC01009709F48FC055E073
:10EEE00016950795F794E7945A95D1F71E2D1F7044
:10EEF0008081882311F0853EC9F4BB2099F42091CC
:10EF0000A50F3091A60F4091A70F5091A80FD601E1
:10EF10001C962D933D934D935C931F9750961C9395
:10EF2000BB24B3948081882359F418C0892D982D6F
:10EF3000BF014BE050E00E94A7D4009709F46CC0D9
:10EF4000E884F9840A851B8589899A89AB89BC89FB
:10EF5000E816F9060A071B0708F4BBCFA6FE4EC049
:10EF6000A1FE4CC0BB2049F0F6011089C60161E04A
:10EF7000ADD8EC01009761F441C08B81823009F477
:10EF80003DC0CE01FCDE8823C9F110E0C9EADFE014
:10EF900080E2DE011D928A95E9F7DE01292D382DE8
:10EFA000C901FC018BE001900D928150E1F7E091E5
:10EFB000A30FF091A40F309739F0BE01625F7F4F2D
:10EFC000CE014096199508C081E298E2998B888B12
:10EFD00080E098E09F878E87888999899B8B8A8BB0
:10EFE000998F888F8E859F859F8B8E8B2DD18823BF
:10EFF00029F0C601612F4A2D03DC01C080E0DF91BA
:10F00000CF911F910F91FF90EF90DF90CF90BF9025
:10F01000AF909F908F900895A7FEEBCFEFCF2F92E8
:10F020003F924F925F926F927F928F929F92AF9298
:10F03000BF92CF92DF92EF92FF920F931F93DF93D5
:10F04000CF93CDB7DEB7C654D0400FB6F894DEBF2D
:10F050000FBECDBF3C016B01DE01AE5BBF4F119611
:10F060005C934E9325962FAF25971C861F861FA273
:10F070001AA66115710509F47CC0FC0183818823FF
:10F0800009F077C0FA0180818F32F1F08601ECE05F
:10F09000EE2EF12CEC0EFD1E72E4A72EB12CAC0E60
:10F0A000BD1E4E010894811C911C2796FFAEEEAE4A
:10F0B000279767E2262E312C2C0E3D1E270123C0F8
:10F0C0001196B183A08301C0FD01A081B1818C9113
:10F0D0008F32B1F3D60113968C9113978250823000
:10F0E000A8F28E01095D1F4F59966D917C915A9738
:10F0F000C80133DB882359F63CC0342D252D870108
:10F10000832F922F7C01F50180819181B401A501AB
:10F110000E94756F882329F42CC03196D501ED9398
:10F12000FC93D501ED91FC9180818F32B1F388235E
:10F13000B9F0C701B801A40121E0ABDE8823C9F012
:10F140000C151D0511F0C80131D82796EEADFFADA5
:10F150002797EE16FF0689F6C101322D292FCFCF52
:10F16000C301B801A40125962FAD259792DE182F73
:10F1700001C010E0CE01879622D8CE010C961FD890
:10F18000812FCA5BDF4F0FB6F894DEBF0FBECDBF35
:10F19000CF91DF911F910F91FF90EF90DF90CF9073
:10F1A000BF90AF909F908F907F906F905F904F90A7
:10F1B0003F902F9008950F931F93DF93CF93CDB778
:10F1C000DEB76B970FB6F894DEBF0FBECDBF9C01C4
:10F1D000AB0119821C828E010F5F1F4FC801B9015C
:10F1E00022E01DDF882311F410E003C0C801B8D865
:10F1F000182FCE0101960E94DF70812F6B960FB6FB
:10F20000F894DEBF0FBECDBFCF91DF911F910F915C
:10F210000895DB010D900020E9F71197A61BB70BAD
:10F220000496AD0101CCDF93CF930F92CDB7DEB73B
:10F2300069830496BE016F5F7F4F41E050E0F4DBCD
:10F240000F90CF91DF9108958091AB11882399F1B0
:10F250004091A50F5091A60F6091A70F7091A80F34
:10F260008091A9119091AA1129EA3FE00E94846D32
:10F27000882319F14091AC115091AD116091AE11FC
:10F280007091AF11411551056105710591F08091A3
:10F29000A9119091AA1129EA3FE00E94846D882368
:10F2A00061F01092AC111092AD111092AE1110924B
:10F2B000AF111092AB1181E0089580E00895DF92C4
:10F2C000EF92FF920F931F937B018C01D42E8091BC
:10F2D000A50F9091A60FA091A70FB091A80F8E1522
:10F2E0009F05A007B107B9F0AFDF8823E1F0809157
:10F2F000A9119091AA11B801A70129EA3FE00E9443
:10F30000606E882381F0E092A50FF092A60F009323
:10F31000A70F1093A80FDD2011F481E011C081E048
:10F320008093AB110DC08FEF9FEFAFEFBFEF8093D6
:10F33000A50F9093A60FA093A70FB093A80F80E0FE
:10F340001F910F91FF90EF90DF9008958F929F9201
:10F35000AF92BF92CF92DF92EF92FF920F931F93E3
:10F36000CF93DF936C01142F7093AA116093A911AE
:10F37000FC01178A82E090E0A0E0B0E080839183F6
:10F38000A283B3831092AB111092AC111092AD1105
:10F390001092AE111092AF118FEF9FEFAFEFBFEF52
:10F3A0008093A50F9093A60FA093A70FB093A80FDB
:10F3B000442321F48824992454013FC0453008F0A7
:10F3C0001CC160E070E080E090E040E078DF8823DE
:10F3D00009F413C1C12FD0E02197FE0174E0EE0FB4
:10F3E000FF1F7A95E1F7E755F04FE254FE4F808119
:10F3F000EE5BF14090E08F779070892B09F0FDC0B3
:10F40000E653FE4F80819181A281B38184369105BC
:10F41000A105B10508F4F1C064E0CC0FDD1F6A95C9
:10F42000E1F7C159DE4E88809980AA80BB808114A3
:10F430009104A104B10409F4E0C0C501B40140E0A5
:10F440003EDF882309F4D9C08091B40F9091B50FA5
:10F450008050924009F0D1C02091B90F222309F4C5
:10F46000CCC08091B70F9091B80F892B09F4C5C01B
:10F470008091B60F882309F4C0C0F601228B8091D9
:10F48000B60F8483158661E070E007C04F5FF60118
:10F4900045874150483008F0B0C0F6014585848169
:10F4A00090E09B01042E02C0220F331F0A94E2F762
:10F4B0008217930759F72091BF0F3091C00F211584
:10F4C000310519F040E050E008C02091CD0F309197
:10F4D000CE0F4091CF0F5091D00FF6012583368388
:10F4E00047835087E090B70FF090B80F00E010E02E
:10F4F000E80CF91C0A1D1B1DE38AF48A058B168B88
:10F500008091BA0F9091BB0F918F808F6091B90F4E
:10F5100070E080E090E00E949DDC6E0D7F1D801FFA
:10F52000911FF601628F738F848F958F2091BA0F90
:10F530003091BB0F55E0220F331F5A95E1F7215050
:10F540003E4F232F3327269540E050E0260F371FEC
:10F55000481F591F26873787408B518B8091BC0FDE
:10F560009091BD0F009719F0A0E0B0E008C0809125
:10F57000C90F9091CA0FA091CB0FB091CC0F85010C
:10F580007401E21AF30A040B150BA8019701280F66
:10F59000391F4A1F5B1FF601058404C05695479525
:10F5A000379527950A94D2F7218732874387548766
:10F5B000253FFFE03F07F0E04F07F0E05F0720F452
:10F5C0008CE0F601878B19C0255F3F4F40405040CB
:10F5D00018F480E1F6010EC08091D50F9091D60FFE
:10F5E000A091D70FB091D80FF601828F938FA48F7F
:10F5F000B58F80E2878B81E001C080E0DF91CF9101
:10F600001F910F91FF90EF90DF90CF90BF90AF9040
:10F610009F908F9008956F927F928F929F92AF925A
:10F62000BF92CF92DF92EF92FF920F931F93CF93EF
:10F63000DF93EC015A016B01380149014230510559
:10F640006105710508F45DC089859A85AB85BC8527
:10F650000196A11DB11D84179507A607B70708F4E9
:10F6600050C08F89803129F4E52EF62E072F1127FF
:10F670000CC0803209F045C07A018B0187E01695F5
:10F680000795F794E7948A95D1F78B899C89AD8982
:10F69000BE89E80EF91E0A1F1B1FC801B70141E011
:10F6A0000EDE882371F18F89803149F4F501F07005
:10F6B000EE0FFF1FE755F04F718260820DC0F5011C
:10F6C000EF77F070EE0FFF1FEE0FFF1FE755F04FC3
:10F6D00060827182828293828A89823080F08D81F9
:10F6E0009E81AF81B885E80EF91E0A1F1B1FE092AC
:10F6F000AC11F092AD110093AE111093AF1181E0F7
:10F7000001C080E0DF91CF911F910F91FF90EF90AA
:10F71000DF90CF90BF90AF909F908F907F906F9031
:10F720000895CF92DF92EF92FF920F931F93CF93A2
:10F73000DF93EC017A018B01690189859A85AB859C
:10F74000BC850196A11DB11D84179507A607B707B3
:10F7500008F452C08F89803129F45527412F302F6A
:10F760002F2D0CC0803209F047C09A01AB0167E031
:10F7700056954795379527956A95D1F78B899C893A
:10F78000AD89BE89280F391F4A1F5B1F8091A50FC5
:10F790009091A60FA091A70FB091A80F2817390735
:10F7A0004A075B0731F0CA01B90140E088DD8823D0
:10F7B00019F18F89803159F4F701F070EE0FFF1FB6
:10F7C000E755F04F80819181A0E0B0E00EC0F701D5
:10F7D000EF77F070EE0FFF1FEE0FFF1FE755F04FB2
:10F7E00080819181A281B381BF70F6018083918372
:10F7F000A283B38381E001C080E0DF91CF911F91AC
:10F800000F91FF90EF90DF90CF900895AF92BF924D
:10F81000CF92DF92EF92FF920F931F93DF93CF93DC
:10F8200000D00F92CDB7DEB76C017A018B0182E078
:10F8300090E0A0E0B0E0F60180839183A283B383DF
:10F840005E010894A11CB11CC601B801A701950175
:10F8500068DF882339F1C601B801A70100E010E094
:10F8600020E030E0D8DE8823E9F0E980FA800B81DF
:10F870001C81F6018789803151F4F8EFEF16FFEF14
:10F88000FF06F0E00F07F0E01F07F0F209C088EF75
:10F89000E8168FEFF8068FEF08078FE01807A0F241
:10F8A00081E001C080E00F900F900F900F90CF91FA
:10F8B000DF911F910F91FF90EF90DF90CF90BF905D
:10F8C000AF9008954F925F926F927F928F929F9226
:10F8D000AF92BF92CF92DF92EF92FF920F931F935E
:10F8E000DF93CF9300D00F92CDB7DEB76C01498381
:10F8F0005A836B837C833901EE24FF2487012E0118
:10F900000894411C511C812CE2E09E2EA12CB12CAC
:10F9100049815A816B817C81C601920102DF882373
:10F9200039F1D501C401F601058404C0880F991F7F
:10F93000AA1FBB1F0A94D2F7E80EF91E0A1F1B1F4D
:10F9400029813A814B815C818789803131F4285F3C
:10F950003F4F40405040E0F205C0285F3F4F4F4FBF
:10F960005F40B0F2F301E082F1820283138381E011
:10F970000F900F900F900F90CF91DF911F910F91EB
:10F98000FF90EF90DF90CF90BF90AF909F908F90BF
:10F990007F906F905F904F9008952F923F924F927B
:10F9A0005F926F927F928F929F92AF92BF92CF920F
:10F9B000DF92EF92FF920F931F93DF93CF93CDB718
:10F9C000DEB72F970FB6F894DEBF0FBECDBF1C0178
:10F9D0004A875B876C877D873F872E87DC01199676
:10F9E0008D919D910D90BC91A02D0196A11DB11DF1
:10F9F0008E839F83A887B987F901008111812281B5
:10FA00003381011511052105310549F048015901DE
:10FA10000894811C911CA11CB11C1D8210C0D10135
:10FA20008D909D90AD90BC901D828A859B85AC8504
:10FA3000BD850197A105B10511F491E09D83750184
:10FA400064014424552432018E010F5F1F4FF101E0
:10FA500081859285A385B485481659066A067B067A
:10FA600008F08CC08E819F81A885B9858C159D0575
:10FA7000AE05BF0550F4A2E08A2E912CA12CB12C2A
:10FA8000F2E0CF2ED12CE12CF12CC101B701A6015F
:10FA9000980147DE882309F471C089819A81AB817E
:10FAA000BC81A70196012F5F3F4F4F4F5F4F0097DB
:10FAB000A105B10519F049015A010DC028193909EC
:10FAC0004A095B098A859B85AC85BD85281739075E
:10FAD0004A075B0759F00894411C511C611C711CBA
:10FAE0000894C11CD11CE11CF11CB1CFC101A601BD
:10FAF000B7010FEF1FEF2FEF3FE08DDD882391F46B
:10FB00003DC0260137010894410851086108710879
:10FB1000C101B301A201970186017DDD882371F146
:10FB2000730162018C149D04AE04BF0450F3AE85D2
:10FB3000BF854D915D916D917C9141155105610598
:10FB4000710531F0C1019501840165DD8823B1F0B3
:10FB5000EE85FF8580829182A282B382FD81FF23A0
:10FB600059F00894811C911CA11CB11CD1018D92EB
:10FB70009D92AD92BC92139781E001C080E02F96D8
:10FB80000FB6F894DEBF0FBECDBFCF91DF911F91AE
:10FB90000F91FF90EF90DF90CF90BF90AF909F902C
:10FBA0008F907F906F905F904F903F902F9008952F
:10FBB0001092E4111092E6111092E81108958093CA
:10FBC00084030895EFE6F0E08081826080830895E9
:10FBD0001F93FC011FB7F89480819181A281B381AA
:10FBE0008093BE119093BF11A093C011B093C11127
:10FBF000FB0180819181A281B3818093C211909396
:10FC0000C311A093C411B093C511FA0180819181F1
:10FC1000A281B3818093C6119093C711A093C8119C
:10FC2000B093C911F90180819181A281B381809340
:10FC3000CA119093CB11A093CC11B093CD111FBFDB
:10FC40001F910895FC012FB7F89480819181A281C2
:10FC5000B3818093CA119093CB11A093CC11B09330
:10FC6000CD112FBF0895E82F8FB7F894F0E0EE0F75
:10FC7000FF1FEE0FFF1FE254FE4E208131814281B3
:10FC800053818FBFB901CA01089580916F008D7FA4
:10FC900080936F0006C080918A0F8F5F8F70809372
:10FCA0008A0F9091890F80918A0F981751F41092C2
:10FCB000B1111092B01180916F00826080936F003B
:10FCC00008959091890F80918A0F981751F3E3CF8F
:10FCD0009B01882399F4B901882777FD8095982F97
:10FCE0002FEF30E040E050E00E949DDC20ED37E057
:10FCF00040E050E00E9411DD8CE214C08130A9F494
:10FD0000B901882777FD8095982F2FEF30E040E0EC
:10FD100050E00E949DDC20ED37E040E050E00E9482
:10FD200011DD8DE2B9010C94C31A8230A9F4B90136
:10FD3000882777FD8095982F2FEF30E040E050E046
:10FD40000E949DDC20ED37E040E050E00E9411DD94
:10FD50008EE2B9010C94C31A08958CE261E00E940E
:10FD6000A11B8DE261E00E94A11B8EE261E00E9476
:10FD7000A11B60917A0370917B0380E0A9DF609101
:10FD80007C0370917D0381E0A3DF60917E0370911D
:10FD90007F0382E09DDFE1E2F1E08081887F816086
:10FDA00080830895DADF099A3C9A399AEAE0F1E013
:10FDB0008081806480838081846080830D9A159A1D
:10FDC0003E9A469A3B9A439A389A409A808182603A
:10FDD00080839FB7F894EBE0F1E0808182608083BC
:10FDE0009FBF0898109A0C98149A0F98179A0B9A1C
:10FDF0001398159A3D9A4598469A3A9A4298439A8A
:10FE0000EAE0F1E08081806880839FB7F894EBE0BE
:10FE1000F1E080818F7780839FBF409AEAE0F1E034
:10FE20008081816080839FB7F894EBE0F1E080816E
:10FE30008E7F80839FBFA1E8B0E08C918F7E8C93F2
:10FE40008C9188608C93E0E8F0E080818D7F8083E6
:10FE500080818E7F808380818F73808380818F7C7F
:10FE600080838C91887F82608C9380E090E4909373
:10FE70008900809388001092850010928400EFE63C
:10FE8000F0E080818260808381E0809384037894B5
:10FE900008959091890F80918A0F981739F00E94E8
:10FEA000798B0E947A300E94CB94F3CF0895F1DFD2
:10FEB000159A469A439A409A08951F920F920FB648
:10FEC0000F920BB60F921124AF92BF92CF92DF9296
:10FED000EF92FF920F931F932F933F934F935F9354
:10FEE0006F937F938F939F93AF93BF93CF93DF9342
:10FEF000EF93FF938091B0119091B111892B09F08C
:10FF000094C19091890F80918A0F981719F4E0E0BD
:10FF1000F0E014C080918A0F90E02DE430E0829FE1
:10FF2000F001839FF00D929FF00D1124E754F54FDF
:10FF3000E45BFF4F81E08083EC54F040F093B1111B
:10FF4000E093B011309709F46AC1E45BFF4F81E0A0
:10FF50008083EC54F0401092F0111092F111109245
:10FF6000F2111092F31160AD71AD2CE9613472079A
:10FF700018F060E47CE904C03EE46132730730F0BD
:10FF8000769567957695679584E007C047E261317D
:10FF9000740730F07695679582E08093E91107C089
:10FFA0008093E9116032710510F460E270E06052F4
:10FFB000704058E060307507E8F0472F50E0440F7C
:10FFC000551F440F551F495F524F9A012E5F3F4FF7
:10FFD000F901859194919C01AA27639FC001629FBA
:10FFE000810D9A1F06948A1F9A1F1124FA014591C8
:10FFF00054911EC0CB01969587958C7F895F9E4E4C
:020000021000EC
:10000000FC0145915491FC01329625913491862F43
:1000100090E087709070FC012E9FC0012F9F900D83
:100020003E9F900D1124B3E096958795BA95E1F720
:10003000481B590B44365105A8F4E0EEF2E007C026
:100040008091C00085FFFCCF31969093C6009081CF
:100050009923B1F784E49AE04AE050E00E946D569B
:1000600044E650E05093F5114093F4118091E9116A
:100070008093F6111092F711E091B011F091B11147
:1000800064AD75AD7093EF116093EE11FCE96134CE
:100090007F0718F060E47CE904C02EE46132720747
:1000A00030F0769567957695679584E007C037E2DE
:1000B0006131730730F07695679582E08093E9119E
:1000C00008C081E08093E9116032710510F460E2AC
:1000D00070E06052704048E060307407E8F0472FED
:1000E00050E0440F551F440F551F495F524F9A016E
:1000F0002E5F3F4FF901859194919C01AA27639F40
:10010000C001629F810D9A1F06948A1F9A1F1124B5
:10011000FA01459154911EC0CB01969587958C7F2D
:10012000895F9E4EFC0145915491FC0132962591C8
:100130003491862F90E087709070FC012E9FC00153
:100140002F9F900D3E9F900D112433E0969587953B
:100150003A95E1F7481B590B44365105A8F4E0EEF7
:10016000F2E007C08091C00085FFFCCF31969093EC
:10017000C60090819923B1F784E49AE04AE050E008
:100180000E946D5644E650E0CA01A0E0B0E08093C2
:10019000EA119093EB11A093EC11B093ED115093F1
:1001A000890040938800E091B011F091B1118089ED
:1001B0009189A289B389B695A79597958795B095AA
:1001C000A095909581959F4FAF4FBF4F8093CE11D3
:1001D0009093CF11A093D011B093D1118093D211ED
:1001E0009093D311A093D411B093D5118093D611CD
:1001F0009093D711A093D811B093D9118093DA11AD
:100200009093DB11A093DC11B093DD111092DE11FD
:100210001092DF111092E0111092E11106C080EDF2
:1002200097E09093890080938800C091B011D0919D
:10023000B111209709F489C488A18093E21180FF4D
:1002400003C0119A8FEF02C0119881E08093800360
:100250008091E21181FF03C044988FEF02C0449A5D
:1002600081E0809381038091E21180FF36C080910C
:100270008403882391F120B1217031E0232759F1C3
:100280008091E311882339F188819981AA81BB810A
:10029000181619061A061B06F4F48091BE119091E7
:1002A000BF11A091C011B091C1118093B211909370
:1002B000B311A093B411B093B5113093E4118889B0
:1002C0009989AA89BB898093DE119093DF11A0934D
:1002D000E011B093E1112093E3118091E21181FDCF
:1002E0003AC0809184038823B1F180B182958F70E8
:1002F0008095282F217080FF2CC08091E5118823E4
:1003000041F18C819D81AE81BF81181619061A06B4
:100310001B06FCF48091C2119091C311A091C411ED
:10032000B091C5118093B6119093B711A093B811F5
:10033000B093B91181E08093E61188899989AA89DF
:10034000BB898093DE119093DF11A093E011B093ED
:10035000E1112093E5118091E21182FF05C0419ADD
:100360008FEF8093820339C0419881E080938203AC
:1003700080918403882389F120E007992CC021E033
:100380008091E711882339F188859985AA85BB85F5
:10039000181619061A061B06F4F48091C6119091DE
:1003A000C711A091C811B091C9118093BA1190934F
:1003B000BB11A093BC11B093BD112093E8118889A3
:1003C0009989AA89BB898093DE119093DF11A0934C
:1003D000E011B093E1112093E7118091E21183FFC6
:1003E0000AC08FB7F89490910B019F7B90930B01FB
:1003F0008FBF8FEF09C08FB7F89490910B01906475
:1004000090930B018FBF81E08093830360E070E0E5
:1004100079C18091C00087FF19C04091C600E0916A
:10042000400AF091410A31969F012F773070319741
:100430008091420A9091430A2817390739F0E05415
:10044000F64F40833093410A2093400A2881398136
:100450004A815B818091CE119091CF11A091D011F2
:10046000B091D111280F391F4A1F5B1F2093CE1165
:100470003093CF114093D0115093D111121613061F
:10048000140615066CF5139A88899989AA89BB897F
:10049000281B390B4A0B5B0B2093CE113093CF11E5
:1004A0004093D0115093D1112091BE113091BF11C2
:1004B0004091C0115091C11180918003992787FD0F
:1004C0009095A92FB92F820F931FA41FB51F80935A
:1004D000BE119093BF11A093C011B093C111139896
:1004E0002C813D814E815F818091D2119091D311F9
:1004F000A091D411B091D511280F391F4A1F5B1F4D
:100500002093D2113093D3114093D4115093D5112D
:1005100012161306140615066CF5459A88899989F2
:10052000AA89BB89281B390B4A0B5B0B2093D2117C
:100530003093D3114093D4115093D5112091C2110F
:100540003091C3114091C4115091C5118091810324
:10055000992787FD9095A92FB92F820F931FA41F6C
:10056000B51F8093C2119093C311A093C411B0938F
:10057000C5114598288539854A855B858091D611B6
:100580009091D711A091D811B091D911280F391F8E
:100590004A1F5B1F2093D6113093D7114093D81177
:1005A0005093D91112161306140615066CF5429ACB
:1005B00088899989AA89BB89281B390B4A0B5B0B4F
:1005C0002093D6113093D7114093D8115093D9115D
:1005D0002091C6113091C7114091C8115091C91195
:1005E00080918203992787FD9095A92FB92F820FBB
:1005F000931FA41FB51F8093C6119093C711A0939A
:10060000C811B093C91142982C853D854E855F85F0
:100610008091DA119091DB11A091DC11B091DD1184
:10062000280F391F4A1F5B1F2093DA113093DB110B
:100630004093DC115093DD111216130614061506B3
:10064000DCF59FB7F89480910B01806880930B01D3
:100650009FBF88899989AA89BB89281B390B4A0BB6
:100660005B0B2093DA113093DB114093DC11509334
:10067000DD112091CA113091CB114091CC115091D4
:10068000CD1180918303992787FD9095A92FB92FCC
:10069000820F931FA41FB51F8093CA119093CB1193
:1006A000A093CC11B093CD119FB7F89480910B011A
:1006B0008F7780930B019FBF8091DE119091DF11A6
:1006C000A091E011B091E1110196A11DB11D80939F
:1006D000DE119093DF11A093E011B093E11120910E
:1006E000DE113091DF114091E0115091E1116F5F07
:1006F0007F4F88899989AA89BB89281739074A07B2
:100700005B0738F48091E91190E0681779070CF4E1
:1007100080CE2091DE113091DF114091E011509197
:10072000E1118C899D89AE89BF8982179307A4073F
:10073000B50708F4E3C0E090EA11F090EB110091E6
:10074000EC111091ED11AC8CBD8CCE8CDF8CA8011E
:100750009701C601B501AA27279FB12D389FF00147
:10076000489FF00D479FE00DF11D289FB00DE11D42
:10077000FA1F379FB00DE11DFA1F469FB00DE11D16
:10078000FA1F369FB10DEA1FFA1FB695EA1FFA1F2E
:1007900011248CAD9DAD8E0F9F1F9093EF11809310
:1007A000EE1128AD39AD4AAD5BADA0E0B0E0281741
:1007B00039074A075B0720F43093EF112093EE11BD
:1007C0006091EE117091EF118CE96134780718F0A7
:1007D00060E47CE904C09EE46132790730F07695EC
:1007E00067957695679584E007C0E7E261317E07FB
:1007F00030F07695679582E08093E91108C081E03A
:100800008093E9116032710510F460E270E060528B
:100810007040F8E060307F07E8F0472F50E0440F69
:10082000551F440F551F495F524F9A012E5F3F4F8E
:10083000F901859194919C01AA27639FC001629F51
:10084000810D9A1F06948A1F9A1F1124FA0145915F
:1008500054911EC0CB01969587958C7F895F9E4EE3
:10086000FC0145915491FC01329625913491862FDB
:1008700090E087709070FC012E9FC0012F9F900D1B
:100880003E9F900D1124B3E096958795BA95E1F7B8
:10089000481B590B44365105A8F4E0EEF2E007C0BE
:1008A0008091C00085FFFCCF31969093C600908167
:1008B0009923B1F784E49AE04AE050E00E946D5633
:1008C00044E650E050938900409388009A0140E04C
:1008D00050E08091EA119091EB11A091EC11B09150
:1008E000ED11820F931FA41FB51F8093EA119093FF
:1008F000EB11A093EC11B093ED1102C12091DE1128
:100900003091DF114091E0115091E111888D998D66
:10091000AA8DBB8D82179307A407B50708F0E4C022
:100920006091F0117091F1118091F2119091F31199
:100930002C8D3D8D4E8D5F8DAA27639FB12D749FA9
:10094000F001849FF00D839FE00DF11D649FB00DB9
:10095000E11DFA1F739FB00DE11DFA1F829FB00DBC
:10096000E11DFA1F729FB10DEA1FFA1FB695EA1F2B
:10097000FA1F11248091EE119091EF118E179F07AD
:1009800038F4C05CDF4F68817981C054D04003C027
:10099000BC016E1B7F0BC05CDF4F288139814A810F
:1009A0005B81CB01A0E0B0E082179307A407B507F5
:1009B00008F4B901FCE961347F0718F060E47CE9D0
:1009C00004C02EE46132720730F076956795769513
:1009D000679584E007C037E26131730730F07695A0
:1009E000679582E08093E91108C081E08093E91166
:1009F0006032710510F460E270E06052704048E0CF
:100A000060307407E8F0472F50E0440F551F440F43
:100A1000551F495F524F9A012E5F3F4FF901859153
:100A200094919C01AA27639FC001629F810D9A1F28
:100A300006948A1F9A1F1124FA01459154911EC0F1
:100A4000CB01969587958C7F895F9E4EFC014591E1
:100A50005491FC01329625913491862F90E0877055
:100A60009070FC012E9FC0012F9F900D3E9F900D16
:100A7000112423E0969587952A95E1F7481B590B99
:100A800044365105A8F4E0EEF2E007C08091C000C2
:100A900085FFFCCF31969093C60090819923B1F7E2
:100AA00084E49AE04AE050E00E946D5644E650E04B
:100AB00050938900409388009A0140E050E0809173
:100AC000F0119091F111A091F211B091F311820FF8
:100AD000931FA41FB51F8093F0119093F111A09361
:100AE000F211B093F3110CC08091F4119091F511B3
:100AF00090938900809388008091F6118093E9118A
:100B00002091DE113091DF114091E0115091E111FF
:100B1000E091B011F091B11180899189A289B389D6
:100B2000281739074A075B0780F01092B11110921D
:100B3000B0119091890F80918A0F981731F08091B0
:100B40008A0F8F5F8F7080938A0FFF91EF91DF91F3
:100B5000CF91BF91AF919F918F917F916F915F9155
:100B60004F913F912F911F910F91FF90EF90DF9048
:100B7000CF90BF90AF900F900BBE0F900FBE0F9015
:100B80001F9018958091E411882349F48091E61113
:100B9000882329F48091E811882309F490C0E7E0C4
:100BA000F5E1949108C08091C00085FFFCCF90933F
:100BB000C600319694919923B1F7E9E1F5E194915A
:100BC00008C08091C00085FFFCCF9093C60031968D
:100BD00094919923B1F78091E4118823D1F0609129
:100BE000B2117091B3118091B4119091B5110E941E
:100BF000C3D62091590A30915A0A40915B0A50910C
:100C00005C0A0E9428D6AB01BC0185E195E10E94F7
:100C100011348091E6118823D1F06091B611709162
:100C2000B7118091B8119091B9110E94C3D620914B
:100C30005D0A30915E0A40915F0A5091600A0E94FD
:100C400028D6AB01BC0181E195E10E94113480916D
:100C5000E8118823D1F06091BA117091BB11809195
:100C6000BC119091BD110E94C3D62091610A3091B0
:100C7000620A4091630A5091640A0E9428D6AB012F
:100C8000BC018DE095E10E941134E4EFF2E007C071
:100C90008091C00085FFFCCF31969093C600908173
:100CA0009923B1F78091C00085FFFCCF8AE0809343
:100CB000C6001092E4111092E6111092E811089506
:100CC00060E070E08FE793E42091890330918A031C
:100CD00040918B0350918C030E9428D660932C1274
:100CE00070932D1280932E1290932F1260E070E07B
:100CF0008FE793E42091990330919A0340919B03ED
:100D000050919C030E9428D6609334127093351240
:100D100080933612909337120895FC0197FF03C019
:100D20008091091203C0E85FFD4E808190E0089534
:100D30002F923F924F925F926F927F928F929F92EB
:100D4000AF92BF92CF92DF92EF92FF920F931F93D9
:100D5000CF93DF93EC0121E030E0A901440F551F50
:100D6000440F551FFA01E052FA4E85919491C8172D
:100D7000D9070CF059C0B90161507040660F771F58
:100D8000660F771FCB018E519A4EFC01059114918D
:100D900060527A4EFB01C590D490FA01EE51FA4EA2
:100DA000E590F490FA01E052FA4EA590B490B801A3
:100DB000882777FD8095982F0E94C3D61B012C01B0
:100DC000CC19DD09BE01882777FD8095982F0E94F8
:100DD000C3D63B014C01E01AF10A0027F7FC00954D
:100DE000102FC801B7010E94C3D69B01AC01C401FA
:100DF000B3010E94F6D87B018C01AC18BD08CC244D
:100E0000B7FCC094DC2CC601B5010E94C3D69B017F
:100E1000AC01C801B7010E9428D69B01AC01C201F8
:100E2000B1010E9448D519C0822F8F5F2F5F3F4FBD
:100E30002133310509F091CF813329F0E0E070E0F2
:100E400080E060E00CC0E2EAF6E1659174918827E9
:100E500077FD8095982F0E94C3D6E62F692F2E2FFD
:100E6000372F482F562FB901CA01DF91CF911F911B
:100E70000F91FF90EF90DF90CF90BF90AF909F9039
:100E80008F907F906F905F904F903F902F9008953C
:100E900008951092F9111092F81110920812749896
:100EA0001092FB111092FA111092091280E090E05A
:100EB000A0E0B0E08093201290932112A093221220
:100EC000B09323128093241290932512A09326129C
:100ED000B0932712A59808952DEB37E346E05EE323
:100EE0000C94F6D82DEB37E346E05EE30C9428D65D
:100EF0002DEB37E346E05EE30C9428D62DEB37E389
:100F000046E05EE30C94F6D8A5980E94A62F8823AD
:100F100019F5E8E2F5E1949108C08091C00085FFE1
:100F2000FCCF9093C600319694919923B1F7EFE2EC
:100F3000F5E1949108C08091C00085FFFCCF9093AB
:100F4000C600319694919923B1F78091C00085FF36
:100F5000FCCF8AE08093C60083E00C94E22F1F93BD
:100F6000182F97DF0E94A62F882391F5E8E2F5E17C
:100F7000949108C08091C00085FFFCCF9093C6007B
:100F8000319694919923B1F784E49AE0612F70E04F
:100F90004AE050E00E9446568091C00085FFFCCF99
:100FA0008AE08093C600E9E6F5E1949108C080915B
:100FB000C00085FFFCCF9093C60031969491992391
:100FC000B1F78091C00085FFFCCF8AE08093C60016
:100FD00082E00E94E22F1F9108951F93182F59DF7E
:100FE0000E94A62F882391F5E8E2F5E1949108C0CC
:100FF0008091C00085FFFCCF9093C60031969491FC
:101000009923B1F784E49AE0612F70E04AE050E060
:101010000E9446568091C00085FFFCCF8AE08093F5
:10102000C600E6E9F5E1949108C08091C00085FF13
:10103000FCCF9093C600319694919923B1F780919B
:10104000C00085FFFCCF8AE08093C60081E00E944B
:10105000E22F1F9108951F920F920FB60F920BB6B9
:101060000F9211242F933F934F935F936F937F932E
:101070008F939F93AF93BF93EF93FF939091A503AB
:10108000992361F48091081280930E128111749A51
:101090008091091280930D128111A59A80910E12F0
:1010A000981708F0749880910D12981708F0A59879
:1010B0009F5F9F779093A5038091A603843009F4E6
:1010C00071C0853050F4813021F1813098F0823048
:1010D000F1F1833009F07AC049C0863009F468C064
:1010E000863008F463C0873009F466C0883009F0A0
:1010F0006DC06AC088E080937B0080E480937C00B0
:1011000080917A00806480937A000E948A9281E0C4
:101110001BC08091780090917900A0E0B0E0209110
:101120001B1230911C1240911D1250911E12280F5B
:10113000391F4A1F5B1F20931B1230931C124093D0
:101140001D1250931E1282E08093A6033FC088E0D8
:1011500080937B0082E480937C0080917A0080649D
:1011600080937A000E948A9283E0EECF809178008B
:1011700090917900A0E0B0E020910F123091101210
:101180004091111250911212280F391F4A1F5B1FF4
:1011900020930F1230931012409311125093121299
:1011A00084E0D2CF0E948A9285E0CECF86E0CCCF79
:1011B0000E948A9287E0C8CF1092A60380911F12E6
:1011C0008F5F80931F1202C01092A60380911F129E
:1011D000803108F463C080910A12882381F48091E1
:1011E0001B1290911C129093FD118093FC11809121
:1011F0000F1290911012909303128093021281E0CB
:1012000080930A1210921F1210921B1210921C123D
:1012100010921D1210921E12109217121092181294
:101220001092191210921A12109213121092141294
:10123000109215121092161210920F121092101294
:1012400010921112109212122091FC113091FD1186
:101250008091A1039091A2032817390714F080E030
:10126000BCDE2091FC113091FD1180910B12909108
:101270000C128217930714F080E071DE20910212A5
:10128000309103128091A3039091A403281739078A
:101290002CF01092FB111092FA1136DEFF91EF91B3
:1012A000BF91AF919F918F917F916F915F914F917E
:1012B0003F912F910F900BBE0F900FBE0F901F907C
:1012C00018952F926F927F928F929F92AF92BF92BA
:1012D000CF92DF92EF92FF920F931F93DF93CF9302
:1012E000CDB7DEB729970FB6F894DEBF0FBECDBFDE
:1012F0008C01E62E662369F1E8E2F5E1949108C0DD
:101300008091C00085FFFCCF9093C60031969491E8
:101310009923B1F784E49AE06E2D70E04AE050E042
:101320000E944656E3ECF5E1949108C08091C0001C
:1013300085FFFCCF9093C600319694919923B1F725
:101340008091C00085FFFCCF8AE08093C6000E9498
:101350002230AE2DB0E0FD01EE0FFF1FE25EFB4F2D
:101360006081718179876887672B09F49FC0A05ECF
:10137000BB4F7C917B832224239479C0222D30E0C3
:10138000A901440F551F440F551FE885F985E40F47
:10139000F51F85919491081719070CF067C0C901D2
:1013A0000197880F991F880F991FFC013296A88515
:1013B000B985EA0FFB1FC590D4908A0F9B1FFC01D3
:1013C000659174917A836983FA013296EA0FFB1F63
:1013D000E590F490FD01E40FF51FA590B490B601DF
:1013E000882777FD8095982F0E94C3D66C837D83D4
:1013F0008E839F8389819A81081B190BB8018827E6
:1014000077FD8095982F0E94C3D63B014C01EC18C4
:10141000FD080027F7FC0095102FC801B7010E94B6
:10142000C3D69B01AC01C401B3010E94F6D87B0175
:101430008C01A981BA81AA1ABB0ACC24B7FCC0943A
:10144000DC2CC601B5010E94C3D69B01AC01C801CA
:10145000B7010E9428D69B01AC016C817D818E81F1
:101460009F810E9448D5E62F692F09C02394BB8134
:101470002B1608F483CFE0E070E080E060E0FB81B1
:101480002F1679F5E22DF0E0EE0FFF1FEE0FFF1F94
:10149000329768857985E60FF71F659174918827E3
:1014A00077FD8095982F0E94C3D619C0B801882770
:1014B00077FD8095982F0E94C3D620E030E04AEF58
:1014C0005EE30E94F6D820E030E040E85DE30E9451
:1014D000F6D820E030E040E050E00E9448D5E62F0A
:1014E000692F2E2F372F482F562FB901CA01299661
:1014F0000FB6F894DEBF0FBECDBFCF91DF911F9125
:101500000F91FF90EF90DF90CF90BF90AF909F90A2
:101510008F907F906F902F900895EF92FF920F938E
:101520001F93CF93DF930F2EF0E0EF2EF0E0FF2E0E
:10153000F0E00F2FF0E01F2FF02DE0922812F09234
:10154000291200932A1210932B1260E070E08FE7AB
:1015500093E42091890330918A0340918B03509149
:101560008C030E9428D660932C1270932D128093C6
:101570002E1290932F12E0923012F09231120093BB
:1015800032121093331260E070E08FE793E4209101
:10159000990330919A0340919B0350919C030E94C0
:1015A00028D660933412709335128093361290933C
:1015B00037126C9A6D9A9D9A809101018061809397
:1015C000010187ED80937A0010927E0010927D00D9
:1015D00080917D00816080937D0080917D0082609C
:1015E00080937D0080917D00846080937D0080E801
:1015F00088BD80916E00846080936E0085E090E0ED
:10160000909339128093381209C080910B129091F7
:101610000C12409690930C1280930B1280910B1237
:1016200090910C1260E04DDE20E030E040EA50E4A2
:101630000E9421D687FDE9CF83E191E09093A80332
:101640008093A70309C08091A1039091A2034097C2
:101650009093A2038093A1038091A1039091A20390
:1016600060E02FDE20E030E849E853E40E9424D80F
:1016700018164CF3C091A303D091A403EC2E1D2F98
:10168000CE0156DB609720E030E048E453E40E944E
:1016900024D818169CF3E092A3031093A403DF91BF
:1016A000CF911F910F91FF90EF9008958091FC11C1
:1016B0009091FD1160E005DE6093FE117093FF11C3
:1016C0008093001290930112809102129091031264
:1016D0002FDB60930412709305128093061290938F
:1016E00007120E9465D18FB7F89410920A128FBF2B
:1016F00008952F923F924F925F926F927F928F92B6
:101700009F92AF92BF92CF92DF92EF92FF920F9390
:101710001F9380910A12882309F46EC2C7DF60907C
:10172000FE117090FF118090001290900112C090F5
:10173000F811D090F911B601882777FD8095982F80
:101740000E94C3D6A40193010E9447D57B018C015E
:1017500060933A1270933B1280933C1290933D1227
:1017600020E030E04AE754E40E9424D8181624F41C
:1017700081E080933E12E9C0C801B70120E030E06B
:101780004AE754EC0E9421D687FD02C0CD2821F4FF
:1017900081E080933E12C4C080913E12882371F094
:1017A00080E090E0A0E0B0E080933F129093401280
:1017B000A0934112B093421210923E12C801B70199
:1017C00020918503309186034091870350918803CF
:1017D0000E94F6D81B012C016093431270934412AF
:1017E0008093451290934612C801B70120913F1291
:1017F0003091401240914112509142120E9448D5BE
:101800005B016C01E0902812F090291200912A12DD
:1018100010912B12A80197010E9421D687FD12C0BA
:10182000E0902C12F0902D1200912E1210912F1298
:10183000C601B501A80197010E9424D8181614F01A
:1018400086017501E0923F12F0924012009341121E
:1018500010934212C801B7012091890330918A0385
:1018600040918B0350918C030E94F6D85B016C0170
:1018700060934712709348128093491290934A12D2
:10188000C401B30120914B1230914C1240914D1282
:1018900050914E120E9447D520918D0330918E03B6
:1018A00040918F03509190030E94F6D820E037EDCD
:1018B00043E25CE30E94F6D87B018C0160914F12F9
:1018C00070915012809151129091521224EA30E797
:1018D0004DE75FE30E94F6D89B01AC01C801B70158
:1018E0000E9448D57B018C0160934F127093501277
:1018F0008093511290935212C201B101A601950139
:101900000E9448D5A80197010E9447D57B018C0110
:1019100020E030E040E050E00E9421D688235CF4D3
:101920000F2EF0E0EF2EF0E0FF2EF0E00F2FF0E0B2
:101930001F2FF02D14C0C801B70120E030E04FE7A1
:1019400053E40E9424D8181654F40F2EF0E0EF2E22
:10195000F0E0FF2EFFE70F2FF3E41F2FF02D609232
:101960004B1270924C1280924D1290924E126091D6
:10197000381270913912882777FD8095982F0E9430
:10198000C3D69B01AC01C401B3010E9424D8181630
:10199000DCF46091A7037091A803882777FD8095F8
:1019A000982F0E94C3D69B01AC01C401B3010E94D1
:1019B00021D688234CF4C801B7010E9490D67595B2
:1019C00067956093081202C010920812609004128A
:1019D0007090051280900612909007126091FA1193
:1019E0007091FB11882777FD8095982F0E94C3D6B0
:1019F000A40193010E9447D57B018C01609353128F
:101A0000709354128093551290935612209195031F
:101A10003091960340919703509198030E94F6D815
:101A20001B012C01609320127093211280932212CB
:101A300090932312C801B701209157123091581288
:101A40004091591250915A120E9448D55B016C0185
:101A5000E0903012F0903112009132121091331256
:101A6000A80197010E9421D687FD12C0E090341290
:101A7000F09035120091361210913712C601B5015F
:101A8000A80197010E9424D8181614F08601750148
:101A9000E0925712F09258120093591210935A1272
:101AA000C801B7012091990330919A0340919B039B
:101AB00050919C030E94F6D85B016C016093241244
:101AC000709325128093261290932712C401B301BC
:101AD00020915B1230915C1240915D1250915E1228
:101AE0000E9447D520919D0330919E0340919F0312
:101AF0005091A0030E94F6D820E037ED43E25CE36A
:101B00000E94F6D87B018C0160915F127091601287
:101B1000809161129091621224EA30E74DE75FE311
:101B20000E94F6D89B01AC01C801B7010E9448D5BC
:101B30007B018C0160935F1270936012809361123D
:101B40009093621260925B1270925C1280925D12AE
:101B500090925E12C201B101A60195010E9448D582
:101B6000A80197010E9447D57B018C0120E030E05D
:101B700040E050E00E9421D688235CF40F2EF0E074
:101B8000EF2EF0E0FF2EF0E00F2FF0E01F2FF02DF2
:101B900014C0C801B70120E030E04FE753E40E94D1
:101BA00024D8181654F40F2EF0E0EF2EF0E0FF2E9C
:101BB000FFE70F2FF3E41F2FF02DC401B30120E046
:101BC00030E040EA50E40E9424D818169CF4C40186
:101BD000B30120E030E048E453E40E9421D688239A
:101BE0004CF4C801B7010E9490D675956795609333
:101BF000091202C0109209121F910F91FF90EF90ED
:101C0000DF90CF90BF90AF909F908F907F906F901C
